:100000000C940E090C942D090C942D090C94370CAA
:100010000C946D0C0C942D090C942D090C942D0945
:100020000C942D090C942D090C942D090C942D0978
:100030000C942D090C942D090C942D090C940E1080
:100040000C942D090C942D090C942D090C942D0958
:100050000C94AF5F0C94BB560C942D090C942D0995
:100060000C942D090C9491570C942D090C948557E0
:100070000C942D090C942D090C942D090C942D0928
:100080000C94626C0C942D090C942D090C942D0980
:100090000C94CF570C942D090C94C3570C942D0934
:1000A0000C942D090C942D090C942D090C942D09F8
:1000B0000C942D090C942D090C942D090C942D09E8
:1000C0000C942D090C942D090C942D090C942D09D8
:1000D0000C942D090C942D090C942D090C942D09C8
:1000E0000C942D090C94685F0C94725F0C945E5F05
:1000F0000C94185F0C94A35F0C94945F0C94885F2D
:100100000C947C5F0C942D090C942D090C942D09F2
:100110000C942D090C942D090C942D090C942D0987
:10012000084AD73B3BCE016E84BCBFFDC12F3D6C5E
:1001300074319ABD56833DDA3D00C77F11BED9E4C4
:10014000BB4C3E916BAAAABE000000803F076342F1
:1001500036B79BD8A71A39685618AEBAAB558C1D5E
:100160003CB7CC5763BD6DEDFD753EF6177231BFE0
:10017000000000803F08000000BE922449123EAB00
:10018000AAAA2ABECDCCCC4C3E00000080BEABAAB1
:10019000AAAA3E00000000BF000000803F0000004F
:1001A0000000084178D3BB4387D1133D190E3CC3EF
:1001B000BD4282AD2B3E68EC8276BED98FE1A93E6E
:1001C0004C80EFFFBE01C4FF7F3F000000000050E5
:1001D0003A20256C642050612020252D372E326670
:1001E000206D0A002563002563004932433A200050
:1001F00025630074746C3D252D64200074746C3D7F
:10020000252D6420004E65772074746C3D252D6487
:100210002000256300256C642050612020252D37A7
:100220002E3266206D00256C64204320002563007B
:10023000545F52483D252D342E3166200052483DF2
:10024000252D342E316620002563002563002563AB
:100250000025630043757272656E74207265706F5D
:10026000727420696E74657276616C3D252D642010
:100270007365630A004E6577207265706F72742033
:10028000696E74657276616C3D252D6420736563BB
:100290000A002563005573696E67207265706F727E
:1002A000743D3078252D6C7820004E65772072657E
:1002B000706F72743D3078252D6C782000256300B6
:1002C000256300256300256300204F534343414CC1
:1002D0003D2564200020467573653A2065653D25FF
:1002E0003032782068663D25303278206C663D25B6
:1002F000303278206C623D25303278004D43553DD8
:100300002530366C7800256300252D31306C752042
:10031000252D31306C7520252D31306C7520252D23
:1003200031306C75200A007478206C656E202020B6
:1003300020207268206D697373202020207268204D
:100340007374616C652020207268206D6973630A84
:10035000002563004F4B0A002563002563002563D9
:100360000025630025630052454C41593D09093081
:100370007825780A00434F4D504153533D0930785A
:1003800025780A00414343454C3D090930782578DA
:100390000A00505245533D0909307825780A00502B
:1003A0005F5057523D0909307825780A004145537E
:1003B0003D0909307825780A0050315F4C45443DAD
:1003C0000909307825780A0050305F4C45443D09D2
:1003D00009307825780A004556454E543D090930C4
:1003E0007825780A004C45443D0909307825780A7B
:1003F000004F573D0909307825780A00504B543D8D
:100400000909307825780A0054583D0909307825C3
:10041000780A0052583D0909307825780A004F5073
:1004200045523D0909307825780A00437572726596
:100430006E742064656275673D307825580A004EF9
:1004400065772064656275673D307825580A002518
:10045000730A0025372E33662025372E3366002594
:10046000352E326620004572726F72203020566F32
:100470006C74004E6F7420737570706F7274656465
:100480000A004572726F72203020566F6C740045FE
:1004900072726F72203020566F6C740025730A00E0
:1004A00073656E743D252D75206475703D252D7521
:1004B0002069676E6F7265643D252D752074746CBC
:1004C0005F7A65726F3D252D750A00545820506F74
:1004D0007765723D25640A004368616E3D25640AB4
:1004E000005465737420362025730A0054657374B4
:1004F00020352025730A0054657374203420257339
:100500000A005465737420332025730A0054657300
:100510007420322025730A0054657374203120251D
:10052000730A0025730A0025730A00646565700A62
:1005300000666F7263655F69646C650A006E6F6E5A
:10054000650A00707772733D005854414C5F5452F5
:10055000494D3D25640025730A00696E74725F730E
:1005600065635F70313D252D372E33660A00696E55
:1005700074725F70313D252D6C640A00696E74726F
:100580005F7365635F70303D252D372E33660A003B
:10059000696E74725F70303D252D6C640A00765F61
:1005A0006D63753D252D352E32660A0070707772A9
:1005B0003D25730A0064656275673D3078252D78A6
:1005C0000A0025730A006175746F0A006C6F675F1B
:1005D0006D6F64653D007573625F7077723D257362
:1005E0000A007265706F72745F6D61736B3D307875
:1005F000252D6C7820007265706F72745F696E745F
:10060000657276616C3D252D640A0072656C6179B6
:100610003D25730A0074746C3D252D640A0052490F
:100620004D455F616464723D252D642E252D640A5D
:10063000006E65696768626F725F7461626C655FA6
:1006400073697A653D25640A0074785F706F776519
:10065000723D25640A006368616E3D25640A006985
:1006600032633D0069643D007478743D25730A006F
:1006700053797374656D2053756D6D6172790A00DD
:1006800050413D09093078256C7800503D0909300A
:1006900078256C78004144343D09093078256C7820
:1006A000004144333D09093078256C7800414432DB
:1006B0003D09093078256C78004144313D09093005
:1006C00078256C780041333D090930782578004160
:1006D000323D0909307825780041313D09093078EB
:1006E000257800565F494E3D09093078257800523B
:1006F000483D09093078257800555054494D453D0D
:100700000909307825780050315F543D0909307867
:1007100025780050313D0909307825780050305F48
:10072000543D0909307825780050303D090930786A
:10073000257800565F4D43553D09093078257800EE
:10074000545F4D43553D0909307825780054313DBB
:1007500009093078257800543D090930782578005A
:100760004536343D0909307825780049443D09096A
:1007700030782578005458543D09093078257800A0
:100780005041200050200041443420004144332097
:1007900000414432200041443120004133200041D7
:1007A00032200041312000565F494E20005248203F
:1007B00000555054494D45200050315F54200050A1
:1007C00031200050305F54200050302000565F4DE3
:1007D00043552000545F4D435520005431200054B0
:1007E000200045363420004944200054585420004D
:1007F0002530327800765F6164343D252D382E3601
:1008000066002000765F6164333D252D382E366604
:10081000002000765F6164323D252D382E3666005B
:100820002000765F6164313D252D382E366600202C
:1008300000765F6C696768743D252D382E3666003A
:100840002000765F61323D252D372E336600200073
:10085000765F61313D252D372E3366002000765FAF
:10086000696E3D252D352E326600204E6576657207
:100870002D7573656420737461636B203E2025645D
:100880002062797465730A00757074696D653D2521
:100890002D642D646179732D253032643A25303210
:1008A000643A253032642D686F7572730A0074657E
:1008B0007374205B6F66667C317C327C337C347C65
:1008C000355D20202020202020202D207465737489
:1008D000206D6F6465730A0D00776474205B6F6E22
:1008E0007C6F66667C746573745D202020202020F8
:1008F00020202020202D207761746368646F670AB0
:100900000D007570677220202020202020202020DC
:1009100020202020202020202020202020202D20CA
:100920007265626F6F742076696120626F6F746C9C
:100930006F616465720A0D00626F6F742020202061
:1009400020202020202020202020202020202020A7
:10095000202020202D207265626F6F740A0D0070B8
:10096000777273205B646565707C666F7263655F28
:1009700069646C657C6E6F6E655D202D206D63759E
:1009800020736C656570206D6F64650A0D0072657B
:10099000737420656570726F6D20202020202020E8
:1009A000202020202020202020202D2072657374FC
:1009B0006F726520656570726F6D0A0D00707077DB
:1009C00072205B6F6E7C6F66665D20202020202089
:1009D0002020202020202020202D2070726F677280
:1009E000616D6D61626C65207077720A0D007478BC
:1009F00074205B737472696E675D20202020202054
:100A0000202020202020202020202D20536574200D
:100A10007265706F72742074657874207374726973
:100A20006E670A0D0074787077205B31352D305D6C
:100A300020202020202020202020202020202020B6
:100A4000202D205458205077722E20486967686501
:100A50007374203020283364426D290A0D007474A9
:100A60006C205B302D31355D20202020202020207F
:100A7000202020202020202020202D2074696D653A
:100A80002D746F2D6C69766520666F7220706163BE
:100A90006B6574730A0D00737320202020202020C2
:100AA0002020202020202020202020202020202046
:100AB0002020202D2073797374656D2073756D6D02
:100AC0006172790A0D0072732020202020202020DE
:100AD0002020202020202020202020202020202016
:100AE00020202D20726164696F2073746174730A11
:100AF0000D007269205B696E745D2020202020202B
:100B000020202020202020202020202020202D20D8
:100B10007265706F727420696E74657276616C0AAA
:100B20000D007265205B6D61736B5D2020202020BD
:100B300020202020202020202020202020202D20A8
:100B40006D6F7465207265706F7274207365747454
:100B5000696E670A0D006F7720202020202020205A
:100B60002020202020202020202020202020202085
:100B700020202D206F6E652D776972652073656E5C
:100B8000736F72730A0D006C6F67205B6175746F11
:100B90007C6F6E7C6F66665D2020202020202020E8
:100BA0002020202D206D6F74657320646174612096
:100BB0006F6E205553420A0D006E65205B666C75A2
:100BC00073685D202020202020202020202020204D
:100BD00020202020202D206E65696768626F7220BA
:100BE0007461626C650A0D006572722020202020FD
:100BF00020202020202020202020202020202020F5
:100C0000202020202D206572726F7220696E666F21
:100C10000A0D006D63752020202020202020202038
:100C20002020202020202020202020202020202DB7
:100C3000206D637520696E666F0A0D006964205B24
:100C400072657365745D20202020202020202020E4
:100C500020202020202020202D2069642068616E23
:100C6000646C696E670A0D0068756D202020202075
:100C70002020202020202020202020202020202074
:100C8000202020202D2068756D6964697479207397
:100C9000656E736F720A0D0072656C6179205B6F0F
:100CA0006E7C6F66667C73746174735D2020202097
:100CB000202020202D2072656C6179206E6574776C
:100CC0006F726B207265706F7274730A0D006465C9
:100CD000205B6D61736B5D20202020202020202070
:100CE000202020202020202020202D2064656275D7
:100CF000670A0D006368616E205B31312D32365D0D
:100D000020202020202020202020202020202020E3
:100D10002D204368616E2031312D32362028322E4D
:100D20003430352D32343830204D687A290A0D00A0
:100D300063616C69205B5B765F696E7C61317C61AD
:100D4000325D20766F6C747C72657365747C6E6F37
:100D50006E655D202D2063616C6962726174650A45
:100D60000D006164632020202020202020202020EE
:100D700020202020202020202020202020202D2066
:100D800073686F7720765F696E2C2061312C20614B
:100D90003220766F6C74616765730A0D00752020D0
:100DA0002020202020202020202020202020202043
:100DB0002020202020202020202D20757074696D97
:100DC000650A0D00762020202020202020202020D1
:100DD0002020202020202020202020202020202013
:100DE0002D2076657273696F6E0A0D0068202020D1
:100DF00020202020202020202020202020202020F3
:100E000020202020202020202D2068656C700A0DD5
:100E100000256300756E6B6E6F776E20636D640ADC
:100E2000004E484443303231365F004D4350333436
:100E300032585F004C334734323030445F00484D05
:100E400043353838335F004144584C3334355F0004
:100E5000424D503038355F00484948363133305FB5
:100E600000415432344D41435F002025730020255A
:100E7000362E32662000253032780074656D705F42
:100E800065787465726E3D252D362E3266002025FC
:100E900073002025362E3266204F6E2D426F617210
:100EA0006400253032780074656D705F626F617226
:100EB000643D252D362E3266000A00452025642E1D
:100EC000256420636C6F636B20256C7520637075DF
:100ED00020256C75206C706D20256C7520697271F1
:100EE00020256C7520676C656420256C7520796CF5
:100EF000656420256C7520726C656420256C7520F6
:100F0000747820256C75206C697374656E20256C6F
:100F1000752073656E736F727320256C7520736511
:100F20007269616C20256C750A00532025642E259A
:100F30006420636C6F636B20256C752074782025AA
:100F40006C7520727820256C752072747820256C61
:100F5000752072727820256C75207265786D6974C1
:100F600020256C752061636B747820256C75206E6C
:100F70006F61636B747820256C752061636B727888
:100F800020256C752074696D65646F757420256CFF
:100F9000752062616461636B727820256C752074C2
:100FA0006F6F6C6F6E6720256C7520746F6F736840
:100FB0006F727420256C752062616473796E63684A
:100FC00020256C752062616463726320256C752036
:100FD000636F6E74656E74696F6E64726F702025D6
:100FE0006C752073656E64696E6764726F7020251E
:100FF0006C75206C6C747820256C75206C6C727824
:1010000020256C750A00257325730A004F6E6C69E4
:101010006E650A000A002C20636865636B207261AC
:10102000746520257520487A0025732025732C20AF
:101030006368616E6E656C20257520706F776572D0
:10104000202575000A0025783A004D41432061644F
:101050006472657373200052616E646F6D20455534
:1010600049363420616464726573732067656E6508
:1010700072617465640A000A2A2A2A2A2A2A2A42E4
:101080006F6F74696E672025732A2A2A2A2A2A2AF2
:101090000A00020000FFFE00000141544D45474197
:1010A00031323872666131006C6F63616C686F73E6
:1010B0007400454550524F4D20697320636F727222
:1010C0007570742C20726577726974696E67207709
:1010D0006974682064656661756C74732E0A006EAD
:1010E000616E00696E660000407A10F35A00A072CB
:1010F0004E18090010A5D4E80000E8764817000053
:10110000E40B54020000CA9A3B000000E1F5050020
:101110000080969800000040420F000000A0860169
:10112000000000102700000000E803000000006439
:1011300000000000000A00000000000100000000A4
:10114000002C76D888DC674F0823DFC1DFAE59E179
:10115000B1B796E5E3E453C63AE651997696E8E6E8
:10116000C28426EB898C9B62ED407C6FFCEFBC9CBB
:101170009F40F2BAA56FA5F490055A2AF75C936BCD
:101180006CF9676DC11BFCE0E40D47FEF520E6B588
:1011900000D0ED902E0300943577050080841E0862
:1011A0000000204E0A000000C80C333333330F9880
:1011B0006E12831141EF8D2114893BE65516CFFE47
:1011C000E6DB18D1844B381BF77C1D901DA4BBE4D3
:1011D00024203284725E228100C9F124ECA1E53D15
:1011E00027494E46494E4954594E414ECDCCCC3DEF
:1011F0000AD7233C17B7D13877CC2B329595E62404
:101200001FB14F0A000020410000C84200401C46A8
:1012100020BCBE4CCA1B0E5AAEC59D7411241FBE05
:10122000CFEFD1E4DEBFCDBF17E0A0E0B2E0E4E64F
:10123000F2E101E00BBF02C007900D92A233B107AB
:10124000D9F71EE2A2E3B7E001C01D92AE38B107A4
:10125000E1F70E9475550C9430890C94000029E048
:10126000FC0120935700C895802D089500D083E499
:1012700095E0EDB7FEB7928381830E94218680912D
:101280001A0590911B050F900F9093FF04C000D09A
:101290008DE395E009C092FF04C000D081E395E0A2
:1012A00003C000D08BE295E0EDB7FEB79283818357
:1012B0000E9421860F900F900895E091B318F0E0FE
:1012C000EF71F070E85FF64E80838091B3188F5F06
:1012D0008093B3188091C82588608093C82542E424
:1012E00055E0CA0161E10E94BD4680E090E00895AA
:1012F000EF92FF92CF93DF93E82EE7017E01F92E64
:10130000E701809132079091330786FF2DC08DB79A
:101310009EB70C970FB6F8949EBF0FBE8DBFEDB76A
:10132000FEB7319680E092E0ADB7BEB712969C93BF
:101330008E9311978A81828313828B818483158295
:101340008C81868317828D81808711868E8182872A
:1013500013860E940F862DB73EB7245F3F4F0FB60E
:10136000F8943EBF0FBE2DBF87E597E0BE010E94F7
:1013700002488BEA95E0BE010E946E47DF91CF9153
:10138000FF90EF9008954F925F926F927F928F92AD
:101390009F92AF92BF92CF92DF92EF92FF920F9304
:1013A0001F93DF93CF93CDB7DEB760970FB6F89456
:1013B000DEBF0FBECDBF3B010E949A5BE82FF0E07D
:1013C000EE0FFF1FE358F74E8081918101969183C4
:1013D0008083809132079091330781FD74988091CA
:1013E0001A0590911B054424439496FF44240E94BF
:1013F000854D7C01DC018C91982F92959F709130E6
:1014000061F490E08F709070009739F08DEC95E268
:10141000B3010E948A44009751F080918F189091F7
:10142000901801969093901880938F18CEC187E5FD
:1014300097E00E94B4474FC0C8010296B3010E94D2
:101440008A44009709F444C0C8010F9660E074E62E
:1014500048E759E098010E94794AF7019181D80143
:1014600014968C911497981731F51A968C911A97B7
:101470008F5F1A968C9380918D1890918E1801969B
:1014800090938E1880938D1884E00E94B94EF801D5
:10149000208530E02817390728F584E00E94B94EEE
:1014A000D80118968C931897F70180818F70199640
:1014B0008C9319978AC1D8011A961C9284E00E94D5
:1014C000B94EF8018087D7018C918F7081873BC01E
:1014D000C8010E947A48082F192F0115110509F03B
:1014E000ABCF7BC144242FC0C8010296B3010E9438
:1014F0008144F70181818150D80114968C9380E05A
:1015000091E0A0E0B0E0F80183879487A587B687D3
:10151000128684E00E94B94ED80118968C931897D1
:10152000F70180818F7019968C9387E597E0B80159
:101530000E943B48C8010F9660E074E648E759E016
:1015400098010E94794AD70111968C911197F80160
:1015500084838C918F70878384E00E94B94ED80178
:1015600015968C9383E00E94B94E582EF80186831D
:10157000D70111968C9011978481881A9924AA24F6
:10158000BB24B6E0880C991CAA1CBB1CBA95D1F7E9
:10159000638574858585968520EC30E040E050E0D9
:1015A0000E941C81672F782F892F9927860E971EFE
:1015B000A81EB91EF80183869486A586B6868091FA
:1015C00032079091330781FD08C080911A0580FD94
:1015D00004C081FFFAC01D9BF8C08DB79EB7449729
:1015E0000FB6F8949EBF0FBE8DBFCDB6DEB6089481
:1015F000C11CD11C8FE292E0ADB7BEB712969C938E
:101600008E931197C7010296F60193838283D301CB
:101610008C918483158211968C9186831782F701B1
:101620008181D60118968C93189719961C92199758
:10163000808190E08F7090701B969C938E931A9788
:10164000F80185811C968C931C971D961C921D9702
:101650001E965C921E971F961C92BB27AB2D9A2D4F
:10166000892DF601918B808BC501B40124E630E011
:1016700040E050E00E941C81672F782F892F992726
:101680000E946281D60153967C936E9352970E947A
:101690000F862091FD04EDB7FEB774960FB6F8944F
:1016A000FEBF0FBEEDBF2223A9F000D000D0EDB7E2
:1016B000FEB7319687EE91E0ADB7BEB712969C9318
:1016C0008E931197228313820E9421860F900F9090
:1016D0000F900F9080911A0590911B0596FF2FC0D7
:1016E000442069F1F7012081822F90E08F70907083
:1016F00082309105DCF0822F8F708150207F822B09
:10170000808383E497E00E94214580918B1890911B
:101710008C18019690938C1880938B1880913207C7
:101720009091330796FF0BC0739809C08091911870
:1017300090919218019690939218809391188091AD
:10174000511D86FF42C00E946B53C70105960E943F
:101750002A538DB79EB70C970FB6F8949EBF0FBE55
:101760008DBFEDB7FEB731966E010894C11CD11C38
:10177000ADB7BEB71296DC92CE92119780E190E0A1
:101780009383828383E792E095838483D8011596BF
:101790008C9115978683178216968C918087118677
:1017A000D70111968C91828713860E947886EDB7B7
:1017B000FEB73C960FB6F894FEBF0FBEEDBF82E0B9
:1017C0000E944753C6010E942A538091320790918C
:1017D000330781FF0DC0749A0BC08BEA95E00E941D
:1017E0004847082F192F0115110509F07DCEEDCFBF
:1017F00060960FB6F894DEBF0FBECDBFCF91DF91DC
:101800001F910F91FF90EF90DF90CF90BF90AF901E
:101810009F908F907F906F905F904F90089587EE8C
:1018200093E08115910511F00197F1F70895882350
:10183000B9F052985A981DBA8091690080628093DD
:101840006900EA9A53985B98EB9A809169008068E6
:10185000809369008091680081608093680008959A
:10186000109269005A9AEA985B9AEB9808951F9231
:101870000F920FB60F9211248F939F93AF93BF9344
:101880008091680080FF20C08091A8259091A925B3
:10189000A091AA25B091AB250196A11DB11D809301
:1018A000A8259093A925A093AA25B093AB25809154
:1018B00032079091330787FF07C0749882E090E069
:1018C0009093F0048093EF04BF91AF919F918F911B
:1018D0000F900FBE0F901F9018951F920F920FB68A
:1018E0000F9211248F939F93AF93BF9380916800C1
:1018F00080FF20C08091AC259091AD25A091AE25B0
:10190000B091AF250196A11DB11D8093AC25909398
:10191000AD25A093AE25B093AF258091320790916D
:10192000330790FF07C0739882E090E09093F00433
:101930008093EF04BF91AF919F918F910F900FBE55
:101940000F901F90189580937C0080917B00877F7B
:1019500080937B0080917C00806C80937C0085E08C
:1019600080937A0080917A00806880937A008091D9
:101970007B0087FFFCCF80917B0085FFFCCF8091AF
:101980007A00806480937A0080917A0086FDFCCF93
:10199000109279001092780084E090E060E070E0AE
:1019A00020917A00206420937A0020917A0026FD0D
:1019B000FCCF2091780030917900620F731F01975E
:1019C00079F710927C0080917A008F7780937A006B
:1019D000769567957695679580E090E00E949F7E6A
:1019E000089580E00E94A30C2091F1043091F2044C
:1019F0004091F3045091F4040E947D7F21EE3AE778
:101A000044E95EE30E946D7D089580E18093510179
:101A1000809351019091510195FF03C08F5F8F31E9
:101A2000B9F76BE4869FB0011124882777FD809574
:101A3000982F0E94A17E20E030E64FE954E40E94F6
:101A40006D7D20E030E04AE754E40E94377E08953F
:101A50008091140585FF4BC080917B008860809346
:101A60007B0089EC80937C0085E080937A008091F4
:101A70007A00806880937A0080917B0087FFFCCF9A
:101A800080917B0085FFFCCF80917A0080648093F9
:101A90007A0080917A0086FDFCCF80917A00806484
:101AA00080937A0080917A0086FDFCCF6091780067
:101AB0007091790080E090E00E949F7E27ED33EAEC
:101AC00040E95FE30E947D7F26E636E648E853E47E
:101AD0000E946C7D609380187093811880938218A7
:101AE0009093831880917A008F7780937A0008957D
:101AF0006F927F928F929F92AF92BF92CF92DF921E
:101B0000EF92FF920F931F93DF93CF93CDB7DEB782
:101B10002A970FB6F894DEBF0FBECDBF3C011092DE
:101B20003A078FEF898344ECC42E48E1D42E00E0BD
:101B300010E032E0E32EF12CEC0EFD1E4E01089475
:101B4000811C911C2AE0A22EB12CAC0EBD1E3FC000
:101B50000830110509F441C0C401B7012A870E9469
:101B6000775089812A858F3F11F08E3F19F4809339
:101B70003A0734C06114710479F4C7010E9491508E
:101B80008093C525F701ADEBB5E281918D93EA1500
:101B9000FB05D9F721E022C0C7010E949150F60150
:101BA0008083D701F80193E0EE0FFF1F9A95E1F7CC
:101BB000E00FF11FE454F74E8D918193AA15BB05F8
:101BC000D9F70F5F1F4F89E090E0C80ED91E202F74
:101BD0008981882309F0BCCF01C028E0822F2A9692
:101BE0000FB6F894DEBF0FBECDBFCF91DF911F912E
:101BF0000F91FF90EF90DF90CF90BF90AF909F90AC
:101C00008F907F906F90089500D089EB9EE0EDB7A4
:101C1000FEB7928381830E9421860F900F900895D2
:101C20002F923F924F925F926F927F928F929F92EC
:101C3000AF92BF92CF92DF92EF92FF920F931F93DA
:101C4000DF93CF9300D000D0CDB7DEB78C014B012E
:101C5000009741F489E290E06BE270E04AE250E0E4
:101C600027E00AC08130910549F489E290E06BE2F7
:101C700070E04AE250E026E00E94534FC8010E9403
:101C8000780DF801E85CF84F80830115110581F0AB
:101C9000B4ECCB2EB8E1DB2E00E010E03F01A6E76C
:101CA0004A2EAEE05A2EFEE62F2EFEE03F2E44C115
:101CB0008DEB95E20E94C3519C01B901882777FD05
:101CC0008095982F0E94A17EC82EE92E8114910440
:101CD000A1F000D000D000D00DB71EB70F5F1F4F8E
:101CE00087EA9EE0ADB7BEB712969C938E9311978C
:101CF000562F472F3C2D2E2D97C0EDEBAE2EE5E253
:101D0000BE2E02EA1EE0D5018D915D0100D000D00B
:101D1000EDB7FEB73196ADB7BEB712961C930E93D2
:101D20001197828313826B837C830E9421860F909C
:101D30000F900F900F906B817C81B5ECAB16B5E2E4
:101D4000BB0609F700D000D000D00DB71EB70F5F5B
:101D50001F4F82E99EE0EDB7FEB7928381838C2D01
:101D60009E2D20E030E048EC52E40E94377ED801FE
:101D700012966D937D938D939C9315970E94218667
:101D8000EDB7FEB736960FB6F894FEBF0FBEEDBFA7
:101D90008091C525882319F086E892E002C08FE87B
:101DA00092E000D000D02EE83EE0ADB7BEB712966C
:101DB0003C932E93119714969C938E9313970E94A5
:101DC00021860F900F900F900F9048C0780153E03C
:101DD000EE0CFF1C5A95E1F7E00EF11EECEBF8E17A
:101DE000EE0EFF1EC7010E94C3519C01B901882756
:101DF00077FD8095982F0E94A17E5C01811491044B
:101E000081F100D000D000D00DB71EB70F5F1F4F7B
:101E10008BE79EE0ADB7BEB712969C938E93119759
:101E2000562F472F3A2D2B2D652F742F832F922F4E
:101E300020E030E048EC52E40E94377EF8016283F3
:101E40007383848395830E9421862DB73EB72A5FD2
:101E50003F4F0FB6F8943EBF0FBE2DBF0E94040E39
:101E600072C020E030E0D7018D917D0100D000D01C
:101E7000EDB7FEB73196ADB7BEB712965C924E92F3
:101E800011978283138229833A836B837C830E9418
:101E9000218629813A812F5F3F4F0F900F900F903D
:101EA0000F906B817C8128303105E9F600D000D09D
:101EB00000D0EDB6FEB60894E11CF11CEDB7FEB7FC
:101EC000328221828A2D9B2D20E030E048EC52E4C2
:101ED0000E94377ED70112966D937D938D939C93CC
:101EE00015970E942186EDB7FEB736960FB6F89487
:101EF000FEBF0FBEEDBFD6018C91882319F086E896
:101F000092E002C08FE892E000D000D02AE63EE0E6
:101F1000EDB7FEB732832183948383830E942186A9
:101F20000F900F900F900F900E94040E0F5F1F4FA5
:101F300089E090E0C80ED91ED3018C9190E008177B
:101F400019070CF443CF0F900F900F900F90CF9183
:101F5000DF911F910F91FF90EF90DF90CF90BF9096
:101F6000AF909F908F907F906F905F904F903F9039
:101F70002F900895DF93CF9300D0CDB7DEB7809137
:101F8000BE2589838091C4258A83CE0101960E9453
:101F90009C440F900F90CF91DF910895CF93DF93E2
:101FA000EC018091BD258F3FB1F58091BE258F3F1B
:101FB00091F58091BF258F3F71F58091C0258F3FAE
:101FC00051F58091C1258F3F31F58091C2258F3F1A
:101FD00011F58091C3258F3FF1F48091C4258F3F87
:101FE000D1F489E290E06BE270E04AE250E027E051
:101FF0000E94534F80E090E00E94780DC85CD84F5B
:1020000088838DEB95E269E170E049E050E00E9441
:102010006A870E94BA0FDF91CF9108951F920F92A5
:102020000FB60F920BB60F9211241F932F933F936D
:102030004F935F936F937F938F939F93AF93BF93D0
:10204000EF93FF938091C82582608093C82580918B
:102050001A0586FD2B9A80911A0587FD2B9A80918F
:10206000EF049091F0041816190614F4749A739AF8
:10207000809132079091330785FF02C0749873985E
:102080008091B3059091B40501979093B405809326
:10209000B305009709F07EC08091660790916707AD
:1020A00001969093670780936607209153213091A2
:1020B000542140915521509156212F5F3F4F4F4F52
:1020C0005F4F2093532130935421409355215093D7
:1020D000562120E130E03093B4052093B3052091E0
:1020E0001A0520FD02C01D9B05C0109236071092F4
:1020F000350706C021E030E03093360720933507DE
:1021000060911805709119056115710599F0019696
:102110000E943B81009771F47798809132079091EB
:10212000330792FF07C0749884E090E09093F00426
:102130008093EF0460911805709119056115710580
:1021400079F080916607909167070E943B81009724
:1021500039F48EE595E062E140E050E00E94BD4632
:1021600080911A0586FD2B9880911A0590911B0588
:1021700091FF10C00E949A5B8A3119F0182F1F5FDF
:1021800001C01BE00E94DE59812F90E00E94B25BEB
:102190000E947C5A8DEC95E060E040E050E00E94A7
:1021A000BD46FF91EF91BF91AF919F918F917F912C
:1021B0006F915F914F913F912F911F910F900BBEA7
:1021C0000F900FBE0F901F9018958091B3189091AB
:1021D0006721891B08950E94E510882379F0E0911A
:1021E0006721F0E0EF71F070E85FF64E208130E09B
:1021F000809167218F5F8093672102C02FEF3FEFAF
:10220000C9010895CF93DF93EC0110925A07109201
:10221000590788819981009731F023E08431920732
:1022200009F0B9C009C00E94E510882341F484E197
:1022300093E099838883B3C0613109F0B0C0F8940A
:1022400078940E94EB1090E090935E0780935D0776
:102250008D3009F47CC08F3F31F38231910569F1F3
:102260008F37910521F08830910509F053C0809196
:10227000610790916207181619060CF060C0609112
:10228000882E7091892E88E090E00E94E38560910D
:10229000882E7091892E80E290E00E94E385609103
:1022A000882E7091892E88E090E00E94E3858091CD
:1022B00061079091620701973EC06091882E7091EE
:1022C000892E8DE090E00E94E385109260071092C5
:1022D0005F0714C088599E4DFC0180816091882E53
:1022E0007091892E90E00E94E38580915F07909124
:1022F000600701969093600780935F0780915F0766
:1023000090916007209161073091620782179307CF
:102310000CF315C06091882E7091892E0E94E38580
:10232000809161079091620720915D07FC01E85957
:10233000FE4D208301969093620780936107809100
:102340006107909162078F33910509F06CCF10926D
:102350006721809167218093B318809161079091E4
:102360006207FC01E859FE4D108290935A07809352
:10237000590710926207109261078091C6259091CB
:10238000C725009709F44FCF60915B0740E050E00C
:102390000E94BD4648CF1982188283E001C081E0C7
:1023A000DF91CF9108957894809135079091360709
:1023B0000097C9F080911A0590911B0593FD13C0F9
:1023C00092FF03C083B7817F03C083B7817F86609C
:1023D00083BFF89483B7816083BF7894889583B76F
:1023E0008E7F83BF78940895CF93DF93EC0188812B
:1023F0009981009721F02BE0863F920799F40E9483
:10240000CC580E94D31180916C0F90916D0F65E8AC
:1024100040E050E00E94BD4686EF9BE099838883B0
:1024200081E003C01982188283E0DF91CF91089583
:10243000CF93DF930E94CC5880EB0E9443528823B5
:10244000B1F40E94A9528091511D9091521D81605A
:102450009093521D8093511D00D081E69EE0EDB710
:10246000FEB7928381830E9421860F900F908EB1D8
:10247000C82FD0E0C470D070729A0E94CC588EE4FD
:102480000E9443528823B1F40E94A9528091511DA9
:102490009091521D82609093521D8093511D00D0E7
:1024A00088E59EE0EDB7FEB7928381830E94218686
:1024B0000F900F90209709F472980E94CC588EEEDE
:1024C0000E9443528823B1F40E94A9528091511D69
:1024D0009091521D84609093521D8093511D00D0A5
:1024E00080E59EE0EDB7FEB7928381830E9421864E
:1024F0000F900F9086EA0E9443528823B1F40E9405
:10250000A9528091511D9091521D88609093521D47
:102510008093511D00D087E49EE0EDB7FEB7928313
:1025200081830E9421860F900F900E94CC588CE3EB
:102530000E9443528823B1F40E94A9528091511DF8
:102540009091521D80619093521D8093511D00D037
:102550008EE39EE0EDB7FEB7928381830E942186D1
:102560000F900F900E94CC5882ED0E944352882316
:10257000B1F40E94A9528091511D9091521D806228
:102580009093521D8093511D00D084E39EE0EDB7DF
:10259000FEB7928381830E9421860F900F900E9444
:1025A000CC5880ED0E9443528823B1F40E94A95276
:1025B0008091511D9091521D80689093521D80937F
:1025C000511D00D08BE29EE0EDB7FEB79283818370
:1025D0000E9421860F900F90C7E0D0E00E94CC5857
:1025E0008CE70E9443528823B9F40E94A95280913B
:1025F000511D9091521D80649093521D8093511DE6
:1026000000D081E29EE0EDB7FEB7928381830E9405
:1026100021860F900F9002C0219701F70E94A952C6
:102620000E94040EDF91CF910895DF93CF9300D0E5
:10263000CDB7DEB74A8369830E947F526981862FB6
:102640000E94B1524A81842F0E94B1520E94A95225
:102650000F900F90CF91DF910895AF92BF92DF92CC
:10266000EF92FF920F931F93DF93CF9300D00F92BF
:10267000CDB7DEB7082FD22E4A835B8369830E94D1
:102680007F526981862F0E94B152802F81600E9403
:10269000A6524A815B81042F152FAA24BB24ED2C5E
:1026A000FF240894E108F1080FC0AE14BF0419F428
:1026B0000E94CC5202C00E94C252F801808308944A
:1026C000A11CB11C0F5F1F4FAD1478F30E94A952DB
:1026D0000F900F900F90CF91DF911F910F91FF906E
:1026E000EF90DF90BF90AF900895AF92BF92CF92DE
:1026F000DF92EF92FF920F931F93DF93CF93CDB7AB
:10270000DEB760970FB6F894DEBF0FBECDBFB82E10
:10271000A42E662309F455C0AE014F5F5F4F80E1E0
:10272000DA011D928A95E9F780EB68E928E00E94BA
:102730002D13BB2059F000D080E992E0EDB7FEB731
:10274000928381830E940F860F900F908E010F5FFE
:102750001F4F38E0E32EF12CEC0EFD1E27E9C22EB0
:1027600022E0D22ED8018D918D0100D000D0EDB79E
:10277000FEB73196ADB7BEB71296DC92CE921197E6
:10278000828313820E940F860F900F900F900F90FC
:102790000E151F0539F700D000D0EDB7FEB7319602
:1027A0008CE992E0ADB7BEB712969C938E931197C9
:1027B0008885828313820E940F860F900F900F905E
:1027C0000F90AA2009F457C0AE014F5F5F4F80E120
:1027D000FA0111928A95E9F780EB60E828E00E94FF
:1027E0002D13BB2069F000D082EA92E0ADB7BEB7EE
:1027F00012969C938E9311970E940F860F900F90C4
:102800008E010F5F1F4F90E1E92EF12CEC0EFD1EA3
:1028100087E9C82E82E0D82EF80181918F0100D07F
:1028200000D0EDB7FEB73196ADB7BEB71296DC92C9
:10283000CE921197828313820E940F860F900F9081
:102840000F900F900E151F0539F700D000D0EDB78F
:10285000FEB731968CE992E0ADB7BEB712969C9365
:102860008E9311978885828313820E940F860F9022
:102870000F900F900F9060960FB6F894DEBF0FBECA
:10288000CDBFCF91DF911F910F91FF90EF90DF901F
:10289000CF90BF90AF9008950F931F93DF93CF9386
:1028A00000D0CDB7DEB71A8219828EEE6AEA8E01A9
:1028B0000F5F1F4FA80122E00E942D13398120E0F5
:1028C0008A8190E0822B932B909329198093281969
:1028D0008EEE6CEAA80122E00E942D13398120E0DF
:1028E0008A8190E0822B932B90932B1980932A1945
:1028F0008EEE6EEAA80122E00E942D13398120E0BD
:102900008A8190E0822B932B90932D1980932C1920
:102910008EEE60EBA80122E00E942D13398120E0A9
:102920008A8190E0822B932B90933B1980933A19E4
:102930008EEE62EBA80122E00E942D13398120E087
:102940008A8190E0822B932B90933D1980933C19C0
:102950008EEE64EBA80122E00E942D13398120E065
:102960008A8190E0822B932B90933F1980933E199C
:102970008EEE66EBA80122E00E942D13398120E043
:102980008A8190E0822B932B90932F1980932E199C
:102990008EEE68EBA80122E00E942D13398120E021
:1029A0008A8190E0822B932B909331198093301978
:1029B0008EEE6AEBA80122E00E942D13398120E0FF
:1029C0008A8190E0822B932B909335198093341950
:1029D0008EEE6CEBA80122E00E942D13398120E0DD
:1029E0008A8190E0822B932B90933719809336192C
:1029F0008EEE6EEBA80122E00E942D13398120E0BB
:102A00008A8190E0822B932B909339198093381907
:102A10000F900F90CF91DF911F910F9108952F92FA
:102A20003F924F925F926F927F928F929F92AF925E
:102A3000BF92CF92DF92EF92FF920F931F93DF939B
:102A4000CF93CDB7DEB76C970FB6F894DEBF0FBE4D
:102A5000CDBFA82E4A8B2B8FFE01319683E0DF017C
:102A60001D928A95E9F780914C19882339F46C8F6F
:102A70000E944C1481E080934C196C8D662309F4FC
:102A800075C08EEE64EF4EE20E94151369E07AE1A4
:102A900080E090E00E9430528EEE66EFAE014F5F14
:102AA0005F4F22E00E942D13698170E080E090E08A
:102AB000982F872F762F66272A8130E040E050E05C
:102AC000622B732B842B952B20913E1930913F194B
:102AD00040E050E0621B730B840B950B20913C1976
:102AE00030913D1940E050E00E941C817B018C0137
:102AF0003FE015950795F794E7943A95D1F76091E3
:102B0000361970913719882777FD8095982F2BE01B
:102B1000660F771F881F991F2A95D1F720913819C2
:102B200030913919442737FD4095542F2E0D3F1D04
:102B3000401F511F0E9484812E0D3F1D3093331979
:102B400020933219285F3F4F14E0359527951A9549
:102B5000E1F779010027F7FC0095102FE09240196A
:102B6000F09241190093421910934319BA2DB2956E
:102B7000BB0FBB0FB07CBC5CB9872A2D30E03E8B0D
:102B80002D8B63E070E00A2C02C0660F771F0A9459
:102B9000E2F7882777FD8095982F25E335E040E020
:102BA00050E00E941C81DC01CB010296A11DB11DE9
:102BB0008A879B87AC87BD8720E533EC40E050E0F7
:102BC00004C05595479537952795AA94D2F72E8737
:102BD0003F87488B598B18861C821D821E821F825C
:102BE00048E050E08D899E89481B590B5C8B4B8BCC
:102BF00069C18EEE64EF49850E9415136A857B8555
:102C00008C859D850E9430528EEE66EFAE014F5F3F
:102C10005F4F23E00E942D13809132199091331958
:102C2000805A9F401C01442437FC4094542CC2011C
:102C3000B101A20191010E941C816F8B788F898F55
:102C40009A8F20912C1930912D19442737FD4095EA
:102C5000542FC201B1010E941C817B018C01BDE097
:102C600015950795F794E794BA95D1F722E030E0EF
:102C700040E050E0E20EF31E041F151F6F89788DAF
:102C8000898D9A8DACE09595879577956795AA95EE
:102C9000D1F720912E1930912F19442737FD4095F7
:102CA000542F0E941C81BC01992777FD9095892F94
:102CB000E60EF71E081F191FE2E015950795F79419
:102CC000E794EA95D1F780E090E8A0E0B0E0E80E64
:102CD000F91E0A1F1B1F20913A1930913B1940E041
:102CE00050E0C801B7010E941C813B014C017FE00C
:102CF00096948794779467947A95D1F7A980BB24AA
:102D0000CC24DD246501BB24AA248A8190E0A0E0C4
:102D1000B0E0BA2FA92F982F8827A82AB92ACA2A43
:102D2000DB2A8B8190E0A0E0B0E0A82AB92ACA2A69
:102D3000DB2A0B8804C0D594C794B794A7940A944F
:102D4000D2F720912A1930912B19442737FD40954D
:102D5000542FC201B1010E941C817B018C014BE008
:102D600015950795F794E7944A95D1F7809128191E
:102D700090912919AA2797FDA095BA2F32E0880FC4
:102D8000991FAA1FBB1F3A95D1F7E80EF91E0A1F1B
:102D90001B1F2091301930913119442737FD409580
:102DA000542F6F89788D898D9A8D0E941C8127E11F
:102DB00095958795779567952A95D1F7E60EF71E35
:102DC000081F191F0D8804C0EE0CFF1C001F111FE7
:102DD0000A94D2F722E030E040E050E0E20EF31E29
:102DE000041F151F82E015950795F794E7948A95BF
:102DF000D1F7AE18BF08C00AD10AC601B5012E85A9
:102E00003F85488959890E941C8197FD0BC0660F38
:102E1000771F881F991FA40193010E946281790185
:102E20008A010AC0A40193010E94628179018A018A
:102E3000EE0CFF1C001F111F552717FD5A95412F3F
:102E4000302F2F2DCA01B9010E941C812EED3BE0CD
:102E500040E050E00E941C815B016C01C801B70199
:102E600023E433EE4FEF5FEF0E941C81BC019927F2
:102E700077FD9095892F6153714F8F4F9F4F56016A
:102E8000DD24B7FCD094CD2C6A0D7B1D8C1D9D1DBF
:102E900044E095958795779567954A95D1F76E0D9E
:102EA0007F1D801F911F2C813D814E815F81260FE8
:102EB000371F481F591F2C833D834E835F833885FE
:102EC0003F5F388748855A89451708F492CE5523C5
:102ED00091F0252F30E040E050E06C817D818E81C3
:102EE0009F810E9462812093441930934519409339
:102EF0004619509347198B8D8823C9F16091441965
:102F00007091451980914619909147196115710585
:102F10008105910561F10E94A17E20E836EE45EC25
:102F200057E40E94377E21E03EED42E45EE30E94DA
:102F3000E07F562F472F382F292F60E070E080E880
:102F40009FE3DA01F9012B2F3A2F4F2F5E2F0E94BA
:102F50006C7D2BE43AE34DEB57E30E94377E6093A0
:102F600048197093491980934A1990934B196C969C
:102F70000FB6F894DEBF0FBECDBFCF91DF911F918A
:102F80000F91FF90EF90DF90CF90BF90AF909F9008
:102F90008F907F906F905F904F903F902F9008950B
:102FA000DF93CF9300D000D000D0CDB7DEB7FE01C5
:102FB000319686E0DF011D928A95E9F780918A18A3
:102FC000882399F486EA61E340E00E94151386EABB
:102FD0006CE24AE00E94151381E080938A186CE746
:102FE0007EE380E090E00E94305286EA6DE248E0A5
:102FF0000E9415136CE77EE380E090E00E9430525F
:1030000086EA62E3AE014F5F5F4F26E00E942D1318
:1030100086EA6DE247E00E9415139A8180E04981BB
:1030200050E0482B592B50938518409384189C816D
:1030300080E02B8130E0282B392B309387182093A8
:1030400086187E8160E08D8190E0862B972B90938F
:103050008918809388186DB77EB7685070400FB696
:10306000F8947EBF0FBE6DBFEDB7FEB7319666EA2E
:1030700072E0ADB7BEB712967C936E9311975383EF
:10308000428335832483978386830E940F866DB79E
:103090007EB7685F7F4F0FB6F8947EBF0FBE6DBFDF
:1030A00026960FB6F894DEBF0FBECDBFCF91DF914D
:1030B0000895CF92DF92EF92FF920F931F93DF93C9
:1030C000CF9300D000D000D0CDB7DEB78E010F5F18
:1030D0001F4F86E0F80111928A95E9F78CE362E0D0
:1030E00041E00E9415138CE360E048E50E9415134F
:1030F00062E174E380E090E00E9430528CE363E090
:10310000A80126E00E942D138CE362E043E00E94B8
:103110001513998180E00A8110E0082B192B109378
:103120006118009360189B8180E06C8170E0682BCF
:10313000792B70936318609362183D8120E08E8133
:1031400090E0822B932B90936518809364188827C6
:1031500077FD8095982F0E94A17E6B017C01B801BC
:10316000882777FD8095982F0E94A17E9B01AC0156
:10317000C701B6010E94E07D2DB73EB72C5030400C
:103180000FB6F8943EBF0FBE2DBF0DB71EB70F5F31
:103190001F4F24EB32E0EDB7FEB73283218320913D
:1031A000601830916118F8013383228320916218EE
:1031B0003091631835832483209164183091651809
:1031C0003783268320EE3EE245E652E40E947D7F6F
:1031D00020E030E044E353E40E946D7DF801608715
:1031E0007187828793870E940F862DB73EB7245F31
:1031F0003F4F0FB6F8943EBF0FBE2DBF26960FB6B9
:10320000F894DEBF0FBECDBFCF91DF911F910F911C
:10321000FF90EF90DF90CF900895CF93DF93EC0174
:1032200088819981009731F02BE08F3D920709F05A
:1032300071C00BC08BE397E060E870E00E947349B7
:103240008FED9BE09983888369C08BE397E00E94B0
:103250009E49009709F462C080913207909133072C
:1032600093FF3FC08091511D82FF3BC083E061E02E
:1032700048E021E00E940F158DB79EB70A970FB660
:10328000F8949EBF0FBE8DBFEDB7FEB731968FECA1
:1032900091E0ADB7BEB712969C938E931197809133
:1032A000441990914519A0914619B091471982830C
:1032B0009383A483B5838091481990914919A09173
:1032C0004A19B0914B1986839783A087B1870E94D2
:1032D00021868DB79EB70A960FB6F8949EBF0FBE93
:1032E0008DBF809132079091330794FF06C0809183
:1032F000511D83FF02C00E94D01780913207909128
:10330000330795FF97CF8091511D84FF93CF0E9483
:10331000591890CF1982188283E001C081E0DF91B3
:10332000CF910895CF92DF92FF920F931F93CF9387
:10333000DF93729A80911A0583FD06C0C0E5D0E044
:103340000E940F0C2197E1F78EE40E9443528823DC
:10335000B1F08091572190915821A0915921B091BD
:103360005A210196A11DB11D809357219093582198
:10337000A0935921B0935A2121E030E084C0C0E5E8
:10338000D0E00E940F0C2197E1F78FE40E94435296
:103390000E94C252F82E8295869586958370813060
:1033A000A9F420915B2130915C2140915D215091E5
:1033B0005E212F5F3F4F4F4F5F4F20935B21309334
:1033C0005C2140935D2150935E2116C08230A0F0B5
:1033D00020915F21309160214091612150916221C3
:1033E0002F5F3F4F4F4F5F4F20935F2130936021FE
:1033F00040936121509362210E94C2521F2D1F737E
:1034000000E0080F111D0E94C2520E94CC5220E021
:10341000E901C80FD11DD695C795D695C7950E94CD
:10342000A95280911A0583FF7298B80180E090E05C
:103430000E949F7E20E134E048EC5BE30E947D7FA8
:1034400060934D1970934E1980934F1990935019B2
:10345000BE0180E090E00E949F7E24EA3CEF44E2BF
:103460005CE30E947D7F20E030E040E252E40E9475
:103470006C7D6093C9257093CA258093CB2590936A
:10348000CC2520E030E0C901DF91CF911F910F9151
:10349000FF90DF90CF9008957298729A8EE40E9408
:1034A000435280EA0E94B15280E00E94B15280E013
:1034B0000E94B1528FE40E9443520E94C2528295F0
:1034C0008695869583708130A9F420915B21309197
:1034D0005C2140915D2150915E212F5F3F4F4F4F06
:1034E0005F4F20935B2130935C2140935D2150938B
:1034F0005E2116C08230A0F020915F2130916021C2
:1035000040916121509162212F5F3F4F4F4F5F4F9C
:1035100020935F2130936021409361215093622179
:1035200000D000D0EDB7FEB7319629EC32E0ADB750
:10353000BEB712963C932E931197828313820E94FA
:103540000F860F900F900F900F908EE40E944352C1
:1035500080E80E94B15280E00E94B15280E00E9457
:10356000B1520E94A95280E090E0089500D084E119
:103570009EE0ADB7BEB712969C938E9311970E94B2
:1035800021862091FD040F900F902223A9F000D0F6
:1035900000D0EDB7FEB7319681E19EE0ADB7BEB782
:1035A00012969C938E931197228313820E942186F8
:1035B0000F900F900F900F90089500D08CEE9DE02B
:1035C000EDB7FEB7928381830E94218684EC9DE053
:1035D000EDB7FEB7928381830E9421868DE99DE03D
:1035E000EDB7FEB7928381830E94218682E69DE03B
:1035F000EDB7FEB7928381830E94218680E39DE030
:10360000EDB7FEB7928381830E94218684EF9CE010
:10361000EDB7FEB7928381830E9421868EEC9CE0F9
:10362000EDB7FEB7928381830E94218688E99CE0F2
:10363000EDB7FEB7928381830E94218688E69CE0E5
:10364000EDB7FEB7928381830E9421868CE39CE0D4
:10365000EDB7FEB7928381830E94218683E19CE0CF
:10366000EDB7FEB7928381830E94218688EE9BE0AE
:10367000EDB7FEB7928381830E94218689EB9BE0A0
:10368000EDB7FEB7928381830E94218687E89BE095
:10369000EDB7FEB7928381830E94218686E59BE089
:1036A000EDB7FEB7928381830E94218682E29BE080
:1036B000EDB7FEB7928381830E94218682EF9AE064
:1036C000EDB7FEB7928381830E94218686EC9AE053
:1036D000EDB7FEB7928381830E94218687E99AE045
:1036E000EDB7FEB7928381830E9421868EE59AE032
:1036F000EDB7FEB7928381830E94218685E29AE02E
:10370000EDB7FEB7928381830E9421868EEE99E009
:10371000EDB7FEB7928381830E9421868DEB99E0FD
:10372000EDB7FEB7928381830E9421868EE899E0EF
:10373000EDB7FEB7928381830E9421868FE599E0E1
:10374000EDB7FEB7928381830E94218688E399E0DA
:10375000EDB7FEB7928381830E94218682E099E0D3
:10376000EDB7FEB7928381830E94218689ED98E0B0
:10377000EDB7FEB7928381830E9421868EEA98E09E
:10378000EDB7FEB7928381830E9421860F900F9040
:10379000089589ED92E00E94418608952F923F920C
:1037A0004F925F926F927F928F929F92AF92BF9251
:1037B000CF92DF92EF92FF920F931F93CF93DF93FD
:1037C00060915321709154218091552190915621FF
:1037D000A0905321B0905421C0905521D0905621F3
:1037E00060905321709054218090552190905621E3
:1037F00020905321309054214090552150905621D3
:103800002DB73EB72A5030400FB6F8943EBF0FBEDA
:103810002DBFCDB7DEB7219628E838E0EDB7FEB76B
:1038200032832183A0E8EA2EA1E5FA2EA1E00A2F37
:10383000112DA80197010E9462813B832A83C60152
:10384000B501A80197010E946281F0E1EF2EFEE030
:10385000FF2E012D112DA80197010E9462813327AF
:1038600027FD30953D832C83C401B301A801970146
:103870000E946281ECE3EE2EF12C012D112DA801A6
:1038800097010E946281332727FD30953F832E8365
:10389000C201B101A80197010E946281772767FDEB
:1038A0007095798768870E9421862DB73EB7265F7D
:1038B0003F4F0FB6F8943EBF0FBE2DBFDF91CF91A3
:1038C0001F910F91FF90EF90DF90CF90BF90AF903E
:1038D0009F908F907F906F905F904F903F902F9030
:1038E0000895EEE8FEE28081918122E4823492071D
:1038F000B9F000D000D08AE698E0ADB7BEB7129616
:103900009C938E931197EE58FE421496FC93EE937F
:1039100013970E9421860F900F900F900F9008959B
:103920003A96B1E4E53FFB07F0F208950F931F9339
:10393000CF93DF93EC018C9A0E94F10C00D000D061
:1039400000D02EE538E0EDB7FEB7328321836383E4
:103950007483858396830E9421868DB79EB70696D1
:103960000FB6F8949EBF0FBE8DBF209719F00E942E
:10397000040E0BC000D08CE598E0EDB7FEB7928343
:1039800081830E9421860F900F9081E00E94A30CFA
:1039900000D000D000D00DB71EB70F5F1F4F20E53D
:1039A00038E0EDB7FEB7328321832091F5043091E2
:1039B000F6044091F7045091F8040E947D7FF801CD
:1039C00062837383848395830E9421868DB79EB71B
:1039D00006960FB6F8949EBF0FBE8DBF209719F0C4
:1039E0000E94040E0BC000D08EE498E0EDB7FEB745
:1039F000928381830E9421860F900F9082E00E9423
:103A0000A30C00D000D000D00DB71EB70F5F1F4F22
:103A100022E438E0EDB7FEB7328321832091F90428
:103A20003091FA044091FB045091FC040E947D7F88
:103A3000F80162837383848395830E9421868DB706
:103A40009EB706960FB6F8949EBF0FBE8DBF209707
:103A500019F00E94040E0BC000D080E498E0EDB78E
:103A6000FEB7928381830E9421860F900F9083E09E
:103A70000E94A30C00D000D000D021E338E0EDB7C5
:103A8000FEB73283218363837483858396830E9488
:103A900021868C988DB79EB706960FB6F8949EBF78
:103AA0000FBE8DBF209719F00E94040E0BC000D0EE
:103AB0008FE298E0EDB7FEB7928381830E94218662
:103AC0000F900F908091511D87FFA4C080ED61E0A1
:103AD00042E121E00E94C65F00D000D000D022E287
:103AE00038E0EDB7FEB73283218363837483858327
:103AF00096830E9421868DB79EB706960FB6F894DE
:103B00009EBF0FBE8DBF209719F00E94040E0BC000
:103B100000D080E298E0EDB7FEB7928381830E94E7
:103B200021860F900F9080ED62E042E121E00E943B
:103B3000C65F00D000D000D023E138E0EDB7FEB77B
:103B40003283218363837483858396830E942186D5
:103B50008DB79EB706960FB6F8949EBF0FBE8DBF69
:103B6000209719F00E94040E0BC000D081E198E06C
:103B7000EDB7FEB7928381830E9421860F900F904C
:103B800080ED63E042E121E00E94C65F00D000D0FA
:103B900000D024E038E0EDB7FEB7328321836383A1
:103BA0007483858396830E9421868DB79EB706967F
:103BB0000FB6F8949EBF0FBE8DBF209719F00E94DC
:103BC000040E0BC000D082E098E0EDB7FEB7928300
:103BD00081830E9421860F900F9080ED64E042E186
:103BE00021E00E94C65F00D000D000D025EF37E072
:103BF000EDB7FEB732832183638374838583968315
:103C00000E9421868DB79EB706960FB6F8949EBF88
:103C10000FBE8DBF0E94040EDF91CF911F910F91B7
:103C200008950F931F93CF93DF93882389F08DEB33
:103C300095E26FEF70E049E050E00E948A858DEBDD
:103C400095E269E170E049E050E00E946A871CC09B
:103C5000CDEBD5E200EF17E0899100D000D0EDB7B1
:103C6000FEB73196ADB7BEB712961C930E9311975F
:103C7000828313820E9421860F900F900F900F90E5
:103C8000B5E2C53CDB0741F70E94040EDF91CF91FE
:103C90001F910F910895EF92FF920F931F936091E0
:103CA00002057091030580E090E00E947C8564EF3E
:103CB00072E00E949185009709F0B6C08CE498E20A
:103CC000A1E0B0E08093140590931505A09316052C
:103CD000B093170584E195E06EE070E044E050E0B9
:103CE0000E946A878CE390E09093190580931805F1
:103CF00088E195E062E170E042E050E00E946A876E
:103D00008AE090E490931B0580931A058AE195E080
:103D100064E170E042E050E00E946A87109233074D
:103D20001092320782E397E060E070E042E050E0FA
:103D30000E946A870F2EF2E2EF2EFFEFFF2EFCECBF
:103D40000F2FFBE31F2FF02DE092F504F092F60405
:103D50000093F7041093F80485EF94E066E070E0B8
:103D600044E050E00E946A87E092F904F092FA047D
:103D70000093FB041093FC0489EF94E06AE070E088
:103D800044E050E00E946A8787ED94E3AFEEBCE325
:103D90008093F1049093F204A093F304B093F4049D
:103DA00081EF94E062E070E044E050E00E946A87B6
:103DB0001092370780E090E00E94255D87E397E04E
:103DC00066E170E041E050E00E946A878AE18093FA
:103DD0001C058AE190E00E949D5B8CE195E067E123
:103DE00070E041E050E00E946A878FE080931D05FB
:103DF0008DE195E068E170E041E050E00E946A8763
:103E000086E798E12AE0FC0111922A95E9F762E23F
:103E100070E04AE050E00E946A8781E00E94111E33
:103E200080E090E00E94CE0F1F910F91FF90EF90E5
:103E30000895882309F4B4C18091140580FF0BC054
:103E400000D08BEE97E0EDB7FEB7928381830E949E
:103E500021860F900F908091140581FF0BC000D038
:103E600087EE97E0EDB7FEB7928381830E942186AB
:103E70000F900F908091140582FF0BC000D082EE4E
:103E800097E0EDB7FEB7928381830E9421860F9061
:103E90000F908091140583FF0BC000D08FED97E049
:103EA000EDB7FEB7928381830E9421860F900F9019
:103EB0008091140584FF0BC000D08BED97E0EDB727
:103EC000FEB7928381830E9421860F900F9080918C
:103ED000140585FF0BC000D084ED97E0EDB7FEB769
:103EE000928381830E9421860F900F908091140508
:103EF00086FF0BC000D08DEC97E0EDB7FEB7928344
:103F000081830E9421860F900F908091140587FF76
:103F10000BC000D089EC97E0EDB7FEB792838183A8
:103F20000E9421860F900F908091140590911505A5
:103F3000A0911605B091170590FF0BC000D083EC3F
:103F400097E0EDB7FEB7928381830E9421860F90A0
:103F50000F908091140590911505A0911605B091D0
:103F6000170591FF0BC000D08FEB97E0EDB7FEB7C0
:103F7000928381830E9421860F900F908091140577
:103F800090911505A0911605B091170592FF0BC0F1
:103F900000D089EB97E0EDB7FEB7928381830E9452
:103FA00021860F900F908091140590911505A09196
:103FB0001605B091170593FF0BC000D081EB97E079
:103FC000EDB7FEB7928381830E9421860F900F90F8
:103FD0008091140590911505A0911605B0911705D3
:103FE00094FF0BC000D08DEA97E0EDB7FEB7928347
:103FF00081830E9421860F900F90809114059091EB
:104000001505A0911605B091170595FF0BC000D0BE
:1040100087EA97E0EDB7FEB7928381830E942186FD
:104020000F900F908091140590911505A0911605A1
:10403000B091170596FF0BC000D083EA97E0EDB76B
:10404000FEB7928381830E9421860F900F9080910A
:10405000140590911505A0911605B091170597FFCD
:104060000BC000D08FE997E0EDB7FEB79283818354
:104070000E9421860F900F90809114059091150554
:10408000A0911605B0911705A0FF0BC000D08BE9D9
:1040900097E0EDB7FEB7928381830E9421860F904F
:1040A0000F908091140590911505A0911605B0917F
:1040B0001705A1FF0BC000D086E997E0EDB7FEB76A
:1040C000928381830E9421860F900F908091140526
:1040D00090911505A0911605B0911705A2FF0BC090
:1040E00000D081E997E0EDB7FEB7928381830E940B
:1040F00021860F900F908091140590911505A09145
:104100001605B0911705A3FF0BC000D08CE897E00F
:10411000EDB7FEB7928381830E9421860F900F90A6
:104120008091140590911505A0911605B091170581
:10413000A4FF0BC000D087E897E0EDB7FEB79283ED
:1041400081830E9421860F900F9080911405909199
:104150001505A0911605B0911705A5FF0BC000D05D
:1041600084E897E0EDB7FEB7928381830E942186B1
:104170000F900F908091140590911505A091160550
:10418000B0911705A6FFA5C200D080E897E0EDB773
:10419000FEB7928381830E9421860F900F9099C26F
:1041A00000D000D000D085E797E0EDB7FEB792834E
:1041B000818381E090E0A0E0B0E083839483A583D5
:1041C000B6830E9421868DB79EB706960FB6F894E7
:1041D0009EBF0FBE8DBF0E94040E00D000D000D045
:1041E0008BE697E0EDB7FEB79283818382E090E0A3
:1041F000A0E0B0E083839483A583B6830E942186E8
:104200008DB79EB706960FB6F8949EBF0FBE8DBFB2
:104210000E94040E00D000D000D080E697E0EDB7F9
:10422000FEB79283818384E090E0A0E0B0E08383D6
:104230009483A583B6830E9421868DB79EB7069688
:104240000FB6F8949EBF0FBE8DBF0E94040E00D023
:1042500000D000D087E597E0EDB7FEB79283818369
:1042600088E090E0A0E0B0E083839483A583B683E8
:104270000E9421868DB79EB706960FB6F8949EBF12
:104280000FBE8DBF0E94040E00D000D000D08DE480
:1042900097E0EDB7FEB79283818380E190E0A0E0E4
:1042A000B0E083839483A583B6830E9421868DB773
:1042B0009EB706960FB6F8949EBF0FBE8DBF0E94A4
:1042C000040E00D000D000D080E497E0EDB7FEB738
:1042D0009283818380E290E0A0E0B0E083839483C6
:1042E000A583B6830E9421868DB79EB706960FB62A
:1042F000F8949EBF0FBE8DBF0E94040E00D000D068
:1043000000D083E397E0EDB7FEB79283818380E42A
:1043100090E0A0E0B0E083839483A583B6830E94FD
:1043200021868DB79EB706960FB6F8949EBF0FBE36
:104330008DBF0E94040E00D000D000D089E297E02B
:10434000EDB7FEB79283818380E890E0A0E0B0E013
:1043500083839483A583B6830E9421868DB79EB7FD
:1043600006960FB6F8949EBF0FBE8DBF0E94040E36
:1043700000D000D000D08DE197E0EDB7FEB792837A
:10438000818380E091E0A0E0B0E083839483A58303
:10439000B6830E9421868DB79EB706960FB6F89415
:1043A0009EBF0FBE8DBF0E94040E00D000D000D073
:1043B00083E197E0EDB7FEB79283818380E092E0DE
:1043C000A0E0B0E083839483A583B6830E94218616
:1043D0008DB79EB706960FB6F8949EBF0FBE8DBFE1
:1043E0000E94040E00D000D000D087E097E0EDB727
:1043F000FEB79283818380E094E0A0E0B0E0838305
:104400009483A583B6830E9421868DB79EB70696B6
:104410000FB6F8949EBF0FBE8DBF0E94040E00D051
:1044200000D000D089EF96E0EDB7FEB7928381838C
:1044300080E098E0A0E0B0E083839483A583B68316
:104440000E9421868DB79EB706960FB6F8949EBF40
:104450000FBE8DBF0E94040E00D000D000D08FEEA2
:1044600096E0EDB7FEB79283818380E090E1A0E013
:10447000B0E083839483A583B6830E9421868DB7A1
:104480009EB706960FB6F8949EBF0FBE8DBF0E94D2
:10449000040E00D000D000D083EE96E0EDB7FEB75A
:1044A0009283818380E090E2A0E0B0E083839483F4
:1044B000A583B6830E9421868DB79EB706960FB658
:1044C000F8949EBF0FBE8DBF0E94040E00D000D096
:1044D00000D089ED96E0EDB7FEB79283818380E04E
:1044E00090E4A0E0B0E083839483A583B6830E9428
:1044F00021868DB79EB706960FB6F8949EBF0FBE65
:104500008DBF0E94040E00D000D000D08FEC96E04A
:10451000EDB7FEB79283818380E090E8A0E0B0E041
:1045200083839483A583B6830E9421868DB79EB72B
:1045300006960FB6F8949EBF0FBE8DBF0E94040E64
:1045400000D000D000D085EC96E0EDB7FEB79283A6
:10455000818380E090E0A1E0B0E083839483A58331
:10456000B6830E9421868DB79EB706960FB6F89443
:104570009EBF0FBE8DBF0E94040E00D000D000D0A1
:1045800089EB96E0EDB7FEB79283818380E090E0FF
:10459000A2E0B0E083839483A583B6830E94218642
:1045A0008DB79EB706960FB6F8949EBF0FBE8DBF0F
:1045B0000E94040E00D000D000D08DEA96E0EDB746
:1045C000FEB79283818380E090E0A4E0B0E0838333
:1045D0009483A583B6830E9421868DB79EB70696E5
:1045E0000FB6F8949EBF0FBE8DBF0E94040E00D080
:1045F00000D000D081EA96E0EDB7FEB792838183C8
:1046000080E090E0A8E0B0E083839483A583B68344
:104610000E9421868DB79EB706960FB6F8949EBF6E
:104620000FBE8DBF0E94040E00D000D000D085E9DF
:1046300096E0EDB7FEB79283818380E090E0A0E141
:10464000B0E083839483A583B6830E9421868DB7CF
:104650009EB706960FB6F8949EBF0FBE8DBF0E9400
:10466000040E00D000D000D08BE896E0EDB7FEB786
:104670009283818380E090E0A0E2B0E08383948322
:10468000A583B6830E9421868DB79EB706960FB686
:10469000F8949EBF0FBE8DBF0E94040E00D000D0C4
:1046A00000D080E896E0EDB7FEB79283818380E08A
:1046B00090E0A0E4B0E083839483A583B6830E9456
:1046C00021868DB79EB706960FB6F8949EBF0FBE93
:1046D0008DBF0E94040E089500D080E796E0ADB72C
:1046E000BEB712969C938E9311970E9421860F90CD
:1046F0000F900E94C91B00D000D088E696E0EDB76D
:10470000FEB79283818386E798E1948383830E9436
:1047100021860F900F9084E696E0ADB7BEB7129653
:104720009C938E9311970E9421860F900F9080E0AA
:104730000E94111E00D08FE596E0EDB7FEB7928380
:1047400081830E9421860F900F900E941812809101
:10475000511D80FF05C081E061E041E00E947513BA
:104760000E94CE1B00D000D0EDB7FEB7319686E593
:1047700096E0ADB7BEB712969C938E931197809139
:104780001C05828313820E942186EDB7FEB7319605
:1047900089E496E0ADB7BEB712969C938E931197BD
:1047A00080913707828313820E94218681E396E0FD
:1047B000EDB7FEB79283818380E490E09483838396
:1047C0000E94218600D0EDB7FEB731968EE196E0CB
:1047D000ADB7BEB712969C938E9311978091CD255D
:1047E000828313828091CE25848315820E94218644
:1047F0000F900F90EDB7FEB7319685E196E0ADB71B
:10480000BEB712969C938E93119780911D0582835B
:1048100013820E94218680911A0590911B050F90AA
:104820000F900F900F9096FF03C08BEF92E002C0A5
:104830008EEF92E000D000D02BE036E0EDB7FEB76F
:1048400032832183948383830E94218686EF95E0BF
:10485000ADB7BEB712969C938E93119780911805B1
:104860009091190514969C938E9313970E9421861C
:1048700000D082EE95E0EDB7FEB792838183809100
:10488000140590911505A0911605B0911705838325
:104890009483A583B6830E9421868DB79EB7069622
:1048A0000FB6F8949EBF0FBE8DBF81E00E94191F06
:1048B0001D9B03C08BEF92E002C08EEF92E000D010
:1048C00000D026ED35E0ADB7BEB712963C932E93DF
:1048D000119714969C938E9313970E9421860F90A4
:1048E0000F908CEC95E0EDB7FEB7928381830E9428
:1048F000218680911A050F900F9081FF0EC000D085
:1049000086EC95E0ADB7BEB712969C938E93119747
:104910000E9421860F900F9017C080FF03C08BEF7D
:1049200092E002C08EEF92E000D000D022EC35E0A1
:10493000EDB7FEB732832183948383830E9421865F
:104940000F900F900F900F90809132079091330746
:1049500000D000D025EB35E0ADB7BEB712963C9342
:104960002E93119714969C938E9313970E942186F1
:104970000F900F900F900F90779903C08BEF92E0FC
:1049800002C08EEF92E000D000D02CEA35E0EDB707
:10499000FEB732832183948383830E9421860F9004
:1049A0000F900F900F900E9436090E94280D0E94D0
:1049B000050D00D000D000D02EE935E0ADB7BEB770
:1049C00012963C932E931197EDB7FEB763837483D1
:1049D000858396830E9421868DB79EB706960FB673
:1049E000F8949EBF0FBE8DBF81E090E00E94961CA0
:1049F0008091A8259091A925A091AA25B091AB25D9
:104A000000D000D000D020E935E0EDB7FEB732830A
:104A1000218383839483A583B6830E9421868CE7B8
:104A200095E0ADB7BEB712969C938E931197809187
:104A3000B5259091B625A091B725B091B825EDB7D1
:104A4000FEB783839483A583B6830E9421868091D9
:104A5000AC259091AD25A091AE25B091AF252EE665
:104A600035E0EDB7FEB73283218383839483A5833A
:104A7000B6830E9421868AE595E0ADB7BEB712964F
:104A80009C938E9311978091B9259091BA25A0910E
:104A9000BB25B091BC25EDB7FEB783839483A58376
:104AA000B6830E9421868DB79EB706960FB6F894FE
:104AB0009EBF0FBE8DBF80E090E061E070E00E947D
:104AC000100E81E090E061E070E00E94100E089509
:104AD0002F923F924F925F926F927F928F929F920E
:104AE000AF92BF92CF92DF92EF92FF920F931F93FC
:104AF000DF93CF9300D0CDB7DEB79A838983DC01F3
:104B00008D919C911197009711F00C942F38609122
:104B100002057091030588E691E20E947C8588E693
:104B200091E260E470E00E94A985009759F46091D9
:104B3000882E7091892E8AE090E00E94E38581E0C2
:104B40000C9435388130910549F420906821332444
:104B500044245524662477244301BFC18230910543
:104B600099F43091682120916921932F80E0820F80
:104B7000911D1C01892F880F880B482E582E682EF6
:104B8000782E882E982EA9C18330910509F09CC0FB
:104B900020916821A090692180906A2130E040E056
:104BA00050E060E070E080E090E000E10E94097970
:104BB000F22E132FE42ED52EC62EB72E282E992E88
:104BC0002A2D30E040E050E060E070E080E090E0CE
:104BD00008E00E9409792F0DB1E02F1508F0B0E030
:104BE000310FE1E0311708F0E0E0B30FF1E0B31767
:104BF00008F0F0E0EF2B4E0D31E04E1508F030E0FC
:104C0000E40FF1E0E41708F0F0E03F2B5D0D41E028
:104C10005D1508F040E0A32FA50F31E0A51708F0BF
:104C200030E0432B6C0D31E06C1508F030E0F42FD0
:104C3000F60F41E0F61708F040E0342B7B0D41E021
:104C40007B1508F040E0532F570F31E0571708F05D
:104C500030E0432B820D31E0821508F030E0480F40
:104C600061E0481708F060E0362B990D930F022F92
:104C7000080D11E0021708F010E01B0F81E01B1770
:104C800008F080E0B82FBE0F71E0BE1708F070E0AA
:104C90007A0F61E07A1708F060E06F0F31E06F176C
:104CA00008F030E0350F21E0351708F020E0240F40
:104CB00081E0241708F080E018014B2E572E662E55
:104CC000732E822E982EFEC0843091050CF4FCC009
:104CD00020916821A090692170906A2180906B21B9
:104CE00030E040E050E060E070E080E090E008E11B
:104CF0000E940979F22E132FE42ED52EC62EB72E40
:104D0000282E992E2A2D30E040E050E060E070E03F
:104D100080E090E000E10E9409792F0DF1E02F156D
:104D200008F0F0E0310FE1E0311708F0E0E0F30FB8
:104D3000A1E0F31708F0A0E0EA2B4E0D31E04E158C
:104D400008F030E0E40FA1E0E41708F0A0E03A2B0F
:104D50005D0D41E05D1508F040E0B32FB50F31E087
:104D6000B51708F030E0432B6C0D31E06C1508F0FE
:104D700030E0A42FA60F41E0A61708F040E0342B46
:104D80007B0D41E07B1508F040E0532F570F31E0D9
:104D9000571708F030E0432B820D31E0821508F000
:104DA00030E0480F61E0481708F060E0362B990EBC
:104DB000930E122F180D81E0121708F080E0282EB4
:104DC0002F0E81E02F1608F080E0F82EFE0E81E015
:104DD000FE1608F080E0E82EEB0E81E0EB1608F0FE
:104DE00080E0D82EDA0E81E0DA1608F080E0C82ED6
:104DF000C50E81E0C51608F080E0B82EB40E81E043
:104E0000B41608F080E0980E272D30E040E050E026
:104E100060E070E080E090E008E00E940979210FF6
:104E2000E1E0211708F0E0E0320DF1E0321508F082
:104E3000F0E0E30FA1E0E31708F0A0E0FA2B4F0D3C
:104E400031E04F1508F030E0F40FA1E0F41708F05E
:104E5000A0E03A2B5E0D41E05E1508F040E0A32F84
:104E6000A50F31E0A51708F030E0432B6D0D31E0C0
:104E70006D1508F030E0542F560F41E0561708F03A
:104E800040E0342B7C0D41E07C1508F040E0632FBE
:104E9000670F31E0671708F030E0432B8B0D31E0EE
:104EA0008B1508F030E0480F71E0481708F070E00B
:104EB000372B990D222E3E2E4F2E5A2E652E762EF2
:104EC000842E932E990E09C0BAE02B2E332444244D
:104ED000552466247724882499240E94040EB22D38
:104EE000B73691F4E32DEF3679F4F42DFC3661F406
:104EF000552051F4662041F4772031F4882021F4C4
:104F0000992011F40C944E339101A201B301C40114
:104F1000A7E6AA2EFFE6BF2EECE6CE2EDD24EE2479
:104F2000FF2400E010E00E947A79823008F0A6C2E7
:104F3000822D893689F4932D923771F4442061F4DF
:104F4000552051F4662041F4772031F4882021F473
:104F5000992011F40C94FB359101A201B301C40115
:104F600009E6A02E12E7B12ECC24DD24EE24FF2486
:104F700000E010E00E947A79823008F025C1A22D6D
:104F8000A53681F4B32DB43669F4442059F4552084
:104F900049F4662039F4772029F4882019F49920FF
:104FA00009F43CC79101A201B301C401B5E6AB2EDF
:104FB000A4E6BA2ECC24DD24EE24FF2400E010E089
:104FC0000E947A79823008F07EC0E22DE53781F4C4
:104FD000332071F4442061F4552051F4662041F4EB
:104FE000772031F4882021F4992011F40C940D31AC
:104FF0009101A201B301C401F5E7AF2EBB24CC247B
:10500000DD24EE24FF2400E010E00E947A79823053
:1050100018F5F22DF83611F00C942D38332011F0DC
:105020000C942D38442011F00C942D38552011F09B
:105030000C942D38662011F00C942D38772011F047
:105040000C942D38882011F00C942D38992011F0F3
:105050000C942D380C943030822D863781F4332017
:1050600071F4442061F4552051F4662041F4772016
:1050700031F4882021F4992011F40C941C31922DE4
:10508000943611F00C942D38A32DA13611F00C9408
:105090002D38442011F00C942D38552011F00C942B
:1050A0002D38662011F00C942D38772011F00C94D7
:1050B0002D38882011F00C942D38992011F00C9483
:1050C0002D380C946C36B22DB73789F4E32DEF36BA
:1050D00071F4442061F4552051F4662041F47720A6
:1050E00031F4882021F4992011F40C948434910136
:1050F000A201B301C401E7E7AE2E0FE6B02ECC2427
:10510000DD24EE24FF2400E010E00E947A79823052
:10511000C0F5F22DF43689F4832D893671F44420DC
:1051200061F4552051F4662041F4772031F4882051
:1051300021F4992011F40C94ED30922D953611F054
:105140000C942D38A32DAE3611F00C942D3844203C
:1051500011F00C942D38552011F00C942D38662048
:1051600011F00C942D38772011F00C942D388820F4
:1051700011F00C942D38992011F00C942D380C94CA
:10518000AE34B22DB33389F4E32DE13771F444200A
:1051900061F4552051F4662041F4772031F48820E1
:1051A00021F4992011F40C946C36F22DF53611F09F
:1051B0000C942D38832D823711F00C942D38442017
:1051C00011F00C942D381EC2922D923689F4A32D25
:1051D000A53671F4B42DB43659F4552049F466203F
:1051E00039F4772029F4882019F4992009F416C697
:1051F0009101A201B301C40112E6A12EB5E6BB2EB6
:10520000A4E6CA2EDD24EE24FF2400E010E00E9474
:105210007A79823008F098C0E22DE13389F4F32DD9
:10522000F43671F4842D813659F4552049F4662002
:1052300039F4772029F4882019F4992009F401C45D
:105240009101A201B301C401F1E3AF2EE4E6BE2E49
:1052500001E6C02EDD24EE24FF2400E010E00E94D1
:105260007A798230C0F5922D933789F4A32DA23735
:1052700071F4442061F4552051F4662041F4772004
:1052800031F4882021F4992011F40C944E36B22D7B
:10529000B33711F00C942D38E32DE33711F00C9453
:1052A0002D38442011F00C942D38552011F00C9419
:1052B0002D38662011F00C942D38772011F00C94C5
:1052C0002D38882011F00C942D38992011F00C9471
:1052D0002D380C945D36F22DF33691F4832D8436FF
:1052E00079F4942D913661F4552051F4662041F4FF
:1052F000772031F4882021F4992011F40C946C3635
:10530000A22DA83711F00C942D38B32DB43611F01E
:105310000C942D38E42DE13611F00C942D385520E5
:1053200011F00C942D38662011F00C942D38772054
:1053300011F00C942D38882011F00C942D38992000
:1053400011F00C942D3879C3F22DFD3691F4832D94
:10535000853779F4942D983661F4552051F4662000
:1053600041F4772031F4882021F4992011F40C9431
:105370007D369101A201B301C4011DE6A12EB5E75E
:10538000BB2EA8E6CA2EDD24EE24FF2400E010E0A8
:105390000E947A798230C8F5A22DA23791F4B32DFC
:1053A000B23779F4E42DE53661F4552051F46620E6
:1053B00041F4772031F4882021F4992011F40C94E1
:1053C000A733F22DF33611F00C942D38832D8D3642
:1053D00011F00C942D38942D983611F00C942D3832
:1053E000552011F00C942D38662011F00C942D38B6
:1053F000772011F00C942D38882011F00C942D3862
:10540000992011F00C942D3840C3A22DA33689F4B5
:10541000B32DB23371F4E42DE93659F4552049F433
:10542000662039F4772029F4882019F4992009F4AA
:1054300028C3F22DF43611F00C942D38832D8336C9
:1054400011F00C942D38942D9C3611F00C942D38BD
:10545000552011F00C942D38662011F00C942D3845
:10546000772011F00C942D38882011F00C942D38F1
:10547000992011F00C942D380C944B33A22DA633A7
:1054800091F4B32DB93679F4E42DE53761F4F52DB7
:10549000F53649F4662039F4772029F4882019F488
:1054A000992009F4E1C59101A201B301C401F6E319
:1054B000AF2EE9E6BE2E05E7C02E15E6D12EEE246E
:1054C000FF2400E010E00E947A79823008F04CC19D
:1054D000822D8C3691F4932D943779F4A42DA43732
:1054E00061F4552051F4662041F4772031F488208E
:1054F00021F4992011F40C945E379101A201B301BB
:10550000C401BCE6AB2EA4E7BA2EF4E7CF2EDD240F
:10551000EE24FF2400E010E00E947A79823008F047
:1055200087C0B22DB03391F4E32DE13379F4F42D3B
:10553000F13761F4552051F4662041F4772031F4BD
:10554000882021F4992011F40C94A7339101A20131
:10555000B301C401E0E3AE2E01E3B02E11E7C12E8A
:10556000DD24EE24FF2400E010E00E947A798230EE
:1055700028F5822D853711F00C942D38932D933614
:1055800011F00C942D38A42DAD3611F00C942D385B
:10559000552011F00C942D38662011F00C942D3804
:1055A000772011F00C942D38882011F00C942D38B0
:1055B000992011F00C942D380C940A34B22DB1338B
:1055C00091F4E32DE13379F4F42DF13761F45520B2
:1055D00051F4662041F4772031F4882021F4992099
:1055E00011F40C940A34822D803711F00C942D386C
:1055F000932D953611F00C942D38A42DA23711F06F
:105600000C942D38552011F00C942D38662011F093
:105610000C942D38772011F00C942D38882011F03F
:105620000C942D38992011F00C942D380C9482355F
:10563000B22DB43791F4E32DEF3679F4F42DFF3623
:1056400061F4852D823649F4662039F4772029F4F7
:10565000882019F4992009F44FC69101A201B301E1
:10566000C401B4E7AB2EAFE6BA2EFFE6CF2EE2E6DA
:10567000DE2EEE24FF2400E010E00E947A798230D2
:10568000C8F5922D943789F4A32DA83771F4B42D61
:10569000B43759F4552049F4662039F4772029F4B9
:1056A000882019F4992009F42AC6E22DE43711F074
:1056B0000C942D38F32DF43611F00C942D38842DE4
:1056C000873711F00C942D38552011F00C942D389B
:1056D000662011F00C942D38772011F00C942D38A1
:1056E000882011F00C942D38992011F00C942D384D
:1056F0000C94BE37922D993691F4A32DAC3679F4E3
:10570000B42DB13661F4E52DE33649F4662039F461
:10571000772029F4882019F4992009F4E2C1F22DA8
:10572000FE3611F00C942D38832D813611F00C9437
:105730002D38942D983611F00C942D38A52DA336C4
:1057400011F00C942D38662011F00C942D38772030
:1057500011F00C942D38882011F00C942D389920DC
:1057600011F00C942D389DC5B22DB13691F4E32D76
:10577000EC3679F4F42DF53661F4852D823749F451
:10578000662039F4772029F4882019F4992009F447
:1057900082C49101A201B301C40101E6A02E1CE65E
:1057A000B12EB5E6CB2EA2E7DA2EEE24FF2400E0E0
:1057B00010E00E947A79823008F0A0C0922D9237D2
:1057C00091F4A32DA73779F4B42DB03761F4E52D0A
:1057D000E03749F4662039F4772029F4882019F459
:1057E000992009F456C19101A201B301C401F2E765
:1057F000AF2EE7E7BE2E00E7C02E10E7D12EEE2435
:10580000FF2400E010E00E947A798230D8F5F22D72
:10581000F03791F4832D8C3679F4942D953661F41C
:10582000A52DA83649F4662039F4772029F488207C
:1058300019F4992009F414C4B22DB13611F00C9466
:105840002D38E32DED3611F00C942D38F42DF5376D
:1058500011F00C942D38852D883611F00C942D38CC
:10586000662011F00C942D38772011F00C942D380F
:10587000882011F00C942D38992011F00C942D38BB
:105880000C949D34922D933799F4A32DA53681F471
:10589000B42DB23769F4E52DE03751F4662041F4B8
:1058A000772031F4882021F4992011F40C94C73624
:1058B000F22DF33711F00C942D38832D823711F02F
:1058C0000C942D38942D973711F00C942D38A52D6C
:1058D000A03711F00C942D38662011F00C942D385F
:1058E000772011F00C942D38882011F00C942D386D
:1058F000992011F00C942D380C944E35B22DB737F9
:1059000091F4E32DE03779F4F42DF83761F4852D27
:10591000843749F4662039F4772029F4882019F473
:10592000992009F498C49101A201B301C401B7E719
:10593000AB2EA0E7BA2EF8E7CF2EE4E7DE2EEE245A
:10594000FF2400E010E00E947A798230D8F5922D91
:10595000943799F4A32DA33781F4B42DB53669F4A7
:10596000E52DE23751F4662041F4772031F48820A8
:1059700021F4992011F40C944B35F22DF43711F0E9
:105980000C942D38832D833711F00C942D38942DE1
:10599000953611F00C942D38A52DA43711F00C94E8
:1059A0002D38662011F00C942D38772011F00C94CE
:1059B0002D38882011F00C942D38992011F00C947A
:1059C0002D38C4C4B22DB23791F4E32DE73679F403
:1059D000F42DF03761F4852D853749F4662039F4CC
:1059E000772029F4882019F4992009F423C6922DF0
:1059F0009C3611F00C942D38A32DA13611F00C9487
:105A00002D38B42DB43711F00C942D38E52DE8372E
:105A100011F00C942D38662011F00C942D3877205D
:105A200011F00C942D38882011F00C942D38992009
:105A300011F00C942D380C9422370E94D0170C943E
:105A40002F3880ED61E04CE021E00E94C65F80EDE0
:105A500061E04EE021E00E94C65F80ED61E040E140
:105A600021E00E94C65F80ED61E042E121E00E94FA
:105A7000C65F80ED61E040E122E00E94C65F0C94C9
:105A80002F380E9418120C942F380E9459180C9429
:105A90002F38609102057091030580E090E00E942C
:105AA0007C858C016BEF72E00E949185009719F460
:105AB00077980C942F38C8016EEF72E00E949185A0
:105AC000009719F4779A0C942F38779903C08BEFCD
:105AD00092E002C08EEF92E000D000D02FE434E0DC
:105AE0002FC6609102057091030580E090E00E944E
:105AF0007C858C0162E073E00E949185009709F03B
:105B000052C0609102057091030580E090E00E9410
:105B10007C858C01009711F40C942F3865E073E0BC
:105B20000E949185009729F482E29FEFACECBBE3E1
:105B30000BC0C8016BE073E00E949185009769F487
:105B400082E29FEFACECBAE38093F5049093F60405
:105B5000A093F704B093F8041DC0C8010E946F849D
:105B60007B018C0120E030E0A9010E94337E882374
:105B7000B1F081E00E94A30C9B01AC01C801B70108
:105B80000E94377E6093F5047093F6048093F704C7
:105B90009093F80485EF94E066E070E0BEC000D01A
:105BA0008FE894E08CC0C80160E173E00E949185A9
:105BB000009709F052C0609102057091030580E0E2
:105BC00090E00E947C858C01009711F40C942F3892
:105BD00065E073E00E949185009729F482E29FEFCF
:105BE000ACECBBE30BC0C8016BE073E00E94918595
:105BF000009769F482E29FEFACECBAE38093F9047A
:105C00009093FA04A093FB04B093FC041DC0C80158
:105C10000E946F847B018C0120E030E0A9010E948A
:105C2000337E8823B1F082E00E94A30C9B01AC017B
:105C3000C801B7010E94377E6093F9047093FA049B
:105C40008093FB049093FC0489EF94E06AE070E099
:105C500064C000D082E894E067C0C80163E173E0EB
:105C60000E949185009709F06BC0609102057091C8
:105C7000030580E090E00E947C858C01009711F480
:105C80000C942F3865E073E00E949185009769F4C9
:105C900087ED94E3AFEEBCE38093F1049093F204BC
:105CA000A093F304B093F40434C0C8016BE073E034
:105CB0000E949185009741F400D083E794E0EDB70E
:105CC000FEB79283818336C0C8010E946F841B0196
:105CD0002C0120E030E0A9010E94337E882309F1E5
:105CE00080E00E94A30C7B018C01C201B10121EE76
:105CF0003AE744E95EE30E946C7DA80197010E94A7
:105D0000377E6093F1047093F2048093F3049093D0
:105D1000F40481EF94E062E070E044E050E00C9421
:105D2000013800D086E694E0ADB7BEB712969C93DA
:105D30008E9311970E9421860F900F900C942F380C
:105D40000E94F10C00D000D000D02FE534E0EDB778
:105D5000FEB732832183ADB7BEB713966D937D93A3
:105D60008D939C9316970E942186EDB7FEB73696C9
:105D70000FB6F894FEBF0FBEEDBF81E00E94A30CEA
:105D80002091F5043091F6044091F7045091F80405
:105D90000E947D7F7B018C0182E00E94A30C9B010D
:105DA000AC018DB79EB70A970FB6F8949EBF0FBE91
:105DB0008DBFCDB6DEB60894C11CD11C83E594E03E
:105DC000ADB7BEB712969C938E9311978E2D9F2DD3
:105DD000A02FB12FF60182839383A483B583CA01D8
:105DE000B9012091F9043091FA044091FB045091DB
:105DF000FC040E947D7FD60116966D937D938D9352
:105E00009C9319970E942186EDB7FEB73A960FB67C
:105E1000F894FEBF0FBEEDBF0C945B376091020596
:105E20007091030580E090E00E947C85009761F10D
:105E300060E070E040E150E00E9461832091320711
:105E4000309133072617370799F170933307609322
:105E5000320782E397E060E070E042E050E00E94A9
:105E60006A87809132079091330700D000D02FE3EA
:105E700034E0ADB7BEB712963C932E9311971496AB
:105E80009C938E9313970EC08091320790913307A5
:105E900000D000D02BE234E0EDB7FEB7328321838F
:105EA000948383830E9421860F900F900F900F9010
:105EB0000E94040E00D000D08EE194E0ADB7BEB7D2
:105EC00012969C938E93119781E090E014969C9388
:105ED0008E9313970E94218683E194E0EDB7FEB77D
:105EE0009283818382E090E0948383830E94218661
:105EF00088E094E0ADB7BEB712969C938E9311974D
:105F000084E090E014969C938E9313970E942186D0
:105F10008CEF93E0EDB7FEB79283818388E090E049
:105F2000948383830E94218681EF93E0ADB7BEB74F
:105F300012969C938E93119780E190E014969C9317
:105F40008E9313970E94218685EE93E0EDB7FEB7FE
:105F50009283818380E290E0948383830E942186F0
:105F600087ED93E0ADB7BEB712969C938E931197D1
:105F700080E490E014969C938E9313970E94218660
:105F800088EC93E0EDB7FEB79283818380E890E0E0
:105F9000948383830E94218689EB93E0ADB7BEB7DB
:105FA00012969C938E93119780E091E014969C93A7
:105FB0008E9313970E9421868DEA93E0EDB7FEB78A
:105FC0009283818380E092E0948383830E94218680
:105FD0008FE993E0ADB7BEB712969C938E9311975D
:105FE00080E094E014969C938E9313970E942186F0
:105FF00082E993E0EDB7FEB79283818380E098E079
:10600000948383830E94218684E893E0ADB7BEB772
:1060100012969C938E93119780E090E114969C9336
:106020008E9313970E94218685E793E0EDB7FEB724
:106030009283818380E090E2948383830E9421860F
:1060400087E693E0ADB7BEB712969C938E931197F7
:1060500080E090E414969C938E9313970C942638CA
:106060000E94DD1A0C942F3880916C21843329F41E
:1060700080E061E040E00E9475132091FD0422233E
:1060800011F40C942F3800D000D0EDB7FEB7319644
:1060900084E693E099C080916C21893709F088C02B
:1060A000609102057091030580E090E00E947C857C
:1060B0008C016BEF72E00E949185009731F4809122
:1060C0001A0590911B0590640CC0C8016EEF72E038
:1060D0000E949185009791F480911A0590911B057B
:1060E0009F7B90931B0580931A058AE195E064E1FC
:1060F00070E042E050E00E946A875AC0C80168E13F
:1061000073E00E9491850097A1F5EDB7FEB73A972D
:106110000FB6F894FEBF0FBEEDBF319680EA94E053
:10612000ADB7BEB712969C938E93119780918B1842
:1061300090918C189383828380918D1890918E1802
:106140009583848380918F1890919018978386838C
:106150008091911890919218918780870E94218652
:10616000EDB7FEB73A960FB6F894FEBF0FBEEDBF7F
:106170001FC080911A0590911B0596FF03C08BEFFD
:1061800092E002C08EEF92E000D000D02CE934E023
:10619000ADB7BEB712963C932E93119714969C936D
:1061A0008E9313970E9421860F900F900F900F905F
:1061B0002091FD04222309F452C700D000D0EDB78E
:1061C000FEB7319681E693E0ADB7BEB712969C93C9
:1061D0008E9311972283138239C7609102057091C3
:1061E000030580E090E00E947C8565E073E00E94FA
:1061F0009185009711F481E001C080E00E94111E9A
:106200002091FD04222309F42AC700D000D0EDB765
:10621000FEB731968EE593E0D7CF0E94CE1B20913A
:10622000FD04222309F41BC700D000D0EDB7FEB750
:1062300031968BE593E0C8CF0E94C91B2091FD04E5
:10624000222309F40CC700D000D0EDB7FEB7319679
:1062500088E593E0B9CF609102057091030580E075
:1062600090E00E947C850E947384803150F480937A
:10627000370790E00E94255D87E397E066E170E0D4
:1062800027C000D000D0EDB7FEB731968BEC94E07C
:10629000ADB7BEB712969C938E9311978091370736
:1062A00029C0609102057091030580E090E00E9492
:1062B0007C850E947384982F9B50903160F480936A
:1062C0001C0590E00E949D5B8CE195E067E170E029
:1062D00041E050E096C600D000D0EDB7FEB7319651
:1062E00088ED94E0ADB7BEB712969C938E9311974C
:1062F00080911C0582836FCF0C940000B0C6609122
:1063000002057091030580E090E00E947C85BC014D
:10631000009769F086E798E14AE050E00E949A858C
:1063200086E798E162E270E04AE050E06AC600D099
:1063300000D08EE193E0EDB7FEB79283818386E7CC
:1063400098E1948383830E940F8682C66091020540
:106350007091030580E090E00E947C858C0166E2EC
:1063600073E00E949185009739F4219A80911A0573
:1063700090911B0580613BC6C80168E273E00E94F2
:106380009185009739F4229A80911A0590911B0506
:1063900080622DC6C8016AE273E00E949185009771
:1063A00039F4239A80911A0590911B0580641FC6C9
:1063B000C8016CE273E00E949185009739F4239A3A
:1063C00080911A0590911B05806811C6C8016EE284
:1063D00073E00E9491850097C9F480911A0590910D
:1063E0001B05916090931B0580931A058AE195E047
:1063F00064E170E042E050E00E946A878EE595E03B
:1064000062E140E050E00E94BD4629C6C80160E359
:1064100073E00E949185009771F4E3E9F8E111922D
:10642000119288E1E33BF807D1F780911A0590912A
:106430001B059260DCC5C8016EEF72E00E94918579
:106440009C0180911A0590911B0521153105A9F435
:106450008F709C7F90931B0580931A052B9A8AE17D
:1064600095E064E170E042E050E00E946A8780912C
:10647000B42590E00E94B25BF2C584FF03C08BEFAD
:1064800092E002C08EEF92E000D000D028E135E02B
:10649000ADB7BEB712963C932E93119714969C936A
:1064A0008E9313970E94218680911A050F900F906A
:1064B0000F900F9085FF03C08BEF92E002C08EEF2C
:1064C00092E000D000D02DE035E0EDB7FEB732838A
:1064D0002183948383830E94218680911A050F90E3
:1064E0000F900F900F9086FF03C08BEF92E002C0D9
:1064F0008EEF92E000D000D022E035E0ADB7BEB71D
:1065000012963C932E93119714969C938E93139707
:106510000E94218680911A050F900F900F900F9086
:1065200087FF03C08BEF92E002C08EEF92E000D0B5
:1065300000D027EF34E0EDB7FEB732832183948398
:1065400083830E94218680911A0590911B050F90EC
:106550000F900F900F9090FF03C08BEF92E002C05E
:106560008EEF92E000D000D02CEE34E0ADB7BEB795
:1065700012963C932E93119714969C938E93139797
:106580000E94218680911A0590911B050F900F9013
:106590000F900F9091FF03C08BEF92E002C08EEF3F
:1065A00092E000D000D021EE34E0EDB7FEB73283A8
:1065B0002183948383830E94218680911A05909180
:1065C0001B050F900F900F900F9091FF48C582E32D
:1065D00093E00E94418603E918E18BE0C82ED12C9C
:1065E000BAE3EB2EB3E0FB2ED8018D919D918D0186
:1065F00000D000D000D0EDB7FEB73196ADB7BEB732
:106600001296FC92EE921197D382C2829583848374
:106610000E940F860894C11CD11CEDB7FEB73696B8
:106620000FB6F894FEBF0FBEEDBFFBE1CF16D1044D
:10663000D9F615C500D084E593E0ADB7BEB7129684
:106640009C938E9311970E9421862091FD040F90B8
:106650000F902223A9F000D000D0EDB7FEB73196FD
:1066600081E593E0ADB7BEB712969C938E931197D8
:10667000228313820E9421860F900F900F900F901B
:1066800088E10FB6F89480936000109260000FBE0E
:106690000C94007CE4C40E94CF53E1C460910205D5
:1066A0007091030580E090E00E947C851C016BEFF7
:1066B00072E00E949185009749F40E947C5A809173
:1066C0001A0590911B0581608D7F91C4C1016EEF09
:1066D00072E00E949185009741F40E94DE598091FA
:1066E0001A0590911B058C7F82C405E413E0C1015B
:1066F000B8010E949185009749F40E94DE5980916B
:106700001A0590911B058E7F826071C480911A05D5
:1067100081FF0BC000D000D087E295E0EDB7FEB757
:10672000928381831483038391C480FF03C08BEF22
:1067300092E002C08EEF92E000D000D023E235E07C
:10674000ADB7BEB712963C932E93119783CC00D071
:1067500087E293E0EDB7FEB7928381830E942186A2
:106760008DB79EB740970FB6F8949EBF0FBE8DBFF2
:10677000EDB7FEB7319689E093E0ADB7BEB712969C
:106780009C938E9311978091632190916421A091A5
:106790006521B091662182839383A483B583809120
:1067A000572190915821A0915921B0915A21868367
:1067B0009783A087B18780915B2190915C21A09104
:1067C0005D21B0915E2182879387A487B5878091F0
:1067D0005F2190916021A0916121B0916221868713
:1067E0009787A08BB18B0E9421862091FD04EDB785
:1067F000FEB772960FB6F894FEBF0FBEEDBF222310
:1068000009F42DC400D000D0EDB7FEB7319686E074
:1068100093E0DACCF89481E090E00E942F09182FE1
:1068200080E090E00E942F09082F7894F89483E08C
:1068300090E00E942F09F82E82E090E00E942F093C
:10684000E82E789400D000D000D02CEF32E0EDB7E5
:10685000FEB73283218320910419309105194091AC
:10686000061950910719ADB7BEB713962D933D93F6
:106870004D935C9316970E94218600D000D0EDB70F
:10688000FEB7319625ED32E0ADB7BEB712963C9318
:106890002E931197E2821382F48215820683178267
:1068A000108711860E942186EDB7FEB73A960FB683
:1068B000F894FEBF0FBEEDBF0E94711C20916600D0
:1068C00000D000D0EDB7FEB7319689EC92E0ADB7BD
:1068D000BEB712969C938E931197228313820E94C7
:1068E00021860F900F900F900F900E94040E209120
:1068F000FD04222309F4B3C300D000D0EDB7FEB7E6
:10690000319686EC92E060CC80E090E060E070E050
:106910000E94100E81E090E060E070E00E94100E96
:106920002091FD04222309F49AC300D000D0EDB7D2
:10693000FEB7319683EC92E047CC0E944C1A0E943D
:10694000040E2091FD04222309F489C300D000D055
:10695000EDB7FEB7319680EC92E036CC609102053F
:106960007091030580E090E00E947C856AE473E00A
:106970000E949185009741F5F89487E597E00E9481
:10698000B4470CC0C8010F960E94004B8BEA95E0FB
:10699000B8010E946E47C8010E947A48082F192F3B
:1069A0000115110579F704C087E597E00E94F547C6
:1069B00087E597E00E945A480097B1F787E597E08E
:1069C0000E94B04778945AC087E597E00E94B44788
:1069D000482F592F7A0100E513E04CC0EDB7FEB700
:1069E00074970FB6F894FEBF0FBEEDBF3196ADB7EA
:1069F000BEB712961C930E931197D7011A968C91DD
:106A00001A978283138212968C911297848315822F
:106A100013968C9113978683178214968C911497F2
:106A20008087118617968C911797828713861996FF
:106A30008C9119978487158615968C911597868762
:106A4000178618968C911897808B118A16968C91C0
:106A5000828B138A0E940F86EDB7FEB774960FB62D
:106A6000F894FEBF0FBEEDBFC7010E947A48482FC1
:106A7000592F7A01E114F10409F0B0CF2091FD04FF
:106A8000222309F4ECC200D000D0EDB7FEB7319656
:106A90008DEB92E099CB0E944B1EE1C26091020502
:106AA0007091030580E090E00E947C858C016FE886
:106AB00073E00E949185009731F480911A059091BE
:106AC0001B05937F94C2C8016BE073E00E9491851F
:106AD000009739F480911A0590911B05937F986077
:106AE00086C2C80164E973E00E949185009739F479
:106AF00080911A0590911B05937F946078C20E9443
:106B00003609ADC2609102057091030580E090E006
:106B10000E947C850097A9F160E070E040E150E0C0
:106B20000E94618360931405709315058093160588
:106B30009093170500D000D000D02AEA32E0EDB7DC
:106B4000FEB732832183ADB7BEB713966D937D93A5
:106B50008D939C9316970E942186EDB7FEB73696CB
:106B60000FB6F894FEBF0FBEEDBF84E195E06EE076
:106B700070E044E050E00E946A8781E00E94191FA3
:106B80006EC280E00E94191F0E94040E00D000D047
:106B900000D085E992E0ADB7BEB712969C938E9374
:106BA00011978091140590911505A0911605B0914B
:106BB0001705EDB7FEB783839483A583B6830E9440
:106BC00021868DB79EB706960FB6F8949EBF0FBE6E
:106BD0008DBF81E00E94191F0E94040E2091FD04C8
:106BE000222309F43CC200D000D0EDB7FEB73196A5
:106BF00082E992E0E9CA609102057091030580E0A4
:106C000090E00E947C85009741F160E070E04AE0EE
:106C100050E00E946183709319056093180500D0BD
:106C200000D0EDB7FEB7319625E732E0ADB7BEB77D
:106C300012963C932E931197738362830E94218650
:106C40000F900F900F900F9088E195E062E170E057
:106C500042E050E00E946A8714C000D000D084E572
:106C600092E0EDB7FEB792838183809118059091F1
:106C70001905948383830E9421860F900F900F90B3
:106C80000F902091FD04222309F4E9C100D000D027
:106C9000EDB7FEB7319681E592E096CA0E943D4B72
:106CA0002091FD04222309F4DAC100D000D0EDB711
:106CB000FEB731968EE492E087CA0E946C23209141
:106CC000FD04222309F4CBC100D000D0EDB7FEB7FC
:106CD00031968BE492E078CA80E090E00E94961CA6
:106CE0002091FD04222309F4BAC100D000D0EDB7F1
:106CF000FEB7319688E492E067CA0E949219009725
:106D0000B9F500D000D000D08DE392E0EDB7FEB72A
:106D10009283818380914D1990914E19A0914F19C2
:106D2000B091501983839483A583B6830E942186F2
:106D300080E392E0ADB7BEB712969C938E93119705
:106D40008091C9259091CA25A091CB25B091CC25E1
:106D5000EDB7FEB783839483A583B6830E94218613
:106D60008DB79EB706960FB6F8949EBF0FBE8DBF27
:106D70000E94040E2091FD04222309F470C100D06A
:106D800000D0EDB7FEB731968DE292E01DCA83E0E8
:106D900061E048E021E00E940F1500D000D000D053
:106DA00086E292E0EDB7FEB792838183809140192D
:106DB00090914119A0914219B09143198383948312
:106DC000A583B6830E94218600D000D0EDB7FEB720
:106DD000319685E192E0ADB7BEB712969C938E9343
:106DE00011978091441990914519A0914619B0913D
:106DF000471982839383A483B58380914819909126
:106E00004919A0914A19B0914B1986839783A0879D
:106E1000B1870E942186EDB7FEB73A960FB6F89477
:106E2000FEBF0FBEEDBF0E94040E2091FD04222381
:106E300009F415C100D000D0EDB7FEB7319682E15C
:106E400092E0C2C9609102057091030580E090E074
:106E50000E947C856FE973E00E9491850097B1F4F0
:106E6000609102057091030580E090E00E947C85AE
:106E7000009709F4F4C00E947384803108F0EFC0D9
:106E800090915201982B90935201E9C08091520148
:106E900000D000D029E435E0EDB7FEB7328321837E
:106EA00090E08F709070948383830E9421860F906E
:106EB0000F900F900F900E94040ED1C060910205B8
:106EC0007091030580E090E00E947C85009781F13D
:106ED00060E070E04AE050E00E943482603100F5EA
:106EE00060931D0500D000D0EDB7FEB7319685E068
:106EF00092E0ADB7BEB712969C938E9311976283C2
:106F000013820E9421860F900F900F900F908DE1B9
:106F100095E068E170E041E050E00E946A871FC0A0
:106F200000D000D0EDB7FEB731968CEF91E007C0EE
:106F300000D000D0EDB7FEB7319683EF91E0ADB74A
:106F4000BEB712969C938E93119780911D058283F4
:106F500013820E9421860F900F900F900F900E9435
:106F6000040E2091FD04222309F479C000D000D042
:106F7000EDB7FEB7319680EF91E026C9609102052A
:106F80007091030580E090E00E947C858C016BEF9E
:106F900072E00E949185009741F40E94C058809150
:106FA0001A0590911B05906122C0C8016EEF72E036
:106FB0000E949185009741F5F8940E94CE5888E18F
:106FC0000FB6F89480936000109260000FBE84B7F3
:106FD000877F84BF809160008861809360001092F9
:106FE0006000789480911A0590911B059F7E909384
:106FF0001B0580931A058AE195E064E170E042E0A8
:1070000050E00E946A872BC0C80164EA73E00E94C6
:1070100091859C0180911A0590911B0521153105E0
:1070200021F494FF1CC0F894FFCF94FF03C08BEFB2
:1070300092E002C08EEF92E000D000D026E535E06D
:10704000EDB7FEB732832183948383830E94218628
:107050000F900F900F900F9002C00E94B61AA98156
:10706000BA8111961C921E9283E00F900F90CF91DF
:10707000DF911F910F91FF90EF90DF90CF90BF9025
:10708000AF909F908F907F906F905F904F903F90C8
:107090002F900895F89491E2E0E0F0E0909357008B
:1070A0008491E2E0F0E0909357002491E4E0F0E076
:1070B00090935700E49190E0A0E0B0E0DC019927C4
:1070C000882730E040E050E0542F432F322F222712
:1070D000820F931FA41FB51F8E0F911DA11DB11DFF
:1070E0008093041990930519A0930619B09307197A
:1070F00078940895DF93CF93CDB7DEB761970FB63D
:10710000F894DEBF0FBECDBFCE0104966EE070E0F6
:1071100044E050E00E944C878C819D81AE81BF810C
:107120008F3F2FEF92072FEFA2072FEFB20749F4FF
:1071300084E195E06EE070E044E050E00E946A87F0
:1071400008C08093140590931505A0931605B0937D
:107150001705CE01029662E170E042E050E00E9425
:107160004C878A819B812FEF8F3F920779F48CE3C4
:1071700090E0909319058093180588E195E062E10D
:1071800070E042E050E00E946A8704C090931905C5
:1071900080931805CE01029664E170E042E050E071
:1071A0000E944C878A819B812FEF8F3F920779F451
:1071B0008AE090E490931B0580931A058AE195E09C
:1071C00064E170E042E050E00E946A8704C090935E
:1071D0001B0580931A05CE01029660E070E042E044
:1071E00050E00E944C878A819B812FEF8F3F92074E
:1071F00069F4109233071092320782E397E060E05F
:1072000070E042E050E00E946A8704C09093330728
:10721000809332078DEB95E269E170E049E050E040
:107220000E944C870E94BA0FCE01049666E070E07F
:1072300044E050E00E944C878C819D81AE81BF81EB
:107240008F3F2FEF92072FEFA2072FEFB20749F4DE
:1072500085EF94E066E070E044E050E00E946A87C9
:1072600008C085EF94E066E070E044E050E00E94E2
:107270004C87CE0104966AE070E044E050E00E9442
:107280004C878C819D81AE81BF818F3F2FEF92070C
:107290002FEFA2072FEFB20749F489EF94E06AE0DD
:1072A00070E044E050E00E946A8708C089EF94E0F3
:1072B0006AE070E044E050E00E944C87CE01049602
:1072C00062E070E044E050E00E944C878C819D8138
:1072D000AE81BF818F3F2FEF92072FEFA2072FEFD5
:1072E000B20749F481EF94E062E070E044E050E0DE
:1072F0000E946A8708C081EF94E062E070E044E099
:1073000050E00E944C87CE01019666E170E041E0BA
:1073100050E00E944C8789818F3F49F487E397E0D2
:1073200066E170E041E050E00E946A8708C087E3B0
:1073300097E066E170E041E050E00E944C87CE01AA
:10734000019667E170E041E050E00E944C8789813E
:107350008F3F49F48CE195E067E170E041E050E057
:107360000E946A8708C08CE195E067E170E041E027
:1073700050E00E944C87CE01019668E170E041E048
:1073800050E00E944C8789818F3F49F48DE195E060
:1073900068E170E041E050E00E946A8708C08DE13A
:1073A00095E068E170E041E050E00E944C87CE013A
:1073B000089662E270E04AE050E00E944C878885BF
:1073C0008F3F49F486E798E162E270E04AE050E0DE
:1073D0000E946A8708C086E798E162E270E04AE0AE
:1073E00050E00E944C8761960FB6F894DEBF0FBE46
:1073F000CDBFCF91DF9108950E94B4586C9A6B9ADB
:107400006A9A6F9A729A749A739A779A809880B3EC
:10741000897F80BB8398849887E080937E00549A0C
:107420000E944A380E947A3881E00E94170C80E05E
:1074300090E00E94CE0F0E943D5280911A0586FD79
:10744000239A0895CF93DF93EC0188819981009767
:1074500031F02BE0803D920709F099C08FC00E9467
:10746000FC3980911A0580FD06C081FF02C01D997C
:1074700002C00E94DE59809170008C7F8093700062
:107480008091B60080628093B6001092B20082E0D4
:107490008093B1008091B60090E087709070009763
:1074A000C9F78091700081608093700080E090E067
:1074B0006DE579E00E9497580E94C91B80E00E9408
:1074C000111E00D08AEE91E0ADB7BEB712969C9324
:1074D0008E9311970E9421860F900F900E94181290
:1074E0008091511D86FF02C00E947A538091370718
:1074F00090E00E94255D80911C0590E00E949D5BBC
:107500000E949A5B8093650780911C0590E00E9421
:107510009D5B00D000D000D0EDB7FEB7319689EA70
:1075200093E0ADB7BEB712969C938E93119780915E
:1075300065078283138280913707848315820E94B6
:107540000F861092640710926307EDB7FEB7369668
:107550000FB6F894FEBF0FBEEDBF8AE295E09093A0
:10756000C7258093C62583E290E090935C078093C3
:107570005B0780ED9BE0998388830DC0633259F4EB
:1075800083E697E060E070E00E946825E6CF19820C
:10759000188283E001C081E0DF91CF9108958436A5
:1075A000910564F1209132073091330720FF10C01C
:1075B00000D000D02BEB33E0EDB7FEB73283218350
:1075C000948383830E940F860F900F900F900F90EB
:1075D0008091632190916421A0916521B0916621F1
:1075E0000196A11DB11D8093632190936421A09306
:1075F0006521B093662121E030E002C020E030E058
:10760000C90108954F925F926F927F928F929F92DD
:10761000AF92BF92CF92DF92EF92FF920F931F93A0
:10762000DF93CF93CDB7DEB7CB58D0400FB6F894E9
:10763000DEBF0FBECDBF2C01633871F483E497E049
:10764000C557DF4F6883CB58D0400E94F444C557DC
:10765000DF4F6881CB58D040D2012D913C911197DA
:10766000BBE023383B0711F40C940C44EBE02438C6
:107670003E0750F421153105A9F0FAE02D353F07FA
:1076800011F00C945E441AC04BE02439340711F415
:107690000C9435445BE02B39350711F00C945E44B3
:1076A0000C944D4483E497E061E870E047EA55E0CC
:1076B0000E94D9448DE59AE00C940744623111F0A0
:1076C0000C94644480911A0590911B0591FDF2CFB2
:1076D0008091140590911505A0911605B09117059C
:1076E000A0FD8C9A0E94280D80911405909115059B
:1076F000A0911605B091170594FF02C00E9492193F
:107700008091140590911505A0911605B09117056B
:1077100095FF0AC00E94F10C6093B0257093B125CB
:107720008093B2259093B3258091140580FF32C0D9
:10773000EDB7FEB738970FB6F894FEBF0FBEEDBF9A
:107740003196CE014396ADB7BEB712969C938E93F9
:10775000119787E790E0938382838FEC93E0958382
:10776000848386E798E1978386830E947886E82E53
:10777000092FEDB7FEB738960FB6F894FEBF0FBECF
:10778000EDBF0E94CF3A009709F094CF802F0E2DC5
:10779000182F02C000E010E08091140581FF5FC047
:1077A00043E1C42ED12CCC0EDD1E00D000D000D081
:1077B000EDB7FEB73196C601800F911FADB7BEB7CA
:1077C00012969C938E93119787E790E09383828320
:1077D00087ED93E0958384830E947886080F191FB4
:1077E0003DEBE32E35E2F32EEDB7FEB736960FB63E
:1077F000F894FEBF0FBEEDBF27E7A22EB12C97E98C
:10780000892E92E0992ED7012D917D01EDB7FEB71B
:1078100038970FB6F894FEBF0FBEEDBF3196C60184
:10782000800F911FADB7BEB712969C938E931197A0
:10783000B382A28295828482268317820E947886F0
:10784000080F191FEDB7FEB738960FB6F894FEBFB4
:107850000FBEEDBFF5ECEF16F5E2FF06A1F6809145
:10786000140582FF6EC083E1C82ED12CCC0EDD1E24
:1078700000D000D000D0EDB7FEB73196C601800F22
:10788000911FADB7BEB712969C938E93119787E761
:1078900090E0938382838BED93E0958384830E94B1
:1078A0007886080F191F7E010894E11CF11C80E105
:1078B000F70111928A95E9F72DB73EB72A5F3F4F3E
:1078C0000FB6F8943EBF0FBE2DBF80EB68E9A7014D
:1078D00028E00E942D13B9E0AB2EB12CAC0EBD1EDA
:1078E000A7E78A2E912CF7E96F2EF2E07F2ED701C1
:1078F0002D917D01EDB7FEB738970FB6F894FEBF16
:107900000FBEEDBF3196C601800F911FADB7BEB758
:1079100012969C938E9311979382828275826482D1
:10792000268317820E947886080F191FEDB7FEB7CD
:1079300038960FB6F894FEBF0FBEEDBFEA14FB04F5
:10794000B1F68091140590911505A0911605B0919E
:1079500017050097A105B10581F12DB73EB7285055
:1079600030400FB6F8943EBF0FBE2DBFEDB7FEB747
:107970003196CE014396800F911FADB7BEB71296D8
:107980009C938E93119787E790E09383828380EE98
:1079900093E0958384838091350790913607978390
:1079A00086830E947886080F191FEDB7FEB73896B8
:1079B0000FB6F894FEBF0FBEEDBF8091140583FF94
:1079C00050C089E290E06BE270E04AE250E027E0CC
:1079D0000E94534F8DEB95E20E94C3512DB73EB7E5
:1079E0002A5030400FB6F8943EBF0FBE2DBFEDB603
:1079F000FEB60894E11CF11C9E012D5E3F4F200F46
:107A0000311FADB7BEB712963C932E93119727E75F
:107A100030E0F7013383228327EE33E0358324837C
:107A20009C01B901882777FD8095982F0E94A17E3F
:107A300020E030E048EC52E40E94377ED7011696F1
:107A40006D937D938D939C9319970E947886080F70
:107A5000191FEDB7FEB73A960FB6F894FEBF0FBEEA
:107A6000EDBF8091140584FF56C089E290E06BE27F
:107A700070E04AE250E026E00E94534F81E090E03F
:107A80000E94780D809339078CEB98E10E94C351D6
:107A90002DB73EB72A5030400FB6F8943EBF0FBE08
:107AA0002DBFEDB6FEB60894E11CF11C9E012D5EC3
:107AB0003F4F200F311FADB7BEB712963C932E93A8
:107AC000119727E730E0F7013383228321EF33E07A
:107AD000358324839C01B901882777FD8095982FF1
:107AE0000E94A17E20E030E048EC52E40E94377E04
:107AF000D70116966D937D938D939C9319970E9451
:107B00007886080F191FEDB7FEB73A960FB6F894AE
:107B1000FEBF0FBEEDBF8091140585FF36C02DB7A7
:107B20003EB72A5030400FB6F8943EBF0FBE2DBF6F
:107B3000EDB7FEB73196CE014396800F911FADB7DA
:107B4000BEB712969C938E93119787E790E093832C
:107B500082838CEF93E09583848380918018909149
:107B60008118A0918218B091831886839783A0878B
:107B7000B1870E947886080F191FEDB7FEB73A96B5
:107B80000FB6F894FEBF0FBEEDBF8091140586FFBF
:107B900031C00E94050D2DB73EB72A5030400FB6B8
:107BA000F8943EBF0FBE2DBFEDB7FEB731969E01D4
:107BB0002D5E3F4F200F311FADB7BEB712963C93DD
:107BC0002E93119727E730E0338322832AE034E0B5
:107BD0003583248366837783808791870E947886A4
:107BE000080F191FEDB7FEB73A960FB6F894FEBF0F
:107BF0000FBEEDBF8091140587FF3AC0F8948091C5
:107C0000A8259091A925A091AA25B091AB2578949B
:107C10002DB73EB72A5030400FB6F8943EBF0FBE86
:107C20002DBF4DB75EB74F5F5F4F9E012D5E3F4F3B
:107C3000200F311FEDB7FEB73283218327E730E0F5
:107C4000FA013383228328E134E035832483868359
:107C50009783A087B1870E947886080F191F2DB7D8
:107C60003EB7265F3F4F0FB6F8943EBF0FBE2DBF05
:107C70008091140590911505A0911605B0911705F6
:107C800090FF92C08091180590911905009709F412
:107C90008BC0F894C090A825D090A925E090AA2583
:107CA000F090AB2578948091B4189091B518A0917C
:107CB000B618B091B718A7019601281B390B4A0BCB
:107CC0005B0BCA01B9010E949F7E862EA72E682EEB
:107CD000B92E609118057091190580E090E00E941E
:107CE0009F7E9B01AC01682D7A2D862D9B2D0E94D5
:107CF000377E5C014DB75EB74A5050400FB6F894DE
:107D00005EBF0FBE4DBFEDB7FEB73196CE014396B5
:107D1000800F911FADB7BEB712969C938E931197AB
:107D200087E790E09383828381E294E09583848364
:107D3000262F372F4A2D5B2D268337834087518787
:107D4000C557DF4F6883CB58D040C657DF4F788385
:107D5000CA58D0400E947886080F191FC557DF4FB8
:107D60006881CB58D040C657DF4F7881CA58D04081
:107D7000862F972FAA2DBB2D8093B5259093B625DE
:107D8000A093B725B093B825C092B418D092B51877
:107D9000E092B618F092B718EDB7FEB73A960FB664
:107DA000F894FEBF0FBEEDBF8091140590911505AC
:107DB000A0911605B091170591FF40C0F8948091ED
:107DC000AC259091AD25A091AE25B091AF257894CA
:107DD0002DB73EB72A5030400FB6F8943EBF0FBEC5
:107DE0002DBF4DB75EB74F5F5F4F9E012D5E3F4F7A
:107DF000200F311FEDB7FEB73283218327E730E034
:107E0000FA01338322832EE234E035832483868390
:107E10009783A087B1870E947886080F191F2DB716
:107E20003EB7265F3F4F0FB6F8943EBF0FBE2DBF43
:107E3000C8010E94CF3A009709F03CCC809114050C
:107E400090911505A0911605B091170592FF92C06B
:107E50008091180590911905009709F48BC0F8944A
:107E6000C090AC25D090AD25E090AE25F090AF2528
:107E700078948091B8189091B918A091BA18B091DF
:107E8000BB18A7019601281B390B4A0B5B0BCA01D3
:107E9000B9010E949F7E862EA72E682EB92E609172
:107EA00018057091190580E090E00E949F7E9B016B
:107EB000AC01682D7A2D862D9B2D0E94377E5C01AA
:107EC0004DB75EB74A5050400FB6F8945EBF0FBE34
:107ED0004DBFEDB7FEB73196CE014396800F911F8F
:107EE000ADB7BEB712969C938E93119787E790E03B
:107EF0009383828387E394E095838483262F372FAF
:107F00004A2D5B2D2683378340875187C557DF4F26
:107F10006883CB58D040C657DF4F7883CA58D040CB
:107F20000E947886080F191FC557DF4F6881CB580C
:107F3000D040C657DF4F7881CA58D040862F972F40
:107F4000AA2DBB2D8093B9259093BA25A093BB256C
:107F5000B093BC25C092B818D092B918E092BA1864
:107F6000F092BB18EDB7FEB73A960FB6F894FEBF85
:107F70000FBEEDBF8091140590911505A0911605D7
:107F8000B091170593FF3EC08091532190915421E9
:107F9000A0915521B09156212DB73EB72A503040BF
:107FA0000FB6F8943EBF0FBE2DBF4DB75EB74F5F03
:107FB0005F4F9E012D5E3F4F200F311FEDB7FEB783
:107FC0003283218327E730E0FA013383228324E4DC
:107FD00034E03583248386839783A087B1870E940A
:107FE0007886080F191F2DB73EB7265F3F4F0FB693
:107FF000F8943EBF0FBE2DBFC8010E94CF3A009734
:1080000009F058CB8091140590911505A0911605A3
:10801000B091170594FF3CC04DB75EB74A50504031
:108020000FB6F8945EBF0FBE4DBFEDB7FEB73196E9
:10803000CE014396800F911FADB7BEB712969C93A9
:108040008E93119787E790E0938382838DE494E089
:108050009583848380914D1990914E19A0914F1969
:10806000B091501986839783A087B1870E94788644
:10807000080F191FEDB7FEB73A960FB6F894FEBF7A
:108080000FBEEDBFC8010E94CF3A009709F012CB96
:108090008091140590911505A0911605B0911705D2
:1080A00095FF3CC02DB73EB72A5030400FB6F8942C
:1080B0003EBF0FBE2DBFEDB7FEB73196CE01439642
:1080C000800F911FADB7BEB712969C938E931197F8
:1080D00087E790E09383828388E594E095838483A7
:1080E0008091B0259091B125A091B225B091B32592
:1080F00086839783A087B1870E947886080F191F0F
:10810000EDB7FEB73A960FB6F894FEBF0FBEEDBFBF
:10811000C8010E94CF3A009709F0CCCA809114059B
:1081200090911505A0911605B091170596FF48C0CE
:1081300081E00E94A30C2DB73EB72A5030400FB605
:10814000F8943EBF0FBE2DBFEDB6FEB60894E11CFD
:10815000F11C9E012D5E3F4F200F311FADB7BEB702
:1081600012963C932E93119727E730E0F701338363
:10817000228325E634E0358324832091F504309171
:10818000F6044091F7045091F8040E947D7FD701D6
:1081900016966D937D938D939C9319970E94788684
:1081A000080F191FEDB7FEB73A960FB6F894FEBF49
:1081B0000FBEEDBFC8010E94CF3A009709F07ACAFE
:1081C0008091140590911505A0911605B0911705A1
:1081D00097FF48C082E00E94A30C2DB73EB72A50FB
:1081E00030400FB6F8943EBF0FBE2DBFEDB6FEB6C1
:1081F0000894E11CF11C9E012D5E3F4F200F311FA2
:10820000ADB7BEB712963C932E93119727E730E097
:10821000F7013383228322E734E0358324832091DE
:10822000F9043091FA044091FB045091FC040E943F
:108230007D7FD70116966D937D938D939C931997AF
:108240000E947886080F191FEDB7FEB73A960FB651
:10825000F894FEBF0FBEEDBFC8010E94CF3A009751
:1082600009F028CA8091140590911505A091160572
:10827000B0911705A0FF39C083E00E94A30C2DB771
:108280003EB72A5030400FB6F8943EBF0FBE2DBF08
:10829000EDB7FEB731969E012D5E3F4F200F311F87
:1082A000ADB7BEB712963C932E93119727E730E0F7
:1082B000338322832FE734E03583248366837783F7
:1082C000808791870E947886080F191F8C98EDB7D8
:1082D000FEB73A960FB6F894FEBF0FBEEDBFC801C9
:1082E0000E94CF3A009709F0E5C98091140590915A
:1082F0001505A0911605B0911705A1FF3FC080910B
:10830000511D87FF3BC080ED61E042E121E00E940A
:10831000C65F2DB73EB72A5030400FB6F8943EBF27
:108320000FBE2DBFEDB7FEB731969E012D5E3F4FBC
:10833000200F311FADB7BEB712963C932E93119705
:1083400027E730E0338322832CE834E0358324832D
:1083500066837783808791870E947886080F191F2C
:10836000EDB7FEB73A960FB6F894FEBF0FBEEDBF5D
:10837000C8010E94CF3A009709F09CC9809114056A
:1083800090911505A0911605B0911705A2FF3FC069
:108390008091511D87FF3BC080ED62E042E121E00A
:1083A0000E94C65F2DB73EB72A5030400FB6F894F2
:1083B0003EBF0FBE2DBFEDB7FEB731969E012D5EBD
:1083C0003F4F200F311FADB7BEB712963C932E938F
:1083D000119727E730E0338322832AE934E035839D
:1083E000248366837783808791870E947886080F2D
:1083F000191FEDB7FEB73A960FB6F894FEBF0FBE41
:10840000EDBFC8010E94CF3A009709F053C980918F
:10841000140590911505A0911605B0911705A3FFBD
:108420003FC08091511D87FF3BC080ED63E042E17A
:1084300021E00E94C65F2DB73EB72A5030400FB6EC
:10844000F8943EBF0FBE2DBFEDB7FEB731969E012B
:108450002D5E3F4F200F311FADB7BEB712963C9334
:108460002E93119727E730E03383228328EA34E004
:108470003583248366837783808791870E947886FB
:10848000080F191FEDB7FEB73A960FB6F894FEBF66
:108490000FBEEDBFC8010E94CF3A009709F00AC98C
:1084A0008091140590911505A0911605B0911705BE
:1084B000A4FF3FC08091511D87FF3BC080ED64E069
:1084C00042E121E00E94C65F2DB73EB72A503040FE
:1084D0000FB6F8943EBF0FBE2DBFEDB7FEB7319675
:1084E0009E012D5E3F4F200F311FADB7BEB71296D4
:1084F0003C932E93119727E730E03383228326EBBA
:1085000034E03583248366837783808791870E9454
:108510007886080F191FEDB7FEB73A960FB6F89494
:10852000FEBF0FBEEDBFC8010E94CF3A009709F011
:10853000C1C88091140590911505A0911605B091C0
:108540001705A5FF06C083E061E046E020E00E9439
:108550000F158091140590911505A0911605B09105
:108560001705A6FF06C083E061E046E021E00E9417
:108570000F158091140590911505A0911605B091E5
:108580001705A5FF3CC02DB73EB72A5030400FB6A7
:10859000F8943EBF0FBE2DBFEDB7FEB73196CE01AA
:1085A0004396800F911FADB7BEB712969C938E93E2
:1085B000119787E790E09383828384EC94E095831E
:1085C00084838091441990914519A0914619B091E6
:1085D000471986839783A087B1870E947886080F02
:1085E000191FEDB7FEB73A960FB6F894FEBF0FBE4F
:1085F000EDBFC8010E94CF3A009709F05BC8809197
:10860000140590911505A0911605B0911705A6FFC8
:108610003CC02DB73EB72A5030400FB6F8943EBF4D
:108620000FBE2DBFEDB7FEB73196CE014396800F3A
:10863000911FADB7BEB712969C938E93119787E7A3
:1086400090E0938382838CEC94E095838483809183
:10865000481990914919A0914A19B0914B198683F4
:108660009783A087B1870E947886080F191FEDB7FE
:10867000FEB73A960FB6F894FEBF0FBEEDBFC80125
:108680000E94CF3A009709F015C8779A8091320777
:108690009091330792FD749A80913207909133073D
:1086A00082FD08C080911A0580FD04C081FF31C0A1
:1086B0001D9B2FC000D000D087ED94E0ADB7BEB7B2
:1086C00012969C938E931197CE01439614969C9389
:1086D0008E9313970E940F862091FD040F900F90A8
:1086E0000F900F902223A9F000D000D0EDB7FEB775
:1086F000319684EE91E0ADB7BEB712969C938E93FF
:108700001197228313820E9421860F900F900F9061
:108710000F9080911D058061898B809156078A8B0F
:10872000FE01E00FF11F138A68010894C11CD11CDF
:10873000809132079091330780FF12C000D000D0A3
:108740008EED94E0EDB7FEB7928381830D5F1F4FEE
:10875000148303830E940F860F900F900F900F9049
:10876000E2E0EE2EF12CEC0CFD1C8E010F5E1F4F93
:10877000C801B7010E94514E80911A0582FF08C0BE
:1087800084E095E0B801A70128EA31E20E94D652C0
:10879000809132079091330782FD73980E947C5A32
:1087A00083E497E00E94F74480911A0590911B059D
:1087B00090FF43C000911805109119050E949A5B23
:1087C000E82E109219051092180589E190E00E9498
:1087D000B25B24C07398809156078F5F80935607D1
:1087E0008A8BB6016F5F7F4FCE0141960E94514E3A
:1087F00083E497E00E94F74480916C0F90916D0F95
:1088000065E840E050E00E94BD4683E89BE0D2016D
:1088100011969C938E9358C0CC24DD2420911A0588
:1088200030911B0530FDD6CF8E2D90E00E94B25BBB
:108830001093190500931805739A8091350790914C
:108840003607009711F00E94DE59809156078F5F1E
:1088500080935607809132079091330782FD02C0C2
:108860000C945A3B739A0C945A3B8EE497E00E9406
:108870009E49009749F10E947C5A80911A0587FD14
:108880002B988EE497E060E470E00E9473498BE9D6
:108890009BE0F2019183808317C08EE497E00E94F1
:1088A0009E49009789F00E94DE5980911A0587FD44
:1088B00002C00C945A3B2B9A0C945A3BD20111964D
:1088C0001C921E9283E001C081E0C557DF4F0FB6B6
:1088D000F894DEBF0FBECDBFCF91DF911F910F91F6
:1088E000FF90EF90DF90CF90BF90AF909F908F90D0
:1088F0007F906F905F904F9008950E94214508955A
:108900000895FC01DB018C91808311968C91119765
:1089100081830895FC01DB0190818C91981741F4CB
:1089200021E030E0918111968C911197981711F008
:1089300020E030E0C9010895FC0180818093CD25BD
:1089400081818093CE250895DC011996ED91FC91EB
:108950001A970280F381E02D309709F00995089568
:10896000EF92FF920F931F93DF93CF9300D0CDB779
:10897000DEB78C0188E10E94CC4EBC017E010894D8
:10898000E11CF11CC7010E948144D8011996ED91A8
:10899000FC911A970190F081E02DC801B70109956B
:1089A0000F900F90CF91DF911F910F91FF90EF905B
:1089B0000895EF92FF920F931F93CF93DF93EC01F3
:1089C0008B017A0147EB55E00E940545FA86E9865E
:1089D000C8016BEB75E00E946445DF91CF911F9158
:1089E0000F91FF90EF9008950E941E450895CF9338
:1089F000DF93EC0188E16DEC75E20E94C24ECE017E
:108A00000E942145DF91CF910895EF92FF920F933D
:108A10001F93CF93DF93EC018B017A010E943D45B8
:108A2000F886EF82C8016FEB75E00E946445DF9124
:108A3000CF911F910F91FF90EF9008950E944645AE
:108A400008950E9443610895FC01A781B0852D918E
:108A50003C91F90109950895DC011796ED91FC917F
:108A600018970280F381E02D309709F00995089559
:108A700088E69FE00E94B0470895FC0173836283FB
:108A800088E69FE0BF010E943B480895BC0188E64C
:108A90009FE00E9402480895CF93DF93EC0188E69F
:108AA0009FE00E94B44708C0828193818C179D0784
:108AB00039F0CF010E947A48E82FF92F3097A1F7BB
:108AC000CF01DF91CF9108950F931F93CF93DF9341
:108AD0008B010E944C45EC01009731F01D830C8303
:108AE000C8010E949B638E83DF91CF911F910F91EC
:108AF00008951F93CF93DF93EC01162F888580FF95
:108B00001DC0EC81FD813097C9F0D0936D0FC093EB
:108B10006C0F82E08887CE0106960995992787FD1C
:108B2000909502978230910510F0133829F4CE0108
:108B3000BE010E94A24502C081E08887DF91CF91EB
:108B40001F910895CF92DF92EF92FF920F931F93A0
:108B5000CF93DF93EC017B01C0906C0FD0906D0F31
:108B600000916A0F10916B0FF80103C00190F08122
:108B7000E02DEC17FD0719F03097C1F746C020979C
:108B800009F443C08885882309F118860BC0C017F3
:108B9000D10729F0C80167E8AE010E947945F801C4
:108BA000008111810115110591F7EC81FD8130974C
:108BB00069F0CE15DF0551F0D0936D0FC0936C0FA7
:108BC000CE01069663E840E050E00995E0916A0F17
:108BD000F0916B0FCE17DF0791F488819981909304
:108BE0006B0F80936A0F0DC0808191818C179D0758
:108BF00029F4888199819183808303C0FC01309797
:108C000099F7D0926D0FC0926C0FDF91CF911F91A9
:108C10000F91FF90EF90DF90CF9008951F93CF9327
:108C2000DF9310926E0FC0916A0FD0916B0F11E01D
:108C30000EC08985882341F018871986CE0162E825
:108C400040E050E00E9479450990D881C02D2097DE
:108C500081F7DF91CF911F91089580911910982F7E
:108C60009F5F90931910089560916C0F70916D0F34
:108C70000E94A24508958AE8809319101092700FFF
:108C800010926F0F10926B0F10926A0F10926D0F6F
:108C900010926C0F089580916E0F882311F00E943E
:108CA0000E4670916F0F772309F455C02091700F15
:108CB00030E0F901EE0FFF1FEE0FFF1FE20FF31F71
:108CC000EF58F04F608160931810418152815093AA
:108CD0001710409316108381948190931510809300
:108CE00014102F5F3F4F2F7130702093700F715011
:108CF00070936F0F009741F580916A0F90916B0F01
:108D000018C080916E0F882311F00E940E4640918A
:108D100016105091171080911210909113106091BD
:108D200018100E947945E0911210F0911310808183
:108D30009181909313108093121080911210909152
:108D400013100097F1F607C0613819F421E0FC0117
:108D500020870E94794580916E0F20916F0F30E03F
:108D6000280F311DC901089580916E0F20916F0F5A
:108D700030E0280F311DC901089570916F0F7032D6
:108D8000D9F02091700F270F2F712093111030E030
:108D9000F901EE0FFF1FEE0FFF1FE20FF31FEF5859
:108DA000F04F608352834183948383837F5F70930A
:108DB0006F0F20E030E002C021E030E0C9010895EB
:108DC000CF93DF93C0916C0FD0916D0F0E947945C6
:108DD000D0936D0FC0936C0FDF91CF910895FC017C
:108DE000AB0190916A0F80916B0F9C01A32FB22F62
:108DF00003C00D90BC91A02DAE17BF0791F0109746
:108E0000C1F7309771F090838183F0936B0FE093FB
:108E10006A0F81E0808717821682CF0161E80E9485
:108E2000E0460895FC01009741F080858150823032
:108E300020F481E0818780936E0F089521E030E077
:108E4000FC018085882311F420E030E0C9010895F9
:108E5000CF93DF93EC014A815B818C819D8160E03F
:108E600070E00E948A854A815B8188819981489F50
:108E70009001499F300D589F300D11248E819F81A4
:108E800060E070E0A9010E948A85DF91CF9108958A
:108E9000FC018281938120E030E019C0A481B5817A
:108EA000A20FB31F4C91442381F481E08C93408145
:108EB0005181249FC001259F900D349F900D112456
:108EC00026813781280F391F07C02F5F3F4F281792
:108ED000390720F320E030E0C9010895FC01268124
:108EE00037814281538180E090E018C02617370710
:108EF00081F4A481B581A80FB91F2C91121614F426
:108F000021502C930480F581E02DE80FF91F80811A
:108F10000895A081B1812A0F3B1F01968417950700
:108F200028F38FEF0895FC01CB012681378162176A
:108F3000730790F0A081B18162817381A69FA00127
:108F4000A79F500DB69F500D1124420F531F21E0D3
:108F500030E08417950710F020E030E0C901089553
:108F6000FC01118210820895FC0180819181089595
:108F7000FB0120813181FC01318320830895FC01B4
:108F8000208131812115310511F407C09C01F901BF
:108F9000808191810097D1F702C020E030E0C901C3
:108FA0000895CF93DF93DC012D913C91119721150A
:108FB0003105A9F0F90180819181009729F411967A
:108FC0001C921E920EC0F90120813181D9018D9130
:108FD0009C9111970097B9F71182108202C020E08E
:108FE00030E0C901DF91CF910895DC01ED91FC9152
:108FF0001197309729F08081918111969C938E93DF
:10900000CF010895CF93DF93FC01A081B181109728
:10901000D9F0C0E0D0E016C0A617B70771F48D9163
:109020009C911197209719F49183808302C09983B2
:10903000888311961C921E9207C0ED019881898148
:10904000A92FB82F109741F7DF91CF9108950F9373
:109050001F93CF93DF938C01EB010E940248F8012C
:109060008081918199838883D183C083DF91CF915F
:109070001F910F910895EF92FF920F931F93CF933B
:10908000DF93EC017B010E940248F70111821082FC
:10909000CE010E94BF47FC01009719F4E882F982D3
:1090A00002C0F182E082DF91CF911F910F91FF907A
:1090B000EF900895DC01ED91FC91119720E030E0F4
:1090C00005C02F5F3F4F0190F081E02D3097C9F729
:1090D000C9010895FB01309721F4BA010E94274885
:1090E0000895DA018081918111969C938E9351832A
:1090F00040830895009721F0FC012081318102C056
:1091000020E030E0C901089580911A1090911B1061
:10911000009729F410921D1010921C1008950E94BF
:109120004057E0911A10F0911B1022813381408149
:109130005181240F351F281B390B0CC042815381EC
:1091400060817181460F571F481B590B4217530707
:1091500008F49A010480F581E02D309779F7280F03
:10916000391F30931D1020931C1008958DEC95E04D
:109170000E9412470895CF92DF92EF92FF920F93D1
:109180001F93CF93DF937C01FC0180819181009735
:1091900029F08A35910509F06EC00BC010921B10A2
:1091A00010921A108AE590E0F7019183808381E0A4
:1091B00066C0673849F5CA01E0911A10F0911B109A
:1091C00003C00480F581E02D309741F3268137817B
:1091D00028173907B1F3E0931A10F0931B100FC052
:1091E00016962D913C9117972817390739F4149644
:1091F0002D913C91159735832483DF01FD01A481D6
:10920000B581109769F7CECF623861F6C0911A1018
:10921000D0911B1000E010E02BC0CE010E9493679C
:109220000097F1F08E819F8168E8AE010E94BD46F3
:109230000097A1F41F821E828C819D81011511056A
:1092400021F0F8019583848304C090931B108093D0
:109250001A101D821C820E948448D8CF0E94B648F2
:109260008E019C818D81C92EE6016E01D82EE6010A
:10927000209799F697CFF7011182108283E0DF9152
:10928000CF911F910F91FF90EF90DF90CF900895B5
:10929000CF93DF93EC010E94B6488E819F810097A7
:1092A00069F0E0911A10F0911B1006C0EC17FD0751
:1092B000A9F00480F581E02D3097C1F780916C0F03
:1092C00090916D0F9F838E8380911A1090911B1047
:1092D0009D838C83D0931B10C0931A100E948448E6
:1092E000DF91CF910895CF93DF93EC010E947367D4
:1092F000CE010E944849DF91CF910895CF93DF932B
:10930000EC010E947F67CE010E944849DF91CF9116
:109310000895CF93DF93EC010E948967CE010E94EC
:109320004849DF91CF910895FC0180819181860F9A
:10933000971F918380830E948448089521E030E044
:10934000FC0186819781009711F020E030E0C9018F
:109350000895FC012281338180819181280F391F7A
:10936000C9010895FC0180819181089521E030E0D8
:1093700080911A1090911B10009711F420E030E0BA
:10938000C901089580911A1090911B10009729F03F
:1093900020911C1030911D1002C020E030E0C90166
:1093A0000895CF93DF93EC01E0911A10F0911B1018
:1093B0008E179F0741F48C819D8190931B108093A1
:1093C0001A1014C0FC01309731F0848195818C17FC
:1093D0009D07C1F707C01D821C821F821E82DF917C
:1093E000CF9108958C819D81958384830E948448C8
:1093F000F2CFCF92DF92EF92FF920F931F93CF9312
:10940000DF938C017A01FC0180819181009729F022
:109410008B34910509F051C01EC08FE190E10E948C
:10942000B447C82EE6017E01F92EE70109C06C8120
:109430007D81CE0102960E9473490990D881C02D8A
:109440002097A9F781E080931E108BE490E0F8014B
:109450009183808337C06838A9F58FE190E10E943D
:10946000B447C82EE6016E01D92EE60123C0CE0115
:109470000296E816F906D9F48FE190E1BE010E9448
:109480000248E0906C0FF0906D0F8A859B85909359
:109490006D0F80936C0FEC85FD85309719F08E85EC
:1094A0009F850995F0926D0FE0926C0FCECF0990D9
:1094B000D881C02D2097D9F6C8CFF801118210822B
:1094C00083E001C081E0DF91CF911F910F91FF9068
:1094D000EF90DF90CF90089510921E108FE190E1F1
:1094E0000E94B04786EE95E060E070E00E94EF4693
:1094F00008950F931F93CF93DF93EC0100916C0FAE
:1095000010916D0F1B870A875D874C873F872E87D9
:1095100080911E10882379F086EE95E090936D0F70
:1095200080936C0FCE0102960E94734910936D0FC9
:1095300000936C0F02C07D836C838FE190E1BE01CC
:109540000E9402488FE190E1BE010E943B48DF91FA
:10955000CF911F910F9108950F931F93CF93DF9396
:10956000EC0180911E10882391F000916C0F1091F6
:109570006D0F86EE95E090936D0F80936C0FCE018A
:1095800002960E947E4910936D0F00936C0F8FE13D
:1095900090E1BE010E9402488FE190E1BE010E946D
:1095A0003B48DF91CF911F910F9108950F931F9327
:1095B000CF93DF93EC0180911E10882391F00091EE
:1095C0006C0F10916D0F86EE95E090936D0F809368
:1095D0006C0FCE0102960E94894910936D0F009383
:1095E0006C0F8FE190E1BE010E9402488FE190E193
:1095F000BE010E943B48DF91CF911F910F910895CA
:10960000CF93DF93EC0180911E10882329F0CE01C7
:1096100002960E94D14904C01F821E8219861886B4
:109620008FE190E1BE010E940248DF91CF91089541
:10963000CF93DF93EC0180911E10882331F0CE018F
:1096400002960E949E499C0114C08FE190E10E9405
:10965000B447E82FF92F06C0EC17FD0741F0019041
:10966000F081E02D3097C1F721E030E002C020E02A
:1096700030E0C901DF91CF9108950F931F930091BE
:10968000CD251091CE250E946D572DB73EB722559E
:1096900030400FB6F8943EBF0FBE2DBFEDB7FEB7FA
:1096A00031962AE23FE0ADB7BEB712963C932E93B7
:1096B00011970283138214831582668377838087D0
:1096C00091878091C0279091C127A091C227B09126
:1096D000C32782879387A487B5878091C4279091F9
:1096E000C527A091C627B091C72786879787A08BEB
:1096F000B18B8091C8279091C927A091CA27B091BA
:10970000CB27828B938BA48BB58B8091CC279091A8
:10971000CD27A091CE27B091CF27868B978BA08F96
:10972000B18F8091D0279091D127A091D227B0916D
:10973000D327828F938FA48FB58F8091D427909158
:10974000D527A091D627B091D727868F978FA0A332
:10975000B1A38091D8279091D927A091DA27B09111
:10976000DB2782A393A3A4A3B5A38091DC279091C8
:10977000DD27A091DE27B091DF2786A397A3A0A7BE
:10978000B1A78091E0279091E127A091E227B091C5
:10979000E32782A793A7A4A7B5A78091E427909178
:1097A000E527A091E627B091E72786A797A7A0AB6A
:1097B000B1AB8091E8279091E927A091EA27B09179
:1097C000EB2782AB93ABA4ABB5AB8091EC27909128
:1097D000ED27A091EE27B091EF2786AB97ABA0AF16
:1097E000B1AF8091F0279091F127A091F227B0912D
:1097F000F32782AF93AFA4AFB5AFEDB7FEB7FF9637
:109800008091F4279091F527A091F627B091F72742
:1098100080839183A283B383EDB7FEB7ED5BFF4FE7
:109820008091F8279091F927A091FA27B091FB2712
:1098300080839183A283B383EDB7FEB7E95BFF4FCB
:109840008091FC279091FD27A091FE27B091FF27E2
:1098500080839183A283B383EDB7FEB7E55BFF4FAF
:109860008091002890910128A0910228B0910328AE
:1098700080839183A283B383EDB7FEB7E15BFF4F93
:109880008091042890910528A0910628B09107287E
:1098900080839183A283B3830E9421860091CD258A
:1098A0001091CE252DB73EB72E5A3F4F0FB6F894E4
:1098B0003EBF0FBE2DBF0E946D57ADB7BEB7D2974A
:1098C0000FB6F894BEBF0FBEADBFEDB7FEB7319671
:1098D0002BEB3EE012963C932E931197028313825A
:1098E0001483158266837783808791878091082807
:1098F00090910928A0910A28B0910B28828793871C
:10990000A487B58780910C2890910D28A0910E28EE
:10991000B0910F2886879787A08BB18B80911028F4
:1099200090911128A0911228B0911328828B938BCB
:10993000A48BB58B8091142890911528A09116289E
:10994000B0911728868B978BA08FB18F80911828A4
:1099500090911928A0911A28B0911B28828F938F7B
:10996000A48FB58F80911C2890911D28A0911E284E
:10997000B0911F28868F978FA0A3B1A38091202834
:1099800090912128A0912228B091232882A393A30B
:10999000A4A3B5A38091242890912528A0912628DE
:1099A000B091272886A397A3A0A7B1A780913028BC
:1099B00090913128A0913228B091332882A793A7A3
:1099C000A4A7B5A78091342890913528A091362876
:1099D000B091372886A797A7A0ABB1AB0E9421868C
:1099E0002DB73EB72E5C3F4F0FB6F8943EBF0FBE6B
:1099F0002DBF1F910F91089580E38093211008954A
:109A0000EF92FF92CF93DF932091211030E0C0E3DB
:109A1000D0E0C21BD30B2A5D3F4EB901AE010E94BC
:109A20008185CE01DF91CF91FF90EF900895AF92A5
:109A3000BF92CF92DF92EF92FF920F931F93CF933B
:109A4000DF937C01C0902210D09023102091211030
:109A500030E08601005D1F4F021B130B013811051A
:109A6000E0F4C0E3D0E0C21BD30B2A5D3F4EB90146
:109A7000AE010E948185CE0DDF1D20912410309112
:109A800025108091D8109091D910280F391FCE0140
:109A9000B901A6010E94818502C000E010E0C80162
:109AA000DF91CF911F910F91FF90EF90DF90CF90BA
:109AB000BF90AF90089590912110980F909321102E
:109AC000089540912210509123109C014817590786
:109AD00098F08091D8109091D910820F931F909395
:109AE000D9108093D810421B530B509323104093EE
:109AF000221021E030E002C020E030E0C9010895EA
:109B0000909323108093221008952091D8103091C3
:109B1000D9102A5A3F4EC90108952091211030E0F2
:109B20002A5D3F4EC901089521E030E08091241064
:109B30009091251040E18635940711F420E030E043
:109B4000C90108950E94944D009771F026E530E117
:109B50006091241070912510409122105091231093
:109B6000C9010E9481850895A091D810B091D910A3
:109B70001097B9F02091221030912310205D3F4FB3
:109B8000AA5ABF4EE6E5F0E180E390E003C04D91B4
:109B90004193019682179307D4F31092D910109233
:109BA000D8100895809124109091251008958091E7
:109BB00022109091231008959091211080E3891B29
:109BC000089580E390912110891B209122103091FB
:109BD0002310280F311DC90108951F93CF93DF93E0
:109BE000EC0110912110812F90E08C179D076CF0F3
:109BF0000E94E14D8C0F9D1F8138910530F41C1B94
:109C00001093211021E030E002C020E030E0C901D3
:109C1000DF91CF911F910895CF93DF93E7EDF5E2A8
:109C20001192119286E2E730F807D1F7C0E0D0E058
:109C3000CE01880F991F81539A4D65EB75E00E9404
:109C400081442196C430D10599F7DF91CF910895D1
:109C50001092D9101092D810109223101092221046
:109C600080E38093211086E590E190932510809306
:109C700024100E940C4E08950F931F93CF93DF93EF
:109C8000EC018B010E94284ED0932510C093241024
:109C90001093231000932210DF91CF911F910F9109
:109CA0000895CF92DF92EF92FF920F931F93DF936D
:109CB000CF9300D0CDB7DEB78C0169837A830E9441
:109CC000284E69817A81C62ED72E21E8C216D1048A
:109CD00018F030E8C32ED12C8091241090912510DB
:109CE000B801A6010E948185D0922310C092221053
:109CF000C6010F900F90CF91DF911F910F91FF90B0
:109D0000EF90DF90CF900895282F392FD901E7EDFC
:109D1000F5E280E301900D928150E1F7862F972FB5
:109D2000DC01EFECF5E288E001900D928150E1F763
:109D30000895E7EDF5E2282F392FD90180E30D9042
:109D400001928150E1F7AFECB5E2862F972FFC012D
:109D500088E001900D928150E1F70895E82FF0E03E
:109D6000EE0FFF1FE952FA4D7183608381E090E0AE
:109D70000895E82FF0E0EE0FFF1FE952FA4D8081C1
:109D80009181089590E0880F991F81569A4D0E9405
:109D9000814481E090E00895282F30E0220F331FA6
:109DA00021563A4DC90108958115910511F0019789
:109DB000F1F70895E0910A26F0910B2690818091A9
:109DC000092689230895E0910726F09108268081CD
:109DD00090910926892B8083E0910C26F0910D2625
:109DE000808190910926892B80830895E091072630
:109DF000F09108269081809109268095892380839F
:109E0000E0910C26F0910D26908180910926809595
:109E1000892380830895FF920F931F93E091072673
:109E2000F09108269081809109268095892380836E
:109E3000E0910C26F0910D26808190910926892BC6
:109E400080838FEB93E00E94D44EFFB6F894E091AC
:109E50000C26F0910D26908180910926809589230A
:109E6000808383E890E00E94D44EE0910A26F0912E
:109E70000B26008110910926FFBE78948BE393E0B6
:109E80000E94D44EE0910A26F0910B268081909199
:109E90000926892319F0802F812301C081E01F91B9
:109EA0000F91FF90089550930D2640930C267093C8
:109EB00008266093072690930B2680930A2681E05C
:109EC00090E002C0880F991F2A95E2F78093092637
:109ED0000E940B4F08950F931F93182F0FB7F894FC
:109EE000E0910C26F0910D26808190910926892B16
:109EF000808383E090E00E94D44E112351F0E091E2
:109F00000C26F0910D269081809109268095892359
:109F1000808387E190E00E94D44EE0910A26F09180
:109F20000B26808190910926892309F410E089E5A8
:109F300090E00E94D44EE0910C26F0910D26908185
:109F4000809109268095892380830FBF8BE390E061
:109F50000E94D44E812F1F910F9108950F931F934C
:109F6000182F08E0812F81700E946B4F1695811188
:109F700010680150B9F7812F1F910F9108958FEF4D
:109F80000E94AE4F0895DF92EF92FF920F931F93BE
:109F9000CF93DF93182FEB010E940B4F882389F595
:109FA00080EF0E94AE4FEE2400E498EFD92ED00E41
:109FB00081E00E946B4FF82E81E00E946B4F882356
:109FC00019F0FF2069F020C0FF2051F4011728F09C
:109FD000888180FF05C0101719F0E02EFF24F3944C
:109FE0008F2D0E946B4F888186958883FF2011F00A
:109FF0008068888301500D15D9F6002339F0219629
:10A00000D4CFEE24EA9402C08EEFE82E8E2DDF919D
:10A01000CF911F910F91FF90EF90DF9008950F93D4
:10A020001F93CF93DF93182FEB010E940B4F2097C4
:10A0300051F085E50E94AE4F08E089910E94AE4F35
:10A040000150D9F703C08CEC0E94AE4F812F0E94C3
:10A05000AE4FDF91CF911F910F9108950F931F93F2
:10A06000CF93DF93FB01DA01E801408150E0718179
:10A0700060E0462B572B803171F4BA016E7F13E0FC
:10A08000660F771F1A95E1F796814CE050E0491B67
:10A090005109460F571F57FF06C091E09C935095FA
:10A0A00041955F4F01C01C92883289F4848190E011
:10A0B000BC01607670706036710549F086FF02C0A1
:10A0C0004E7F05C085FF02C04C7F01C0487FCA019A
:10A0D00054E0969587955A95E1F7F90180834F7082
:10A0E000488380E0DF91CF911F910F9108950F93E6
:10A0F0001F93CF93DF938C01EB01F8018081BE01A8
:10A100000E94C34FF801808381508D3F28F48881DD
:10A11000883211F0803189F7DF91CF911F910F9133
:10A1200008951F93CF93DF93EC010E940B4F84EBB4
:10A13000BE010E940F5081E00E946B4F182F0E94B9
:10A140000B4F81E0112309F480E0DF91CF911F9143
:10A1500008951F93CF93DF93182FEB010E940B4FAD
:10A160000E94DA4E882349F084E4BE010E940F5019
:10A17000113029F00E94E34E02C082E001C080E06D
:10A18000DF91CF911F9108956F927F928F929F924E
:10A19000AF92BF92CF92DF92EF92FF920F931F93F5
:10A1A000DF93CF93CDB7DEB729970FB6F894DEBF14
:10A1B0000FBECDBF7C014B013A0159010E940B4FEC
:10A1C0008EEBB7010E940F508E010F5F1F4F8AE088
:10A1D000C82ED12CCC0EDD1E0E94BF4FF8018193FA
:10A1E0008F01EC15FD05C1F78E010F5F1F4FC801F0
:10A1F00069E070E00E94446C882351F4F70180818B
:10A20000B801A401930185010E942E5080E001C095
:10A2100083E029960FB6F894DEBF0FBECDBFCF9175
:10A22000DF911F910F91FF90EF90DF90CF90BF9043
:10A23000AF909F908F907F906F9008957F928F92B4
:10A240009F92AF92BF92CF92DF92EF92FF920F93C5
:10A250001F93DF93CF93CDB7DEB729970FB6F8944E
:10A26000DEBF0FBECDBF782E5B014A0179018EEBB8
:10A2700060E070E00E940F508E010F5F1F4F9AE068
:10A28000C92ED12CCC0EDD1E0E94BF4FF801819348
:10A290008F01EC15FD05C1F78E010F5F1F4FC8013F
:10A2A00069E070E00E94446C882349F4872DB8016E
:10A2B000A501940187010E942E5080E001C083E037
:10A2C00029960FB6F894DEBF0FBECDBFCF91DF91B8
:10A2D0001F910F91FF90EF90DF90CF90BF90AF90C4
:10A2E0009F908F907F9008950F931F93DF93CF934C
:10A2F000CDB7DEB728970FB6F894DEBF0FBECDBF3F
:10A30000182F062FDE011196E8EFF5E088E00190A6
:10A310000D928150E1F7242F332727FD309541E737
:10A3200052E0249FC001259F900D349F900D112471
:10A3300064E670E00E944F81AB0164E6069FB001C5
:10A340001124460F571FFE013196CE0109966191E7
:10A3500070E02617370719F44F5F5F4F03C0E81707
:10A36000F907A9F7112319F0509541955F4FCA01DC
:10A3700028960FB6F894DEBF0FBECDBFCF91DF9108
:10A380001F910F9108950F931F93DF93CF93CDB734
:10A39000DEB72B970FB6F894DEBF0FBECDBF182FD8
:10A3A000092F885F612F792F0E94A950882309F017
:10A3B00049C066E471E48FE090E00E943052812F42
:10A3C000902FBE016F5F7F4FAE014E5F5F4F9E01CA
:10A3D0002D5F3F4F0E94C4508823A1F5DE011496E3
:10A3E000E0EFF5E088E001900D928150E1F74B81BC
:10A3F000642F70E021E732E0629FC001639F900DFF
:10A40000729F900D112464E670E00E944F819A8142
:10A4100084E6989FC0011124680F791FFE013496CD
:10A42000CE010C962191421719F46F5F7F4F03C044
:10A43000E817F907B9F78981882331F0709561959C
:10A440007F4F02C064E371E2CB012B960FB6F89404
:10A45000DEBF0FBECDBFCF91DF911F910F91089549
:10A46000DC01CB0181159105A105B10529F08150D1
:10A470009040A040B040D9F708951092B90080E212
:10A480008093B800089594EA9093BC0020EA36E8DF
:10A4900041E050E005C02150304040405040F1F0D4
:10A4A0009091BC0097FFF7CF1DC09031B9F4809315
:10A4B000BB0084E88093BC0080EA96E8A1E0B0E0AD
:10A4C00004C00197A109B10959F02091BC0027FFF0
:10A4D000F8CF0EC081E0903421F40FC081E00895E0
:10A4E00081E008959091B900987F9830F1F6DFCF20
:10A4F0009091B900987F983169F780E0089544EA17
:10A5000034E824E94093BC009091BC0097FFFCCF55
:10A510009091B900987F983011F0903199F780931D
:10A52000BB003093BC009091BC0097FFFCCF909192
:10A53000B900987F903211F0983539F42093BC001F
:10A540009091BC0094FDFCCFDDCF08950E94435252
:10A55000089584E98093BC008091BC0084FDFCCF09
:10A5600008958093BB0084E88093BC008091BC0078
:10A5700087FFFCCF9091B900987F81E0983209F471
:10A5800080E0089584EC8093BC008091BC0087FF3C
:10A59000FCCF8091BB00089584E88093BC0080913B
:10A5A000BC0087FFFCCF8091BB000895E82FF92FF6
:10A5B00080E1919190933F018150D9F780913C01C6
:10A5C0008F7D80933C0180913C01877F80933C018B
:10A5D000862F972FFC0180E1919190933E0181504D
:10A5E000D9F780913C01806880933C0180913D01C6
:10A5F00080FFFCCF4051504080913C0180628093AD
:10A600003C0180913C01877F80933C0114C0862FE0
:10A61000972FFC0180E1919190933E018150D9F7F1
:10A6200080913C01806880933C0180913D0180FFD6
:10A63000FCCF40515040141615064CF3822F932F37
:10A64000FC0180E190913E0191938150D9F781E026
:10A6500090E008950F931F93CF93DF938C018CE7C5
:10A660000E947F528CE70E94B152C0E0D0E0F80116
:10A6700081918F010E94B1522196C031D105B9F765
:10A680000E94A952DF91CF911F910F9108958130BF
:10A6900039F48CE790E060E070E040E050E006C004
:10A6A0008CE790E060E070E040EC50E00E94151311
:10A6B0000895813039F48CE790E060E070E04EE07E
:10A6C00050E006C08CE790E060E070E048E050E0C9
:10A6D0000E94151308958CE790E060E070E041E07F
:10A6E00050E00E9415136AE67AE080E090E00E9454
:10A6F000305208958CE790E060E070E048E350E06D
:10A700000E9415138CE790E060E070E049E350E0B0
:10A710000E9415138CE790E060E070E044E150E0A7
:10A720000E9415138CE790E060E070E048E750E08D
:10A730000E9415138CE790E060E070E04EE550E079
:10A740000E9415138CE790E060E070E04DE650E069
:10A750000E9415136CE17AE186E090E00E9430528D
:10A760008CE790E060E070E04CE050E00E94151350
:10A770008CE790E060E070E041E050E00E9415134B
:10A780008CE790E060E070E046E050E00E94151336
:10A790006AE67AE080E090E00E9430520895DF930C
:10A7A000CF93CDB7DEB7A2970FB6F894DEBF0FBE3A
:10A7B000CDBFDE011196E0E0F6E081E101900D925F
:10A7C0008150E1F7DE015296E1E1F6E081E101908E
:10A7D0000D928150E1F70E947A53CE0101960E94BA
:10A7E0002A5382E00E9447536AE67AE080E090E0D4
:10A7F0000E943052CE0142960E942A5360E17EEAC6
:10A8000088E290E00E94305280E00E94595360E15B
:10A810007EEA88E290E00E94305281E00E94595323
:10A82000A2960FB6F894DEBF0FBECDBFCF91DF91D9
:10A830000895E6E4F1E08081208190813081829565
:10A8400086958695837022952F70822B832B929507
:10A850009F70892B0895DF92EF92FF920F931F93C1
:10A86000DF93CF9300D0CDB7DEB780E06CE046E059
:10A870000E94015889E18093C4001092C50082E0D3
:10A880008093C00080E00E94AB580E94305784B78C
:10A8900084B784B784B784B7EEE8FEE222E432E4FA
:10A8A000318320833A968DB79EB70A97E817F90748
:10A8B000B8F300D000D087E790E1ADB7BEB71296ED
:10A8C0009C938E93119782E296E014969C938E93BC
:10A8D00013970E9421860F900F900F900F900E9467
:10A8E0005D680E943B468DEC95E060E070E00E9460
:10A8F000EF460E946C4AE0916D06F0916E06099554
:10A900000E94195490E00E949B68CE0101960E941B
:10A910005E56882359F000D087E590E1EDB7FEB789
:10A92000928381830E9421860F900F908E010F5F8A
:10A930001F4FC8010E949C440E9468567C010E94DF
:10A940006D56BC01C701A8010E94B85B0E94C655A4
:10A950000E949D5B0E9472560E94255D00D08AE491
:10A9600090E1ADB7BEB712969C938E9311970E945B
:10A97000218600D0EDB7FEB7319606E410E1ADB701
:10A98000BEB712961C930E9311978A81828313820D
:10A990000E942186EDB7FEB73196ADB7BEB71296CD
:10A9A0001C930E9311978981828313820E942186C2
:10A9B0000F900F9084E490E1EDB7FEB7928381830E
:10A9C0000E9421860F900F900E94A168E091F006EE
:10A9D000F091F1060995E091D706F091D806099516
:10A9E000E0919906F0919A060995E090D506F090CD
:10A9F000D6060091EE061091EF060E949A5BD82EC3
:10AA00000E942D5D2DB73EB72A5030400FB6F89406
:10AA10003EBF0FBE2DBFEDB7FEB7319629E230E144
:10AA2000ADB7BEB712963C932E931197F382E28294
:10AA300015830483D6821782808711860E9421861F
:10AA4000E091FA06F091FB062DB73EB7265F3F4F27
:10AA50000FB6F8943EBF0FBE2DBF3097D1F00995C9
:10AA6000BC0100D000D086E190E1ADB7BEB7129630
:10AA70009C938E93119780E890E00E943B81EDB704
:10AA8000FEB7748363830E9421860F900F900F900E
:10AA90000F9000D084E190E1ADB7BEB712969C93C1
:10AAA0008E9311970E9421860F900F9089E197E075
:10AAB00060E070E00E94EF468BE995E00E944767F6
:10AAC00000D08CE090E1EDB7FEB7928381830E94C5
:10AAD00021860F900F900F900F90CF91DF911F91D3
:10AAE0000F91FF90EF90DF900895EF92FF920F93F8
:10AAF0001F9380E880936100109261000E942B54A4
:10AB00000E944B460E94CC5880910E2690910F26B1
:10AB1000009729F0019790930F2680930E26E090DE
:10AB20001026F090112600911226109113260E94F3
:10AB30006D57E616F7060807190711F30E946D57BF
:10AB400060931026709311268093122690931326FB
:10AB5000D7CF00D000D000D0EDB7FEB7319626E0B9
:10AB600030E1ADB7BEB712963C932E931197938305
:10AB70008283758364830E9421868DB79EB7069673
:10AB80000FB6F8949EBF0FBE8DBF08950F931F930D
:10AB9000DF93CF93CDB7DEB7A2970FB6F894DEBFA1
:10ABA0000FBECDBF8EE490E00E94648789839A83B4
:10ABB000982F9B50903108F08A839A81909589173D
:10ABC00009F470C000D082EB90E1ADB7BEB7129629
:10ABD0009C938E9311970E9421868E010D5F1F4FCB
:10ABE0000F900F90D80180E090E0FC01EE56FF4EF0
:10ABF000E491ED93019688309105B9F7F894CE0170
:10AC000003966CE270E048E050E00E946A87D80149
:10AC100080E090E0FC01E656FF4EE491ED93019652
:10AC20008E309105B9F7CE01039664E370E04EE0F3
:10AC300050E00E946A8780E090E0FC01E855FF4EFA
:10AC4000E491D801ED938D0101968A309105A9F721
:10AC5000CE01039662E470E04AE050E00E946A8709
:10AC600080E590E06DEC7BEA0E94828782E590E0CF
:10AC700060E070E00E94828784E590E060E00E94DE
:10AC800074878CE490E060E070E00E9482878AE143
:10AC9000898385EE8A8369817A818EE490E00E94BF
:10ACA000828778948981A2960FB6F894DEBF0FBE92
:10ACB000CDBFCF91DF911F910F910895F8946CE271
:10ACC00070E042E050E00E944C87789480E0089564
:10ACD00080E590E00E946487089582E590E00E94FC
:10ACE0006487089584E590E00E945C870895209130
:10ACF0001C2630911D2640911E2650911F2690E063
:10AD0000A0E0B0E0280F391F4A1F5B1F20931C26CC
:10AD100030931D2640931E2650931F2620911826FF
:10AD20003091192640911A2650911B26280F391F61
:10AD30004A1F5B1F209318263093192640931A262A
:10AD400050931B262091BC272223A1F0209114268A
:10AD5000309115264091162650911726280F391F3D
:10AD60004A1F5B1F20931426309315264093162606
:10AD70005093172608951F920F920FB60F920BB69D
:10AD80000F9211242F933F934F935F936F937F9371
:10AD90008F939F93AF93BF93EF93FF938091DA10BC
:10ADA0009091DB1001969093DB108093DA108091E4
:10ADB000DC108F5F8093DC108091DC108038A9F468
:10ADC0001092DC1080911C2690911D26A0911E26C9
:10ADD000B0911F260196A11DB11D80931C26909352
:10ADE0001D26A0931E26B0931F268091BC27882382
:10ADF000F1F08091DD108F5F8093DD108091DD1088
:10AE00008038A9F41092DD108091142690911526B7
:10AE1000A0911626B09117260196A11DB11D809311
:10AE2000142690931526A0931626B09317260E94F9
:10AE3000B649009711F00E94B648FF91EF91BF917B
:10AE4000AF919F918F917F916F915F914F913F91C2
:10AE50002F910F900BBE0F900FBE0F901F90189563
:10AE6000F8941092B60016BC83EF87BD82E084BDD3
:10AE700094E095BD95B395BB80936E00789408954A
:10AE80002091DA103091DB108091DA109091DB1074
:10AE900028173907A9F7C901089507C022E330E050
:10AEA000000021503040E1F701970097B9F708956D
:10AEB0000F931F93CF93DF938C010E944057EC01B7
:10AEC0000E9440578C1B9D0B80179107C8F3DF91A0
:10AED000CF911F910F910895089520911C263091D4
:10AEE0001D2640911E2650911F2680911C26909170
:10AEF0001D26A0911E26B0911F26281739074A0744
:10AF00005B0759F7B901CA0108951F920F920FB656
:10AF10000F921124109246060F900FBE0F901F90B3
:10AF200018951F920F920FB60F920BB60F92112425
:10AF30002F933F934F935F936F937F938F939F9341
:10AF4000AF93BF93EF93FF93E0913C06F0913D06E2
:10AF50008081E0914706F0914806309709F0099505
:10AF6000FF91EF91BF91AF919F918F917F916F91E1
:10AF70005F914F913F912F910F900BBE0F900FBE9D
:10AF80000F901F9018951F920F920FB60F921124D9
:10AF9000109253060F900FBE0F901F9018951F929E
:10AFA0000F920FB60F920BB60F9211242F933F936F
:10AFB0004F935F936F937F938F939F93AF93BF93C1
:10AFC000EF93FF93E0914906F0914A068081E0916A
:10AFD0005406F0915506309709F00995FF91EF91CD
:10AFE000BF91AF919F918F917F916F915F914F91A1
:10AFF0003F912F910F900BBE0F900FBE0F901F909F
:10B00000189590E02DE030E0829FF001839FF00DD5
:10B01000929FF00D1124E45CF94FA281B3811C9240
:10B02000A481B5816C93A681B78188ED8C93A085AE
:10B03000B1854C93128614861386089590E02DE016
:10B0400030E0829FF001839FF00D929FF00D11245C
:10B05000E45CF94F81E08287A081B1816C933A96DC
:10B0600080818823E9F708951F93182F8A3031F4DF
:10B070008091DE106DE00E941E5802C08D3029F0D4
:10B080008091DE10612F0E941E5880E090E01F9199
:10B090000895EF92FF921F93CF93DF93182FE62E20
:10B0A000E7017E01F72EE7010CC08A3021F4812FE1
:10B0B0006DE00E941E5869916D3019F0812F0E9439
:10B0C0001E588881882389F7DF91CF911F91FF90C7
:10B0D000EF9008950F931F93DF93CF93CDB7DEB713
:10B0E000FE013A960FED10E1C80160E470E048857A
:10B0F00059859F010E94B6868F81B8010E944958E8
:10B10000CF91DF911F910F9108951F93CF93DF93FC
:10B11000182FEB0104C0812F0E941E582196FE01BA
:10B1200064916623C1F7DF91CF911F91089590E05C
:10B130002DE030E0829FF001839FF00D929FF00D93
:10B140001124E45CF94F748763870895682F80E0C9
:10B150000E941E5808958093DE108EE296E0909330
:10B16000892E8093882E089584B7877F84BF88E1D5
:10B170000FB6F89480936000109260000FBE08959F
:10B180002FE088E190E00FB6F894A89580936000D6
:10B190000FBE209360000895A895089588E10FB62A
:10B1A000F89480936000109260000FBE0895F894A8
:10B1B00028E088E190E00FB6F894A89580936000AD
:10B1C0000FBE20936000FFCF80912F2690E0FC01FE
:10B1D000EE0FFF1F9695982F882797958795E80F74
:10B1E000F91FE05DF94D1082089580912726809126
:10B1F000272690E008958091390181FD0CC081E4FB
:10B2000091E06FE140E00E94CE5E813039F021E0B4
:10B2100030E0813129F020E030E002C021E030E070
:10B22000C90108958091390181FD12C081E491E046
:10B230006FE140E00E94CE5E982F8151823050F045
:10B240009F3141F0913041F081E0923031F402C001
:10B2500081E0089580E0089580E008950E941259E9
:10B260008823E1F3089581E491E06FE140E00E94DA
:10B27000CE5E0895E9E3F1E0808180818D7F808357
:10B280008DE090E00197F1F782E491E06FE140E01A
:10B2900023E00E94D85E83E090E00197F1F70895E3
:10B2A0000E942E591092BC270E943A598091390170
:10B2B00082608093390180913F288823E9F1809151
:10B2C0009400909195002091502830915128821738
:10B2D0009307A0F480911C2890911D28A0911E280E
:10B2E000B0911F288C57914EAF4FBF4F80931C28B1
:10B2F00090931D28A0931E28B0931F28809194003E
:10B3000090919500821B930BA0E0B0E020911C2847
:10B3100030911D2840911E2850911F28820F931FA5
:10B32000A41FB51F80931C2890931D28A0931E284E
:10B33000B0931F2810923F28809141288823E9F17B
:10B340008091940090919500209154283091552837
:10B3500082179307A0F48091242890912528A0912A
:10B360002628B09127288C57914EAF4FBF4F80931E
:10B37000242890932528A0932628B09327288091ED
:10B38000940090919500821B930BA0E0B0E0209177
:10B390002428309125284091262850912728820F73
:10B3A000931FA41FB51F8093242890932528A09352
:10B3B0002628B09327281092412808958091BC2711
:10B3C000882381F080911F11882321F40E94125953
:10B3D000882331F481E08093A21121E030E004C0A1
:10B3E0000E94505920E030E0C90108950F931F9347
:10B3F000182F883049F0863039F0893029F08631AD
:10B4000019F0893109F041C08091390181FD40C0B6
:10B410000E942E590E943359082F181709F43BC077
:10B42000183019F40E943A5929C0193141F4863173
:10B43000A9F482E491E06FE140E029E009C016310F
:10B4400069F4893159F482E491E06FE140E026E04B
:10B450000E94D85EE3E0F0E03197F1F782E491E0FA
:10B460006FE140E0212F0E94D85E083019F4E9E630
:10B47000F1E002C0E3E0F0E03197F1F70E943359C8
:10B48000811749F023E430E008C022E430E005C031
:10B4900024E430E002C020E430E0C9011F910F91A4
:10B4A00008958091940090919500909355288093F1
:10B4B000542821E0209341288091390181FF15C053
:10B4C0002093BB27809194009091950090935128F0
:10B4D0008093502820933F28809139018D7F80935D
:10B4E00039018091BB278823E1F786E10E94F65954
:10B4F00081E08093BC2708958091BC27882351F474
:10B5000080911F11882321F081E08093A11102C056
:10B510000E94515A81E090E008951F93DF93CF93EA
:10B520000F92CDB7DEB78FB7898380911F11882323
:10B5300031F5F8948091BC27882351F0809139012E
:10B5400081FD1BC00E9412598823B9F080E003C01E
:10B550000E947C5A81E0909147019E3010F010E0EB
:10B5600001C01FEF882311F00E94DE5916FF05C0AD
:10B5700089818FBF21E030E004C089818FBF20E046
:10B5800030E0C9010F90CF91DF911F910895809114
:10B59000A111882321F00E94515A1092A11180918B
:10B5A000A211882321F00E9450591092A2111092EA
:10B5B0001F110895EF92FF92CF93DF93B82FA92F19
:10B5C000F62FE72F81E080931F1120910028309102
:10B5D000012840910228509103282F5F3F4F4F4F81
:10B5E0005F4F209300283093012840930228509306
:10B5F0000328862F8E5F87FF0CC08091B92790911A
:10B60000BA2701969093BA278093B927CFEFDFEF3F
:10B610000BC020E231E1C9016B2F7A2F4F2F5E2F33
:10B620000E948185C0E0D0E00E94C75ACE01DF9120
:10B63000CF91FF90EF9008959091390191FD0AC04C
:10B64000282F803108F02FE085E491E06FE040E0A2
:10B650000E94D85E08958093A41108950E943359E2
:10B660008250813130F4E82FF0E0EF57F94F8081BC
:10B67000089581E0089508958FEF80934E018CE640
:10B6800091E060EF44E022E00E94D85E8CE290E01E
:10B690006EE041E025E00E94D85E80E880936F0173
:10B6A0008091460180936D0184E491E060E245E081
:10B6B00021E00E94D85E0895CF93DF93CDEFD3E0D1
:10B6C000CE010197F1F70E94C45E109230261092CD
:10B6D000B2261092342710922F2610922E26E9E3DC
:10B6E000F1E080818E7F808380818D7F80838DE0FB
:10B6F00090E00197F1F780818160808382E491E09E
:10B700006FE140E023E00E94D85E2197F1F780913D
:10B710005D0180915E010E943C5B83E696E060E003
:10B7200070E00E94EF460E94515A81E090E0DF9164
:10B73000CF9108958091A3110895DF93CF930F9235
:10B74000CDB7DEB789830E942E5929812093A3119A
:10B7500088E491E06FE140E00E94D85E0F90CF91C5
:10B76000DF9108950E949D5B86E00E94F65908953E
:10B770008093620190936301609360017093610113
:10B780004115510531F1FA01819180936B01DA0184
:10B7900011968C9180936A01DF01119681818093CB
:10B7A0006901FD01319611968C9180936801DF014A
:10B7B0001196818180936701FD01319611968C91DC
:10B7C00011978093660181818093650182818093C6
:10B7D0006401089583E696E00E94124781E0809319
:10B7E0002726809128269091292601969093292634
:10B7F0008093282681E090E00895EF92FF92CF9306
:10B80000DF9350912F26252F30E0F901EE0FFF1F17
:10B810003695322F222737952795E20FF31FE05DEB
:10B82000F94D4081442309F4CEC02091390121FD16
:10B83000CAC02091BC27222309F4C5C047FF16C007
:10B840000E94E4588091F0279091F127A091F2276F
:10B85000B091F3270196A11DB11D8093F02790931D
:10B86000F127A093F227B093F327ADC04330B0F493
:10B870000E94E4588091EC279091ED27A091EE274B
:10B88000B091EF270196A11DB11D8093EC279093F5
:10B89000ED27A093EE27B093EF2795C0C42FD0E0FB
:10B8A00022976C177D07B0F40E94E4588091E82736
:10B8B0009091E927A091EA27B091EB270196A11D6D
:10B8C000B11D8093E8279093E927A093EA27B093CE
:10B8D000EB2779C0652F70E09B01220F331F76950F
:10B8E000762F662777956795260F371F2F5C394D82
:10B8F000B90150E00E94818520912F26822F90E08F
:10B90000FC01EE0FFF1F9695982F88279795879536
:10B91000E80FF91FE055F94D808180932026822F92
:10B9200090E0FC01EE0FFF1F9695982F88279795C2
:10B930008795E80FF91FE05DF94D10822F5F209386
:10B940002F26233010F010922F2680912F2690E082
:10B95000FC01EE0FFF1F9695982F882797958795E6
:10B96000E80FF91FE05DF94D8081882311F00E94F6
:10B97000EA5B609147016093212680912626882307
:10B9800011F0681710F46093262684E070E00E949E
:10B99000AE4E6091202683E070E00E94AE4E809112
:10B9A000042890910528A0910628B09107280196B7
:10B9B000A11DB11D8093042890930528A09306280B
:10B9C000B093072802C0C0E0D0E0CE01DF91CF9154
:10B9D000FF90EF900895CF93DF93EC0188819981D8
:10B9E000009729F024E08B3F920739F505C08BEFD3
:10B9F00094E09983888325C0623819F51092272630
:10BA00000E94284E0E94854D60E870E00E94FD5B18
:10BA10001816190644F40E94804DE091F406F09146
:10BA2000F5060995E4CF809124269091252601966C
:10BA30009093252680932426DACF1982188283E0FA
:10BA400001C081E0DF91CF91089591E090931F11A3
:10BA50000E941C5B0E94C75A08958091390181FDA4
:10BA600007C085E491E06FE040E00E94CE5E08955B
:10BA700080E10895CF92DF92EF92FF920F931F9390
:10BA8000CF93DF93182F21E020931F110091BC2743
:10BA90008091390181FF16C08091940090919500AA
:10BAA000909351288093502820933F282093BB27C0
:10BAB000809139018D7F809339018091BB27882344
:10BAC000E1F700E00E942E598091BC27882309F4F9
:10BAD00041C0809141288823E9F120919400309160
:10BAE0009500809154289091552828173907A0F483
:10BAF00020912428309125284091262850912728EC
:10BB00002C57314E4F4F5F4F2093242830932528D8
:10BB10004093262850932728209194003091950037
:10BB2000281B390B40E050E0C0902428D0902528F5
:10BB3000E0902628F09027282C0D3D1D4E1D5F1DFE
:10BB40002093242830932528409326285093272893
:10BB50001092412889E10E94F65986E00E94B94E70
:10BB6000009751F00E942D5DC82F86E00E94B94ECB
:10BB700081500E941C5B02C0C0E0D0E08091940024
:10BB800090919500909353288093522881E0809360
:10BB90004028F89480913901826080933901809126
:10BBA00039018D7F80933901612F6E5F80E291E1D1
:10BBB0000E94095F78948091B6279091B7270196EB
:10BBC0009093B7278093B6270E942E5982E491E084
:10BBD00060EE45E00E94CE5E182F86E00E94B94ECE
:10BBE000009719F08C2F0E941C5B002319F00E9413
:10BBF000515A02C00E945059809140288823E9F18F
:10BC00008091940090919500409152285091532832
:10BC100084179507A0F48091202890912128A09165
:10BC20002228B09123288C57914EAF4FBF4F80935D
:10BC3000202890932128A0932228B0932328209194
:10BC4000940030919500241B350B40E050E080912A
:10BC5000202890912128A0912228B0912328280FF4
:10BC6000391F4A1F5B1F20932028309321284093BF
:10BC7000222850932328109240288091BC278823A3
:10BC800061F0809194009091950090935528809355
:10BC9000542881E08093412807C082E491E06FE15D
:10BCA00040E023E00E94D85E0E94C75A1130E1F0C4
:10BCB0001330A9F48091F8279091F927A091FA27E1
:10BCC000B091FB270196A11DB11D8093F827909399
:10BCD000F927A093FA27B093FB2712E00AC015308A
:10BCE00029F0173031F404C010E003C013E001C0A4
:10BCF00011E0812F90E0DF91CF911F910F91FF9084
:10BD0000EF90DF90CF900895CF93DF93EB010E94E7
:10BD1000DA5A9C01009731F4CE010E943A5D9C01F1
:10BD2000009749F08091B9279091BA270196909396
:10BD3000BA278093B927C901DF91CF9108950F9356
:10BD40001F938091BC27882321F40E947C5A11E024
:10BD500001C010E00E943359863111F0813119F48D
:10BD60000091470109C086E491E06FE140E00E9444
:10BD7000CE5E082F000F080F112311F00E94DE592C
:10BD8000802F1F910F9108951092A6111092A51166
:10BD9000EFE6F0E08081806280830895FC0180817D
:10BDA000862390E002C0959587954A95E2F708951D
:10BDB000F894FC019081862F8095892330E002C0A1
:10BDC000220F331F4A95E2F72623282B20837894ED
:10BDD0000895DC01119620917B01FC012083215004
:10BDE00030E0A9014F575E4FE0E8F1E061916D93BB
:10BDF000E417F507D9F7FC01E058FF4F2F573E4FE6
:10BE0000D9012C9120838F579F4F21E0FC01208383
:10BE10000895FC016093800101966350860F911D87
:10BE2000A1E8B1E021912D93E817F907D9F708951A
:10BE30001F920F920FB60F920BB60F9211242F93F1
:10BE40003F934F935F936F937F938F939F93AF93A2
:10BE5000BF93EF93FF938091470180932126209118
:10BE60002E2630E0C901880F991F3695322F2227E0
:10BE700037952795820F931F805D994D0E94E95E4B
:10BE800080912E268F5F80932E26833010F01092A3
:10BE90002E260E94EA5BFF91EF91BF91AF919F9197
:10BEA0008F917F916F915F914F913F912F910F9063
:10BEB0000BBE0F900FBE0F901F9018951F920F9200
:10BEC0000FB60F9211240F900FBE0F901F90189570
:10BED0001F920F920FB60F9211240F900FBE0F906A
:10BEE0001F9018951F920F920FB60F9211240F906A
:10BEF0000FBE0F901F9018951F920F920FB60F92C2
:10BF000011241092BB270F900FBE0F901F90189511
:10BF10001F920F920FB60F9211241092BB270F9011
:10BF20000FBE0F901F9018951F920F920FB60F9291
:10BF300011248F9381E0809327268F910F900FBE5D
:10BF40000F901F9018951F920F920FB60F92112409
:10BF50001092BB270F900FBE0F901F9018951F9245
:10BF60000F920FB60F9211248F939F938091A5117A
:10BF70009091A61101969093A6118093A5119F917F
:10BF80008F910F900FBE0F901F901895DF92EF9238
:10BF9000FF920F931F93DF93CF9300D00F92CDB7F3
:10BFA000DEB7F82E042F122F213031F0223031F07D
:10BFB000243031F0283031F080E005C081E003C04A
:10BFC00082E001C083E00C3059F00E3011F484603F
:10BFD00007C0003111F4886003C0023109F48C609D
:10BFE000613059F0623011F4806207C0633011F49F
:10BFF000806403C0643009F48066682F60688F2D08
:10C0000090E070E0AE014F5F5F4F23E030E00E94B0
:10C010002D1369E07AE180E090E00E94305281E0E7
:10C02000F82A8F2D0E9443520E94C25289830E9497
:10C03000C2528A83023119F40E94C2528B830E9439
:10C04000C25287FDF1CF0E94CC520E94A95269E0F2
:10C050007AE180E090E00E9430528F2D0E9443529E
:10C060000E94C25289830E94C2528A83023119F40B
:10C070000E94C2528B830E94C2522981023181F5F3
:10C08000622F70E080E090E03B814A8121FF12C086
:10C09000CB0177276627630F711D811D911D342FFA
:10C0A00020E040E050E0620F731F841F951F8C6FEB
:10C0B0009F6F0FC0CB0177276627630F711D811D0E
:10C0C000911D342F20E040E050E0620F731F841F69
:10C0D000951F0E94A17E20E83FEF4FEF57E41FC05D
:10C0E000722F60E08A81680F711D882777FD809527
:10C0F000982F0E94A17E0C3029F420E030EE4FEF03
:10C1000054E40DC00E3029F420E038EF4FEF55E431
:10C1100006C0003131F420E03EEF4FEF56E40E94BC
:10C12000377E2FE632E143E050E40E947D7FD62E39
:10C13000E72EF82E092F612F70E0882777FD809574
:10C14000982F0E94A17E9B01AC016D2D7E2D8F2D1D
:10C15000902F0E94377E0F900F900F90CF91DF911C
:10C160001F910F91FF90EF90DF9008950F931F9311
:10C17000CF93DF938091C4279091C527A091C627C4
:10C18000B091C7270196A11DB11D8093C42790933C
:10C19000C527A093C627B093C7270E946763EC0109
:10C1A00087EA91E10E94B4470BC0D8011296ED9145
:10C1B000FC911397309709F00995C8010E947A48BD
:10C1C000082F192F0115110581F7209719F0CE01BD
:10C1D0000E942445DF91CF911F910F9108950E94F5
:10C1E000A1680E94284E0E94716185ED96E09093AF
:10C1F000BF278093BE270E94646382E090E060E0E6
:10C2000074E040E05EE12FEF31E00E942563089585
:10C21000CF92DF92EF92FF920F931F93CF93DF9312
:10C220006C01EB018A0187EA91E10E94B4470CC0DE
:10C23000D7011496ED91FC911597309711F0CE012E
:10C240000995C7010E947A48E82EF92EE114F104FD
:10C2500079F7C601BE01A8010E942C45DF91CF915C
:10C260001F910F91FF90EF90DF90CF900895BC0148
:10C2700087EA91E10E943B480895BC0187EA91E179
:10C280000E9402480895CF93DF93EC018091C0276C
:10C290009091C127A091C227B091C3270196A11DFB
:10C2A000B11D8093C0279093C127A093C227B0935C
:10C2B000C327CE010E947E63009769F00E94A24DC1
:10C2C000E091D906F091DA0688E091E6BE01099581
:10C2D00021E030E002C020E030E0C901DF91CF91E1
:10C2E000089589EA91E10E94B04708950F93CF9392
:10C2F000DF93EC017B836A8318865F834E8389EA30
:10C3000091E1BE010E943B48E091AB11F091AC116C
:10C31000309749F04C815D818A819B81688520E05E
:10C3200030E001E00995DF91CF910F910895BC01B4
:10C3300089EA91E10E94024808950F93DC01189662
:10C340001C921897E091AB11F091AC11309759F015
:10C3500012968D919C91139760E040E050E020E0B0
:10C3600030E000E009950F9108950F93DC01AB01D7
:10C3700014962D913C91159781E018968C931897FF
:10C3800015967C936E931497E091AB11F091AC11DC
:10C39000309739F012968D919C91139761E000E0EF
:10C3A00009950F9108950F93DC01E091AB11F09185
:10C3B000AC11309769F014962D913C911597129617
:10C3C0008D919C91139718966C91A90101E00995A4
:10C3D0000F910895E091AD11F091AE11309709F0F1
:10C3E000099508959093AE118093AD11089590939F
:10C3F000AC118093AB11089589EA91E10E94B44792
:10C400000895EF92FF920F931F93CF93DF938C01C8
:10C41000EB017A0189EA91E10E94B44715C0DC0181
:10C4200012962D913C9113972C173D0759F41696AF
:10C43000ED91FC911797309761F0B801AE0197012B
:10C44000099507C00E947A48282F392FC901009703
:10C4500031F7DF91CF911F910F91FF90EF900895E9
:10C460000895AF92BF92CF92DF92EF92FF920F9317
:10C470001F93DF93CF9300D0CDB7DEB75B010E944F
:10C48000854DFC01008111811A8309830C3011054F
:10C4900018F4EE24FF242EC000D000D08DE996E0E1
:10C4A000EDB7FEB792838183148303830E940F86C6
:10C4B0000F900F900F900F9020C00E94854DF701B4
:10C4C000EE0FFF1FEE0FFF1FE80FF91FC280D38092
:10C4D0000E94854D0894E11CF11CF701EE0FFF1F2F
:10C4E000EE0FFF1FE80FF91F40815181C501B60112
:10C4F0000E940162E016F10600F30F900F90CF91B9
:10C50000DF911F910F91FF90EF90DF90CF90BF9040
:10C51000AF900895CF93DF93CAECD1E16091E01121
:10C520007091E111CE014CEB52E620E030E00E9428
:10C53000794A0E949E686091E0117091E1110E9419
:10C540003B81BC01CE01409741ED52E620E030E056
:10C550000E94794ADF91CF9108950F93013051F4F1
:10C560008091DA119091DB119093E1118093E011A9
:10C570000E948A620F9108958091E0119091E111DB
:10C580002091DE113091DF11880F991F281739078C
:10C5900008F4C9019093E1118093E0110E948A622E
:10C5A0000895EF92FF92CF93DF930E94284E0E944E
:10C5B000854DE82EE7017E01F92EE70119821882E8
:10C5C0000E94FC6126C028813981F901EE0FFF1F0E
:10C5D000EE0FFF1FEC0FFD1FDC0112964D915C91D9
:10C5E0001397538342832F5F3F4FF901EE0FFF1FD5
:10C5F000EE0FFF1FEC0FFD1F14964D915C911597E8
:10C6000051834083398328830E947A48282F392F09
:10C61000C901009721F0FC0120852223A1F6888121
:10C620009981880F991F880F991F02960E94804D4B
:10C6300088819981009721F08FEA91E10E94F74467
:10C64000DF91CF91FF90EF900895EF92FF920F93BB
:10C650001F93CF93DF93FC018B017A01E9018FEAED
:10C6600091E1BF014AEB56E00E94D9441093DB11DF
:10C670000093DA11F092DD11E092DC11D093DF111A
:10C68000C093DE118DEA92E60E94F761DF91CF91AF
:10C690001F910F91FF90EF900895CF93DF93CAEC15
:10C6A000D1E1CE010E94004BCE0140970E94004B89
:10C6B000CE014B970E94F444DF91CF910895809171
:10C6C000E0119091E11108950E9438450895EF928C
:10C6D000FF92CF93DF93E091BE06F091BF060995DC
:10C6E000EC01009729F06A817B8181E00E94AE4EC7
:10C6F000CE01DF91CF91FF90EF9008950F931F939C
:10C70000CF93DF938C01E091C006F091C1060995AB
:10C71000EC01F8016281738181E00E94AE4E21E05C
:10C7200030E0209711F420E030E0C901DF91CF9193
:10C730001F910F910895E091C206F091C3060995EB
:10C740000895FC0120E030E004C08181280F311DF4
:10C75000329680818823C9F7C9010895FC0181813F
:10C7600090E0308120E0822B932B02C0880F991F2C
:10C770006A95E2F7892F9927FA01EC53F94F208146
:10C7800030E08223932328E030E0241B350B02C0E5
:10C79000969587952A95E2F708956F927F928F92EA
:10C7A0009F92AF92BF92CF92DF92EF92FF920F9340
:10C7B0001F93CF93DF936C017B015A0189012830CD
:10C7C000310544F4CB01BA01A9010E94AE63F60120
:10C7D000808341C0390133E0759467943A95E1F75D
:10C7E0004115510521F04C01C0E0D0E016C0DB013D
:10C7F000FC01C0E0D0E08D9181932196C615D7054C
:10C80000D4F3A801477050704115510521F1C701BB
:10C810008C0F9D1F60E070E019C0C7018C0F9D1F39
:10C82000B50148E050E00E94AE63F40181934F01EE
:10C830002196C615D7058CF3A80147705070411595
:10C84000510549F0C7018C0F9D1FB5010E94AE63D1
:10C85000CC0DDD1D8883DF91CF911F910F91FF904B
:10C86000EF90DF90CF90BF90AF909F908F907F9090
:10C870006F9008954F925F926F927F928F929F92E6
:10C88000AF92BF92CF92DF92EF92FF920F931F93DE
:10C89000DF93CF9300D000D0CDB7DEB70E94854D97
:10C8A000E82E092F82E090E00E94614D009709F484
:10C8B00064C0EE2DF02F918180E02081820F911DC8
:10C8C0000E944C457C01009709F459C00E94854D97
:10C8D0003C01F7014681242F30E02770307081E061
:10C8E00090E02115310511F480E090E046954695E1
:10C8F0004695840F911D0E94614D0097F1F1F7015B
:10C9000004811581CC24DD2453E0452E512C4C0E9E
:10C910005D1E4E010894811C911C2AC0F801A18063
:10C92000BB24B60143E0759567954A95E1F7660D1E
:10C93000771DA60147705070883150F0C4019501F1
:10C940000E94CD63F8018081B4010E94C24E0CC0E8
:10C950001C821B82C20195010E94CD636B817C8188
:10C96000F80180810E94AE4ECA0CDB1C0E5F1F4F87
:10C97000F8018081882391F602C0EE24FF24C701CC
:10C980000F900F900F900F90CF91DF911F910F910B
:10C99000FF90EF90DF90CF90BF90AF909F908F90DF
:10C9A0007F906F905F904F900895FC0150E080E180
:10C9B00090E0861B970B821B930B02C0440F551F00
:10C9C0008A95E2F78081852B80838181842B818306
:10C9D00008956F927F928F929F92AF92BF92CF9263
:10C9E000DF92EF92FF920F931F93CF93DF938C010F
:10C9F0005B016A0179012830310524F4C801FA018C
:10CA0000408156C0390163E0759467946A95E1F7F7
:10CA1000A114B10421F04A01C0E0D0E021C0DA0144
:10CA2000F80180E090E02D912193019686159705FD
:10CA3000D4F397012770307021153105D9F1F60133
:10CA4000E80FF91F408150E068E070E0621B730B53
:10CA500002C0559547956A95E2F7800F911F26C051
:10CA6000F40141914F01C8018C0F9D1FB50128E0D1
:10CA700030E00E94D5642196C615D7058CF3970146
:10CA80002770307021153105A9F0F601EC0FFD1F5C
:10CA9000408150E0C5010896821B930B02C055955A
:10CAA00047958A95E2F7C8018C0F9D1F60E070E002
:10CAB0000E94D564DF91CF911F910F91FF90EF906D
:10CAC000DF90CF90BF90AF909F908F907F906F90AE
:10CAD00008954F925F926F927F928F929F92AF9242
:10CAE000BF92CF92DF92EF92FF920F931F93DF934B
:10CAF000CF9300D0CDB7DEB78C01DC0116964C91F8
:10CB00001697842F90E08770907021E030E00097B6
:10CB100011F420E030E04695469546957901E40E03
:10CB2000F11CC70102960E94ED4D009709F453C015
:10CB30000E948D4DFC01D80112968C911297808332
:10CB400013968C9181830E948D4DF2E06F2E712C93
:10CB5000680E791EC30160E070E0A7010E948A851B
:10CB6000F801C480D58000E010E02E010894411C3B
:10CB7000511C2AC0D60111968C90119799247801E6
:10CB8000E3E0F594E794EA95E1F7E60CF71C77E02B
:10CB9000A72EB12CA022B122883130F00E94CC4EB9
:10CBA000AC01C701B50107C00E94B94E9A838983C1
:10CBB000C701B501A20194010E94E964080D191D85
:10CBC000E2E0F0E0CE0EDF1ED6018C91882391F6D4
:10CBD00021E030E002C020E030E0C9010F900F906A
:10CBE000CF91DF911F910F91FF90EF90DF90CF9049
:10CBF000BF90AF909F908F907F906F905F904F907D
:10CC00000895E091F206F091F30609950895E091F8
:10CC10009B06F0919C0609950895E091F606F09127
:10CC2000F70609950895E091F806F091F90609953F
:10CC3000089580E090E008950895E0917D06F091D8
:10CC40007E0609950895009731F0E0917D06F091F8
:10CC50007E0609950895E0917F06F091800609957A
:10CC6000089580E090E008950F931F93DF93CF9392
:10CC7000CDB7DEB7E0970FB6F894DEBF0FBECDBFDD
:10CC80000E94D74D8C010E94854D602FAE014F5FF1
:10CC90005F4F0E94676E882309F445C088A99801F8
:10CCA000281B3109C9010E94614D0097E1F12E81D5
:10CCB000222371F18A859B853BEA8D3C930721F005
:10CCC0003FEF8F3F930779F5223041F088E090E005
:10CCD00007C0019722912F3F41F00BC082E090E006
:10CCE000FE01E80FF91F3C96F4CF181619068CF3D5
:10CCF0000FC089E1BE01645F7F4F0E94C24E89E18F
:10CD00000E94CC4E6DEC75E20E948A44009759F067
:10CD100088E1BE016A5E7F4F0E94C24EE091DB0651
:10CD2000F091DC060995E0960FB6F894DEBF0FBED1
:10CD3000CDBFCF91DF911F910F910895AF92BF9218
:10CD4000CF92DF92EF92FF920F931F93DF93CF93D7
:10CD5000CDB7DEB7E0970FB6F894DEBF0FBECDBFFC
:10CD60006C018B01FE01319680E3DF011D928A95F3
:10CD7000E9F781E089838CE00E94B94E8C831D82A3
:10CD80001F828091E41189878F5F8093E41183E093
:10CD9000E82EE8868DEC9BEA9B878A8789E10E94D2
:10CDA000CC4E65EB75E00E948A44009731F082E03A
:10CDB0008E838FEF8C878D8709C089E10E94CC4ECE
:10CDC000BC01CE010C960E948144EE828DEC9BEA60
:10CDD0009D8B8C8BCE0146966DEC75E20E94814452
:10CDE0000E94854D9FA78EA70E94D74D88AB7E01DC
:10CDF0000894E11CF11CC7010E945E6DA82E90E012
:10CE00000E94ED4D009741F10E948D4DBC01C7017C
:10CE10004A2D0E947C6DA0907306B09074060E940B
:10CE20008D4D7C010E94E14DBC01C701F5010995C2
:10CE3000C114D10489F0009721F08130910561F48B
:10CE400004C0C80160E070E003C0C80164E070E0A5
:10CE500041E050E0F6010995E0960FB6F894DEBF88
:10CE60000FBECDBFCF91DF911F910F91FF90EF903B
:10CE7000DF90CF90BF90AF9008950E949E688093FE
:10CE8000E411E0917D06F0917E0609950895EF92F8
:10CE9000FF92CF93DF93E82EE7017E01F92EE701A1
:10CEA00004C060E070E00E94EF468991999100977C
:10CEB000C1F7DF91CF91FF90EF900895EF92FF922D
:10CEC000CF93DF93E82EE7017E01F92EE70102C040
:10CED0000E943446899199910097D1F7DF91CF91C3
:10CEE000FF90EF900895CF93DF93EC017B836A83EB
:10CEF0000E94405799838883DF91CF910895FC0168
:10CF00008081918122813381820F931F918380835D
:10CF10000895CF93DF93EC010E9440579983888353
:10CF2000DF91CF910895CF93DF93EC010E9440579A
:10CF300028813981821B930B019621E030E04A81E0
:10CF40005B814817590710F020E030E0C901DF91FC
:10CF5000CF910895EF92FF92CF93DF93FC01C281AE
:10CF6000D38180819181C80FD91F0E944057C81B6F
:10CF7000D90BCE01DF91CF91FF90EF900895CF9321
:10CF8000DF93E6E4F8E2C8E0D8E2AAE3B8E211925F
:10CF9000119219921992199219921D9288E2EE3506
:10CFA000F807A9F7DF91CF9108950F931F93CF93BF
:10CFB000DF93FC01DC01A65CB74D8C91882339F12D
:10CFC0000091940010919500EF01CC0FDD1FCC0F64
:10CFD000DD1FC85FD74DDF01AA0FBB1FAA5BB74D8E
:10CFE0008D919C9111979801281B390B40E050E0DE
:10CFF000688179818A819B81260F371F481F591FBD
:10D00000288339834A835B8311961C930E93EE0F1A
:10D01000FF1FEE0FFF1FE85FF74D60817181828176
:10D020009381DF91CF911F910F91089560E070E09F
:10D03000CB010895FC01EE0FFF1FEE0FFF1FE85F0D
:10D04000F74D40835183628373830895EF92FF927B
:10D050000F931F93CF93DF932AE338E2C8E0D8E21F
:10D06000E6E4F8E2D9018D919D018823C9F0409151
:10D07000940050919500808191817A01E81AF90A13
:10D0800000E010E088819981AA81BB818E0D9F1DEF
:10D09000A01FB11F88839983AA83BB8351834083D8
:10D0A00024963296B8E226343B07E1F6DF91CF9121
:10D0B0001F910F91FF90EF9008950E94DB6C0895EF
:10D0C0000F931F93FC01CB014091E5115091E611A4
:10D0D000338322831583048371836083F093E61185
:10D0E000E093E5114115510511F40E94F56C80E0C3
:10D0F00090E01F910F9108958091E5119091E611B4
:10D100000097C1F01092E6111092E511DC0114961F
:10D110006D917C9115971296ED91FC91139709955D
:10D12000E091E511F091E611309721F08081918135
:10D130000E94F56C08950E94298208950E9424821D
:10D1400008958CEF96E00E94284784E097E00E94C3
:10D1500028470895EF92FF92CF93DF930E94944D5A
:10D160000097C9F084E097E00E944847E82EE70165
:10D170007E01F92EE701209731F10E94D74D998366
:10D1800088830E94D24D9B838A83C70104960E94A4
:10D19000004D8CAB18C08CEF96E00E944847EC0124
:10D1A0007E01F92EE701209771F0C70102960E94D7
:10D1B000174D99838883B7016E547F4FC7018E57EF
:10D1C0009F4F0E94844ECE01DF91CF91FF90EF9050
:10D1D0000895BC016E547F4F8E579F4F0E94844E1E
:10D1E0000895CF93DF93EC018CEF96E0BE010E948F
:10D1F0009347009719F08CEF96E009C084E097E020
:10D20000BE010E949347009729F084E097E0BE0199
:10D210000E946E47DF91CF910895EF92FF92CF93D6
:10D22000DF93EC018CEF96E0BE010E9493470097DC
:10D2300079F068817981CE0102960E94514EBE013B
:10D240006E547F4FCE018E579F4F0E94994E1BC048
:10D2500084E097E0BE010E9493470097A1F00E94EE
:10D26000284E688179818A819B810E94514E8CA9C8
:10D2700090E00E94ED4D0E948D4D4CA92496BE0178
:10D2800050E00E948185DF91CF91FF90EF9008954B
:10D29000EF92FF92CF93DF93EC018CEF96E0BE010B
:10D2A0000E949347009711F022960DC084E097E00A
:10D2B000BE010E949347009721F00A80DB81C02DB8
:10D2C00002C0C0E0D0E0CE01DF91CF91FF90EF909F
:10D2D0000895FC0180819181089570E06F5B7F4F1C
:10D2E000660F771F680F791FCB010895E62FF0E0D6
:10D2F000EF5BFF4FEE0FFF1FE80FF91F8081918159
:10D30000089508958DE398E10E949E49009721F0C9
:10D310008DE398E10E9489490895E0914A18F091BF
:10D320004B18309711F00995089580E00895EF9219
:10D33000FF920F931F93CF93DF93EC018A018881B3
:10D340009981009731F023E08C30920709F006C1F3
:10D350002BC080E00BC0E82FF0E0EE0FFF1FEE0FB8
:10D36000FF1FE55DF74E118210828F5F843098F3C6
:10D370008093451880916C0F90916D0F90933C189D
:10D3800080933B180E942D4680935E288DE398E1A0
:10D3900060E470E00E9473490E94F66F8CE093E0B5
:10D3A0009983888381E0DDC0623009F4B9C06330BD
:10D3B00030F4662309F489C0613081F79CC0673876
:10D3C00019F0683859F741C0109246184BE2E42E24
:10D3D00048E1F42E18C0F7018281938180179107EC
:10D3E00049F4808191810E943D71F7011182108280
:10D3F0001382128284E090E0E80EF91E80914618B4
:10D400008F5F8093461880914618843020F3EEE6B3
:10D41000FDE2848D958D8017910719F4158E148E79
:10D42000118EB0969DE2EE3EF90799F7E4E0FEE238
:10D43000818592858017910711F4158214823D969B
:10D440002EE2E638F207A1F7A9CF88E14D3358075D
:10D4500009F0A4CFCA010E949E49009709F49ECF0B
:10D46000109246182DC0F0E035E0EE0FFF1F3A9500
:10D47000E1F7E259F24D818D8823E9F08DE398E1DF
:10D480000E9489498091461890E025E0880F991FF5
:10D490002A95E1F78259924D90936D2D80936C2DD2
:10D4A00082E00E94717180915F28909160280097BE
:10D4B00011F00E948D69809146188F5F8093461805
:10D4C000E0914618E43078F269CF4115510509F42E
:10D4D00065CF50936D2D40936C2D83E00E94717148
:10D4E00080915F2890916028009711F00E948D69CB
:10D4F0000E94826953CF4115510509F44FCF5093D3
:10D50000692D4093682D85E00E94717180915F289C
:10D5100090916028009709F441CF0E948D693ECF19
:10D5200080915F2890916028009709F437CF80910F
:10D530007028863031F48091882881FF02C00E94D3
:10D54000826981E00E94717180915F2890916028CA
:10D55000009709F423CF0E94C06B20CF1982188254
:10D5600083E0DF91CF911F910F91FF90EF9008958D
:10D5700090934B1880934A18089520916C0F309126
:10D580006D0F60E0EBE2F8E113C040815181481774
:10D59000590761F4428153814217530739F460936C
:10D5A0004918118210820E943D71089534966F5F70
:10D5B000643058F360934918089540E0EBE2F8E1D5
:10D5C00016C0542F5F5F208131812115310569F428
:10D5D000409348189183808320916C0F30916D0F98
:10D5E000338322830E94577108953496452F443027
:10D5F00040F3409348180895FC0180916C0F90917E
:10D600006D0F958F848F778F668F0895FC018091C1
:10D610006C0F90916D0F928781877487638708954F
:10D62000CF93DF93EA010E94B970FC01009741F0AB
:10D6300080916C0F90916D0F92878187D487C387FB
:10D64000CF01DF91CF9108950F931F93DF93CF9375
:10D6500000D000D0CDB7DEB78C01AB018FEF89834E
:10D660008A838B838C83CE010196B8010E94106B54
:10D67000FC01009711F015830483CF010F900F90E8
:10D680000F900F90CF91DF911F910F91089589E135
:10D6900097E062E040E050E00E94E046109260288F
:10D6A00010925F280895AC0189E197E061E00E9443
:10D6B000BD460895AC0189E197E060E00E94BD4657
:10D6C00008950F931F93CF93DF93EA010E942F7069
:10D6D0008C01009761F080916C0F90916D0FF801B3
:10D6E000958F848FD78FC68FC8010E945A6BC8014F
:10D6F000DF91CF911F910F910895CF93DF93A09168
:10D700006C2DB0916D2D109719F0ED016C9605C040
:10D71000C091682DD091692D29968091672D86FF43
:10D7200022C01092471840E0EBE2F8E116C02081D9
:10D73000318114968D919C9115972817390759F4CA
:10D7400082819381009739F04093471899838883A9
:10D750001B821A8206C034964F5F443040F34093D8
:10D7600047180E94826988819981009731F04A8127
:10D770005B8160915E280E94E046DF91CF91089521
:10D780000F931F93CF93DF9380917028863009F019
:10D7900074C080915F289091602825E080309207C6
:10D7A00009F06BC0C4E9D2E0D0936028C0935F2831
:10D7B00002E00093692814E910936A2810928C28DB
:10D7C00010928B280E94EE6F8095909590938C28F4
:10D7D00080938B2810927228109271280E94DD6F1E
:10D7E0008095909590937228809371280E948D69FE
:10D7F000D0936028C0935F280093692810936A280B
:10D8000090916A2D80916B2DE92FF82FDF01A4599B
:10D81000BD4F8CE692E00D9001920197E1F78FE702
:10D8200098E26CE672E00E94816F80916328809399
:10D830007F28809164288093802880916528809338
:10D840008128809166288093822810928C281092DB
:10D850008B280E94EE6F8095909590938C288093F2
:10D860008B2810927228109271280E94DD6F80958B
:10D87000909590937228809371280E948D69DF9112
:10D88000CF911F910F910895282F392FF90120E092
:10D8900030E080E0A8E112C0419198E0542F582771
:10D8A000B52FB17050FD8A278695B13009F4806894
:10D8B000915011F04695F2CF2F5F3F4F2617370753
:10D8C00059F708951F920F920FB60F920BB60F9251
:10D8D00011242F933F934F935F936F937F938F9375
:10D8E0009F93AF93BF93EF93FF9380919400909198
:10D8F000950090934B2880934A2881E080933C28A0
:10D9000080917100807D809371000E947C6880917D
:10D910003C288823E9F18091940090919500209112
:10D920004A2830914B2882179307A0F48091102841
:10D9300090911128A0911228B09113288C57914EE4
:10D94000AF4FBF4F8093102890931128A0931228B7
:10D95000B09313288091940090919500821B930BB3
:10D96000A0E0B0E0209110283091112840911228B9
:10D9700050911328820F931FA41FB51F8093102866
:10D9800090931128A0931228B093132810923C284A
:10D99000FF91EF91BF91AF919F918F917F916F9187
:10D9A0005F914F913F912F910F900BBE0F900FBE43
:10D9B0000F901F9018959FB7F894E1E7F0E08081F1
:10D9C000807D808388B38F6288BB10929000E1E9EC
:10D9D000F0E0108210929200109295001092940044
:10D9E0008081856080839FBF08952FB7F8949093BE
:10D9F00099008093980088B38F6288BBE1E7F0E0DC
:10DA00008081826080832FBF0895EF92FF92CF9331
:10DA1000DF93FC01DB0185E0EB0119928A95E9F7C0
:10DA2000858190E083709070009711F082E08C9374
:10DA3000878190E083709070009721F082E01296C9
:10DA40008C931297858190E083709070009799F085
:10DA5000878190E083709070009769F02389348902
:10DA6000818592852817390731F481E084831296E5
:10DA70001C92129701C0148285818370825082307B
:10DA800030F4C82FD0E0CD5DD84F888101C080E050
:10DA900011968C931197E781E370E250E23028F4FD
:10DAA000F0E0ED5DF84F808101C080E013968C932B
:10DAB0001397DF91CF91FF90EF900895DF93CF936D
:10DAC00000D000D00F92CDB7DEB7BE016F5F7F4FA1
:10DAD0000E94056D89819A81890F8D5F9B81890FD5
:10DAE0009C81890F9D81890F0F900F900F900F904F
:10DAF0000F90CF91DF910895AF92BF92CF92DF92B6
:10DB0000EF92FF920F931F93DF93CF9300D000D03B
:10DB100000D0CDB7DEB78C017B01BE016F5F7F4FB8
:10DB20004E830E94056DC9809A81A92EBB24DB809B
:10DB30008C81682F70E095012C0D311D2D5F3F4FBA
:10DB40002D0D311D260F371F5D81250F311D4E8193
:10DB500050E0421753070CF4A8C0D80111964C911D
:10DB6000119750E041705070E3E0440F551FEA9563
:10DB7000E1F712962C91129730E02170307054E04A
:10DB8000220F331F5A95E1F7242B3C913770232B3A
:10DB900013963C911397E32FF0E0E170F07045E0AD
:10DBA000EE0FFF1F4A95E1F72E2B14963C91149728
:10DBB000E32FF0E0E170F07036E0EE0FFF1F3A95D2
:10DBC000E1F72E2BF701208315964C91159750E025
:10DBD00043705070440F551F440F551F16962C91DB
:10DBE000169730E02370307054E0220F331F5A959F
:10DBF000E1F7242B17963C9117973295330F330F8B
:10DC0000307C322B318318962C9118972283FC2D6F
:10DC1000F23069F419962C91D70113962C9313972F
:10DC2000F801228514962C93149745E001C043E037
:10DC3000E92FF0E03B96E00FF11F542F0AC0970147
:10DC4000250F311DC290D901CC925F5F0894A108C5
:10DC5000B108A114B10499F7940FBD2DB23089F425
:10DC6000F701E90FF11DD80153962C9153972083AA
:10DC70009F5FF701E90FF11D54962C915497208373
:10DC80009F5FE82FF0E07596E00FF11F292F08C085
:10DC9000D701A20FB11D32913C932F5F61507040AC
:10DCA00061157105A9F7890F01C080E026960FB6AE
:10DCB000F894DEBF0FBECDBFCF91DF911F910F91C2
:10DCC000FF90EF90DF90CF90BF90AF900895BF92FC
:10DCD000CF92DF92EF92FF920F931F93CF93DF9338
:10DCE0007C01D62EEA01633008F4ADC0FC018081CE
:10DCF000B82EB294B694B694B3E0BB22F1E0BF2242
:10DD0000F7019181292F269526952370C92EC2945B
:10DD1000C694C694A3E0CA22382F37703883382FB0
:10DD200036953695369531703983382F3295317066
:10DD30003A838295869581708B83BC822D83892F4F
:10DD4000829583708E83CF828281888787010D5F61
:10DD50001F4F222361F1F801918180E0F7013381A7
:10DD6000830F911D9A87898787010B5F1F4F223090
:10DD700081F4CA010B9665EB75E00E948144F801BD
:10DD800081818B87F70185818C878701095F1F4F10
:10DD900016C02330A1F4F7013D96DA011B9682915B
:10DDA0008D93E017F107D9F7085F1F4F08C0CA012C
:10DDB0000B9665EB75E00E9481441A861986CC208B
:10DDC00089F1BB2059F4F801918180E02081820F14
:10DDD000911D9C8B8B8B0E5F1F4F04C089859A858C
:10DDE0009C8B8B8BFC2DF23071F4CE01459665EB4C
:10DDF00075E00E948144F80181818D8B80818E8B3A
:10DE00000E5F1F4F17C0FC2DF330A1F4085F1F4FAA
:10DE1000D801FE01759680E09E9191938F5F8830C6
:10DE2000D9F708C0CE01459665EB75E00E948144A4
:10DE30001C8A1B8A802F8E199D2D981B9FA71EA7B9
:10DE40000DA7D81608F480E0DF91CF911F910F91B4
:10DE5000FF90EF90DF90CF90BF9008959C014150CC
:10DE60005040460F571FDB0110C0FC91E0E01196B7
:10DE70008C911197BF01680F711D260F371F261750
:10DE8000370710F42F5F3F4F1296A417B50768F3BA
:10DE9000A417B50749F49C9180E0280F391F281773
:10DEA000390710F42F5F3F4FC9010895CF93DF93D7
:10DEB00090916A28C92FD0E064973091692820E0BA
:10DEC000C20FD31F9E01280F311DC90163E778E2FD
:10DED00048E050E00E942E6F6BE778E2AE010E94AE
:10DEE0002E6F009719F0382F292F02C02FEF3FEF28
:10DEF000C901DF91CF91089590935B1880935A18D0
:10DF00000895FC014381460F40936628872F992787
:10DF10002281280F20936528A181A0936428508135
:10DF20005093632830E02817390748F48A2F8F5F11
:10DF300080936428882319F45F5F50936328842FAB
:10DF400090E070708617970798F4809165288F5F2E
:10DF500080936528882361F4809164288F5F809383
:10DF60006428882329F4809163288F5F8093632835
:10DF70000895BC0180916C2D90916D2D08960E94A2
:10DF8000816FE0916C2DF0916D2D809163288087D9
:10DF90008091642881878091652882878091662896
:10DFA000838708959C01AB0180E090E0B9010E9455
:10DFB0002E6F382F292FC901089580E090E067E681
:10DFC00078E244E150E00E942E6F009719F0382F5C
:10DFD000292F02C02FEF3FEFC901089586E00E946C
:10DFE000566F089581E10E94566F089580E009C040
:10DFF000E82FF0E0EE0FFF1FE251F24D1182108288
:10E000008F5F8430A8F380E00BC0E82FF0E095E04C
:10E01000EE0FFF1F9A95E1F7E259F24D118E8F5FD7
:10E02000843098F380E094E090935D1880935C18BE
:10E0300040E08DE090E00EC0242F30E0289FF001FA
:10E04000299FF00D389FF00D1124EC5FF14D1582E2
:10E0500014824F5F4A3080F34093581808952091FE
:10E060005C1830915D182F5F3F4F4DE7203034072B
:10E0700010F020E030E1522F432FA0E013C0EA2F30
:10E08000F0E0B5E0EE0FFF1FBA95E1F7E259F24D6F
:10E09000B18DBB2331F00480F581E02DE417F50745
:10E0A00011F3AF5FA43059F730935D1820935C18DB
:10E0B0001092581820E0E0E0F0E01EC0A22FB0E07F
:10E0C00035E0AA0FBB1F3A95E1F7A259B24D599618
:10E0D0003C915997332321F420935818FD0110C027
:10E0E000373049F4309731F05A964C915A97328D27
:10E0F000341708F4FD012F5F243000F320935818E3
:10E100003097A9F122E0218F209152182487209185
:10E110005318258720915418268720915518278752
:10E1200028ED34E0338B228B358B248B21E030E0DB
:10E13000318B208B138E21E0228F23E0208F168AD3
:10E1400020E1278B20915C1830915D18322723271E
:10E1500032273583248377836683DC012D913D91BB
:10E160004D915C9113972083318342835383CF0178
:10E1700008950F931F93CF93DF9320915C183091F4
:10E180005D184DE050E02F5F3F4FADE720303A077C
:10E1900010F020E030E1B22FA32F10E012C0C12F09
:10E1A000D0E0C49FF001C59FF00DD49FF00D112465
:10E1B000EC5FF14D0480F581E02DEA17FB0719F3C0
:10E1C0001F5F1A3061F730935D1820935C1810E0E0
:10E1D0002DE030E01AC0012F0F5FC12FD0E0C29FA9
:10E1E000F001C39FF00DD29FF00D1124EC5FF14DB3
:10E1F000DF011496448155814115510529F410938E
:10E200005818309749F433C0102F1A3020F3109368
:10E210005818E0E0F0E02BC020915C1830915D18B8
:10E2200032272327322711963C932E9377836683D8
:10E23000009729F4108211821282138209C0DC0136
:10E240002D913D914D915C91208331834283538385
:10E250008DE090E0C89FD001C99FB00DD89FB00D50
:10E260001124AC5FB14D80E418968C931897CF01C0
:10E27000DF91CF911F910F91089540E013C0E42FDB
:10E28000F0E0542F5F5FEE0FFF1FE251F24D20814F
:10E2900031812817390729F44093581811821082C8
:10E2A0000895452F443058F340935818089540E09E
:10E2B00013C0E42FF0E0542F5F5FEE0FFF1FE25119
:10E2C000F24D208131812115310529F440935818F0
:10E2D000918380830895452F443058F34093581814
:10E2E0000895EF92FF920F931F93CF93DF93C09106
:10E2F0006C2DD0916D2D843009F4F7C10FE818E230
:10E3000010936B2D00936A2D10936228009361285F
:10E31000833071F4898D90E08F7090708330910517
:10E3200009F074C088899989009709F02FC78DC0BA
:10E33000823009F08EC0809155188F5F80935518F8
:10E34000882399F4809154188F5F80935418882300
:10E3500061F4809153188F5F80935318882329F4B8
:10E36000809152188F5F80935218109260281092FB
:10E370005F281092032E1092022E898D873011F0A3
:10E38000853041F48A8D8F5F8A8F843109F0FEC613
:10E39000198EFCC6882309F4F9C628893989211504
:10E3A000310509F44EC09A8D292F21502A8F9923C7
:10E3B00009F0ECC69B8D983031F0282F2150223087
:10E3C00048F4953039F4198E80E88093672D0E94C7
:10E3D0007D6B95C5953048F423E030E0092E02C0EE
:10E3E000220F331F0A94E2F701C020E32A8F9F5FB8
:10E3F0009B8F90E08F70907083309105E1F08430B6
:10E4000091054CF48130910509F461C38230910586
:10E4100009F0BCC60DC08630910509F40CC58830E2
:10E42000910509F408C58430910509F0AFC603C50C
:10E43000109288284FC384E08093672D0E947D6BE3
:10E4400090C58F70833009F0A1C688E08093672D56
:10E450004BC5853019F5E091682DF091692D8481C7
:10E460009581009709F492C610926D2D10926C2D33
:10E470000C50104010936B2D00936A2D109362285E
:10E48000009361281092032E1092022E10926028A1
:10E4900010925F2888E08093672D25C108521040B4
:10E4A00080916728853409F071C69091692880E0D1
:10E4B00020916A287C01E20EF11C80915F289091E6
:10E4C00060288E159F0508F461C6F0926028E092DE
:10E4D0005F2880916D2890E08F739070009709F00D
:10E4E00055C680916E28882309F050C68091FE2D74
:10E4F0009091FF2DC0912907D0912A078C179D0775
:10E5000059F44091002E5091012E20912B0730910B
:10E510002C0742175307A1F02091772830917828D3
:10E520002817390709F032C62091792830917A28C6
:10E530008091002E9091012E2817390709F026C6E8
:10E540000E94DD6F2FEF8F3F920709F01FC6809169
:10E550007028863009F431C18131E9F1813009F048
:10E5600015C680917B28883009F010C610927B2850
:10E5700080917D2890917E284FEF873F940710F07F
:10E58000099601C0089690937E2880937D288091FB
:10E59000732890917428A0917528B0917628809363
:10E5A000772890937828A0937928B0937A2880913F
:10E5B000FE2D9091FF2DA091002EB091012E809301
:10E5C000732890937428A0937528B093762880E4DC
:10E5D000F8018087B8C5C7014C9790936028809355
:10E5E0005F2883E898E290936B2D80936A2D809149
:10E5F000812890918228009739F00E94F26FFFEFF6
:10E600008F3F9F0709F0C2C520917D2830917E2859
:10E610002115310509F4BAC584E09EE29093692D75
:10E620008093682D60912B0770912C0740912507EE
:10E6300050912607009127071091280739C084813F
:10E640009581009781F12817390769F586819781AF
:10E65000009739F0A0917B28B0917C28A817B907C2
:10E6600011F5808191818C179D0729F4A281B381D6
:10E67000A617B70739F18417950729F4A281B3814A
:10E68000A017B107F9F0A0917328B0917428A817CA
:10E69000B90749F4A0917528B091762882819381B9
:10E6A000A817B90779F03D96F093692DE093682D8E
:10E6B000E091682DF091692D8EE2E638F80708F4B4
:10E6C000BECF64C510926D2D10926C2D82E08093A8
:10E6D000672D83E898E290936228809361281092D6
:10E6E000032E1092022E0E947D6B8091022E90913B
:10E6F000032E009709F44AC59C01245E3F4F3093D6
:10E70000602820935F283093692820936A28E0913D
:10E71000682DF091692D208520936F2821E12093A9
:10E7200070280896982789279827909380288093A7
:10E730007F2810928228109281288481958190935D
:10E740007C2880937B288681978190937E28809374
:10E750007D288091FE2D9091FF2DA091002EB091EB
:10E76000012E8093732890937428A0937528B093FA
:10E77000762880819181A281B381809377289093BC
:10E780007828A0937928B0937A288FE898E290931C
:10E790006B2D80936A2D0E94F26F809590959093D7
:10E7A000822880938128009709F0CDC48FEF9FEFD6
:10E7B0009093822880938128C6C40E94EE6FEFEF69
:10E7C0008F3F9E0709F0E2C480917D2890917E28BA
:10E7D000009709F4DBC420917B2830917C28211517
:10E7E000310509F4D3C4CEE6DDE2498D4423E9F0D6
:10E7F0006C817D8186179707C1F46E817F81261712
:10E80000370799F4E0917328F09174286881798131
:10E81000E617F70751F4E0917528F09176286A81A0
:10E820007B81E617F70709F46DC1A096FDE2CE3EA5
:10E83000DF07D9F6209188282F732230B9F49093FE
:10E8400057188093561840E00DC0E42FF0E0EE0F0B
:10E85000FF1FE251F24D208131814F5F82179307F4
:10E8600009F46EC0443088F340935818809188288A
:10E8700082FD8CC484E1F80181A388E290E090934A
:10E88000602880935F2880E580A380918228909102
:10E890008628938F3091812890918528928F368F8A
:10E8A0002091802890918428918F258F90917F28A6
:10E8B0009093581840918328408F948F8F5F878F53
:10E8C000882361F4832F8F5F868F882339F4822F0A
:10E8D0008F5F858F882311F49F5F948F80917B28B1
:10E8E00090917C28909357188093561820917D28FA
:10E8F00030917E28F801358B248B978B868B809105
:10E90000732890917428A0917528B09176288093EF
:10E91000772890937828A0937928B0937A288091CB
:10E92000FE2D9091FF2DA091002EB091012E80938D
:10E93000732890937428A0937528B0937628E8C321
:10E940001092581880E0C0E0D0E022C0E82FF0E03C
:10E9500075E0EE0FFF1F7A95E1F7E259F24D918DC8
:10E96000992321F480935818EF0116C0973079F459
:10E97000209721F0228D9A8D921748F4C82FD0E06D
:10E9800065E0CC0FDD1F6A95E1F7C259D24D8F5F6C
:10E990008430E0F280935818209709F4F7C3D0939D
:10E9A0006D2DC0936C2D83E08A8F888F1E8A84E042
:10E9B0008F8B1B8E80917D2890917E289D838C83E8
:10E9C00080917B2890917C289F838E8380917328EF
:10E9D00090917428A0917528B091762888839983A6
:10E9E000AA83BB8381E0898F809152188C878091A4
:10E9F00053188D87809154188E87809155188F8772
:10EA000081E090E0998B888B809182288B87809120
:10EA100081288A8780918028898780917F288887AC
:10EA200081E090E00E94B96F80918728282F30E024
:10EA3000207F3070213531050CF449C082958F70EC
:10EA400090E00597880F991F880F991F50915918CA
:10EA500040E034C0F901E959F74D50A5552329F498
:10EA6000409358181092591832C0513011F44F5F2A
:10EA700025C05230E1F461A56430C9F440935818C0
:10EA80005093591832A520E083A590E0822B932B58
:10EA90009093571880935618F4E0893D9F0710F023
:10EAA00088ED94E09B8B8A8B9D8B8C8B10C02959B1
:10EAB000374DF90121A5222331F0420F242F30E0F8
:10EAC000281739073CF2409358185093591880E1A1
:10EAD000809388288091882882608093882882E0AB
:10EAE00080938F2884E0809390288093912888EDEC
:10EAF000809392288CE290E09093602880935F2826
:10EB000080E6B3C2D0936D2DC0936C2D1092672D0B
:10EB10008091882890E082FF03C0198E80E24EC267
:10EB20002091872822952F70220F220F20935818AA
:10EB3000B701621B71099B0124513040309360285A
:10EB400020935F2850E04F7050704230510539F4E7
:10EB5000AC014F7350704231510551F42AC041301D
:10EB6000510531F4AC014F7350704230510509F139
:10EB70002115310531F49C012370307021153105C8
:10EB8000C1F030917F282885321709F064C2309196
:10EB900080282985321709F05EC2309181282A85A4
:10EBA000321709F058C2309182282B85321709F0AC
:10EBB00052C284FF4AC0688979896115710509F4D8
:10EBC00044C0CE010C960E94816F309183288091C1
:10EBD00063283817D1F5209184288091642828175C
:10EBE000A1F59091852880916528981771F58091FD
:10EBF000862840916628841741F53C872D879E879B
:10EC00008F878B8D8823D1F42E89888D9A8D891BCF
:10EC1000922F969596959695891B280F2E8B87FD9A
:10EC200081959F89392F36953695931B980F9F8B29
:10EC3000822F869586958695890F888F81E08093AF
:10EC4000672D888D8A8F198A188A298D30E0C9012D
:10EC50008F7090708430910509F4B5C185309105AD
:10EC600064F482309105C9F1833091050CF0B9C08C
:10EC70008130910509F08AC211C08630910509F4EE
:10EC8000E2C1863091050CF4BEC18730910509F4CC
:10EC9000E2C18830910509F079C28AC18091672D5F
:10ECA00080FF14C083E0898F80E48093672D198AE8
:10ECB000188A80915F2890916028009709F410C10C
:10ECC00022E42093672D0E94B96F0AC180918828A1
:10ECD0008F73823009F05AC2FACE8091672D80FF7F
:10ECE00075C0809188288F73823109F06FC0809140
:10ECF0008728282F30E0207F3070213531050CF433
:10ED000049C082958F7090E00597880F991F880FF2
:10ED1000991F5091591840E034C0F901E959F74D55
:10ED200050A5552329F4409358181092591832C011
:10ED3000513011F44F5F25C05230E1F461A56430C9
:10ED4000C9F4409358185093591832A520E083A570
:10ED500090E0822B932B909357188093561874E071
:10ED6000893D970710F088ED94E09B8B8A8B9D8BF3
:10ED70008C8B10C02959374DF90121A5222331F080
:10ED8000420F242F30E0281739073CF240935818DF
:10ED90005093591883E0898F80917F2888878091CC
:10EDA00080288987809181288A87809182288B8713
:10EDB00081E090E00E94B96F82E48093672D198A08
:10EDC000188A1092602810925F288AC080E280938F
:10EDD000672D0E947D6BE0916C2DF0916D2D118E51
:10EDE00045CD8091882880FF2AC024FD28C08889CD
:10EDF0009989009709F0CAC180915F289091602895
:10EE000001960E94B96F2091672D822F80618093B7
:10EE1000672D80915F2890916028009719F02261FA
:10EE20002093672D0E947D6B81E090E0998B888B09
:10EE300088E0898F1B8E81E1809388280FC185FF30
:10EE40001CC050918D2840E080918E2890E0842B4A
:10EE5000952B40916A2D50916B2D480F591F50935F
:10EE60006B2D40936A2D40915F2850916028481B7C
:10EE7000590B5093602840935F2880915F289091B0
:10EE80006028009749F024FD07C02091672D22607B
:10EE90002093672D0E94B96F9091892880E020917E
:10EEA0008A28820F911D90935718809356182C89A9
:10EEB0003D892817390710F0009721F4309357182F
:10EEC0002093561880915618909157189B8B8A8BD7
:10EED0008091672D90E083709070009709F456C17F
:10EEE0001092032E1092022E0E947D6B8091672D4E
:10EEF00085FF07C01092032E1092022E198E84E116
:10EF00009BCF84FF0AC01092032E1092022E81E044
:10EF100090E0998B888B84E08CCF2091022E3091E9
:10EF2000032E21153105E1F080FF02C0198A188AED
:10EF300088899989009781F48A899B898217930728
:10EF400020F49093032E8093022E8091022E9091B4
:10EF5000032E998B888B04C09093032E8093022EEE
:10EF60001B8E809161289091622890936B2D8093E5
:10EF70006A2D8091022E9091032E009759F0888976
:10EF80009989009739F088969093602880935F283C
:10EF900088E10BC08091672D81FFF8C088E290E086
:10EFA0009093602880935F2880E1809388285CC0DC
:10EFB0008091672D80FFEAC0198E80E18093672DD4
:10EFC0000E947D6BE3C080915F289091602800973C
:10EFD00011F00E94B96F909188288091672D90FF61
:10EFE0000BC080FF06C087E0898F1A8E198A188AA5
:10EFF00019C086E0898F16C080FF1EC085E0898F0A
:10F00000198A188AC3C080915F2890916028009760
:10F0100011F00E94B96F8091882880FF0DC087E0B1
:10F02000898F1A8E81E090E00E94B96F80E1809311
:10F03000672D0E947D6B0FC080915F2890916028A2
:10F04000009749F4A3C08091672D80FF9FC087E09F
:10F05000898F1A8E9BC080E1F80181A388E290E03D
:10F060009093602880935F2880E580938728888527
:10F07000809383288985809384288A858093852836
:10F080008B85809386288C8580937F288D858093BF
:10F0900080288E85809381288F858093822886E0C2
:10F0A000809370288C819D8190937C2880937B280D
:10F0B0008E819F8190937E2880937D288091FE2D64
:10F0C0009091FF2DA091002EB091012E8093732876
:10F0D00090937428A0937528B0937628888199819D
:10F0E000AA81BB818093772890937828A093792870
:10F0F000B0937A28898D84FF05C010928A281092D7
:10F10000892806C084E08093892888ED80938A2826
:10F1100080E480936F2880915F289091602890937D
:10F12000692880936A2810928E2810928D28109258
:10F130008C2810928B280E94EE6F8095909590936A
:10F140008C2880938B2885E4809367281092682808
:10F1500010926E2810926D2880915A1890915B1829
:10F16000019690935B1880935A1890936B28809324
:10F170006C2810927228109271280E94DD6F809581
:10F180009095909372288093712804C01092602803
:10F1900010925F281092672DDF91CF911F910F91F0
:10F1A000FF90EF900895382F292FC9010895382F27
:10F1B000292F40E050E076276727762780E090E00F
:10F1C000CB0177276627262B372B482B592BB901E4
:10F1D000CA010895AC01E0916128F09162282227CC
:10F1E00033272E1B3F0B2959324D621773070CF43E
:10F1F0009B011216130664F42093022E3093032E03
:10F200004E175F0729F0CF01BA01A9010E9481853D
:10F2100008950F93DF93CF93CDB7DEB760970FB606
:10F22000F894DEBF0FBECDBF002309F459C0298377
:10F230003A834B835C836D837E838F839887E0E280
:10F24000E01B29813A814B815C811E16BCF0198636
:10F250001A861B861C868E2F992787FD9095909580
:10F2600081959F4F04C0220F331F441F551F8A955D
:10F27000D2F72D873E874F87588B2AC0CA01B90124
:10F28000002E04C0660F771F881F991F0A94D2F7BB
:10F2900069877A878B879C87DA01C90104C0B69594
:10F2A000A79597958795EA95D2F72D813E814F8155
:10F2B000588504C0220F331F441F551F0A95D2F7EB
:10F2C000822B932BA42BB52B8D879E87AF87B88B72
:10F2D00029853A854B855C856D857E858F859889E6
:10F2E00060960FB6F894DEBF0FBECDBFCF91DF9111
:10F2F0000F910895A0E1B0E0E0E8F9E70C94A78150
:10F3000029833A834B835C836D837E838F839887C5
:10F31000A986BA86CB86DC86ED86FE860F87188B9B
:10F320002D813E814F8158858D859E85AF85B88919
:10F33000281739074A075B07C8F082179307A40705
:10F34000B50790F029813A814B815C8189859A8546
:10F35000AB85BC85281739074A075B0738F0821749
:10F360009307A407B50720F482E003C080E001C042
:10F3700081E06096EAE00C94C3812F923F924F9215
:10F380005F926F927F928F929F92AF92BF92CF9235
:10F39000DF92EF92FF920F931F93DF93CF93CDB73E
:10F3A000DEB763970FB6F894DEBF0FBECDBF6C011A
:10F3B0007F876E87FC0117821682838181FD04C0DE
:10F3C0006FC34C855D8504C01E010894211C311C4F
:10F3D000F6019381EE85FF8593FD859193FF8191E1
:10F3E000FF87EE87882309F457C3853241F493FDE4
:10F3F000859193FF8191FF87EE87853259F490E0E4
:10F40000B6014A8B5B8B0E94E3854A895B895D87E5
:10F410004C87D7CF10E0FF2400E00032B0F48B32ED
:10F4200069F08C3228F4803251F0833271F40BC0D1
:10F430008D3239F0803349F401602CC002600460E1
:10F4400029C0086027C0006125C007FD2EC0282FF5
:10F4500020532A3098F406FF08C0812F880F182FF8
:10F46000110F110F180F120F15C08F2D880FF82EC6
:10F47000FF0CFF0CF80EF20E00620CC08E3221F46D
:10F4800006FD0AC3006406C08C3611F4006802C091
:10F49000883659F4EE85FF8593FD859193FF819120
:10F4A000FF87EE87882309F0B8CF982F95549330C3
:10F4B00018F40061805E06C0982F9556933008F0CE
:10F4C0009BC10F7E06FF16E06FE3E62EE022853635
:10F4D00019F4F0E4EF2A07C0863619F420E8E22A8E
:10F4E00002C011111150E7FE06C01C3340F4912EEA
:10F4F000939427E00BC0183030F4212F06C027E08A
:10F500003CE3932E03C027E017E09924CA01049638
:10F510009D878C87FA016081718182819381A1012D
:10F52000092D0E9491845C016980262D30E0398B81
:10F53000288B60FE03C0388933FF06C0E1FC06C09B
:10F54000E2FE06C000E205C00DE203C00BE201C00E
:10F5500000E0888999898C7090700097C1F1002330
:10F5600011F084E001C083E08F1558F4F81AE3FC31
:10F5700009C080E290E0B6010E94E385FA94C9F7E1
:10F5800001C0FF24002329F0802F90E0B6010E94E3
:10F59000E385888983FD03C003EE10E10EC00FED03
:10F5A00010E10BC0A114B10409F0805290E0B60143
:10F5B0000E94E3850F5F1F4F05C0AE2CBB2490E176
:10F5C000A922BB24F8018491882361F762C2E7FE77
:10F5D0000EC09A0CF889F4FF04C08A81813309F4C3
:10F5E0009A94191454F5292D293050F52DC0E6FCB4
:10F5F0002BC0812F90E08A159B054CF03CEFA316A1
:10F600003FEFB30624F080E8E82A01C0115011232F
:10F6100049F0E2E0F0E0EC0FFD1FE10FF11D808109
:10F620008033A1F3E7FE10C0912E9394812F90E0D8
:10F63000A816B90644F41A1907C09924939404C073
:10F6400098E0992E01C010E0E7FE07C01A141B04D1
:10F650003CF495012F5F3F4F05C025E030E002C02C
:10F6600021E030E0002311F02F5F3F4F112329F0FC
:10F67000812F90E00196280F391F8F2D90E02817D9
:10F68000390714F4F21A01C0FF244E2C5524C2018C
:10F6900089709070009749F406C080E290E0B6014E
:10F6A0000E94E385FA94FF20C1F7002329F0802F00
:10F6B00090E0B6010E94E38543FC09C006C080E3E8
:10F6C00090E0B6010E94E385FA94FF20C1F7E7FEBF
:10F6D00046C03501B7FE02C0662477242501089490
:10F6E000411C511C46185708420C531CF501E919DE
:10F6F000F1094F01812F90E000271127081B190BFA
:10F70000FFEF6F16FFEF7F0629F48EE290E0B6015F
:10F710000E94E385A614B70434F0861497041CF401
:10F72000F201808101C080E30894610871080894A7
:10F73000411C511C601671062CF090E0B6010E942D
:10F74000E385DECF6A147B0441F49A81963320F47A
:10F75000953319F4F889F4FF81E390E049C08A8178
:10F76000813311F02FEE622290E0B6010E94E38512
:10F77000112389F08EE290E0B6010E94E38502E059
:10F78000F101E00FF11D0F5F808190E0B6010E9452
:10F79000E3851150A9F744FE03C085E490E002C060
:10F7A00085E690E0B6010E94E385B7FC05C0A11490
:10F7B000B10441F464FE06C0B094A194B108B394BE
:10F7C0008DE201C08BE290E0B6010E94E38580E308
:10F7D00005C08F5FE6EFFFEFAE0EBF1EFAE0AF167B
:10F7E000B104BCF790E0B6010E94E385C501C09664
:10F7F000B6010E94E3854DC1833631F0833789F02D
:10F80000833509F059C022C09A012E5F3F4F3D87D2
:10F810002C87FA0180818983310181E0A82EB12CE7
:10F8200013C09A012E5F3F4F3D872C87FA016080FD
:10F83000718006FF03C0612F70E002C06FEF7FEFA1
:10F84000C3010E94A9855C010F7714C09A012E5F45
:10F850003F4F3D872C87FA016080718006FF03C00F
:10F86000612F70E002C06FEF7FEFC3010E947185CE
:10F870005C01006803FD1CC006C080E290E0B60198
:10F880000E94E385FA948F2D90E0A816B906A8F39C
:10F890000FC0F30107FD859107FF81913F0190E0C3
:10F8A000B6010E94E385F110FA940894A108B1080A
:10F8B000A114B10471F7EDC0843611F0893661F5F9
:10F8C00007FF0BC09A012C5F3F4F3D872C87FA0141
:10F8D00060817181828193810CC09A012E5F3F4FBC
:10F8E0003D872C87FA0160817181882777FD80959B
:10F8F000982F0F7697FF08C0909580957095619529
:10F900007F4F8F4F9F4F0068A1012AE030E00E9497
:10F91000EE86982E921841C0853721F40F7E2AE09A
:10F9200030E020C0097F8F36A9F0803720F4883579
:10F9300009F0B2C00BC0803721F0883709F0ACC0A5
:10F9400001C0006104FF09C0046007C004FF08C0D3
:10F95000066006C028E030E005C020E130E002C0CB
:10F9600020E132E007FF0AC0CA0104969D878C8718
:10F97000FA01608171818281938109C0CA01029676
:10F980009D878C87FA016081718180E090E0A10100
:10F990000E94EE86982E92180F7706FF09C00E7F00
:10F9A000911630F404FF06C002FD04C00F7E02C0B1
:10F9B000E92C01C0E12E802F90E004FF0CC0FE0175
:10F9C000E90DF11D2081203311F4097E09C0E39473
:10F9D00002FF06C004C086789070009709F0E39497
:10F9E000A02EBB2403FD14C000FF0FC0EF1428F4A9
:10F9F000192D1F0D1E19EF2C08C0192D06C080E20D
:10FA000090E0B6010E94E385E394EF14C0F304C0D4
:10FA1000EF1410F4FE1801C0FF24A4FE0FC080E311
:10FA200090E0B6010E94E385A2FE1FC0A1FE03C0C4
:10FA300088E590E010C088E790E00DC0C5018678A9
:10FA40009070009791F0A1FC02C080E201C08BE2AF
:10FA500007FD8DE290E0B6010E94E38506C080E3D9
:10FA600090E0B6010E94E38511509116C0F39A947C
:10FA7000F101E90DF11D808190E0B6010E94E3855E
:10FA80009920A9F706C080E290E0B6010E94E385C4
:10FA9000FA94FF20C1F795CCF6012681378102C088
:10FAA0002FEF3FEFC90163960FB6F894DEBF0FBE8C
:10FAB000CDBFCF91DF911F910F91FF90EF90DF901D
:10FAC000CF90BF90AF909F908F907F906F905F90FE
:10FAD0004F903F902F9008955058BB27AA270ED0E3
:10FAE000CBC1BCD130F0C1D120F031F49F3F11F433
:10FAF0001EF48CC10EF4E095E7FB82C1E92FCDD155
:10FB000080F3BA17620773078407950718F071F43A
:10FB10009EF5E5C10EF4E0950B2EBA2FA02D0B013A
:10FB2000B90190010C01CA01A0011124FF27591B42
:10FB300099F0593F50F4503E68F11A16F040A22F48
:10FB4000232F342F4427585FF3CF469537952795B9
:10FB5000A795F0405395C9F77EF41F16BA0B620BB8
:10FB6000730B840BBAF09150A1F0FF0FBB1F661FFF
:10FB7000771F881FC2F70EC0BA0F621F731F841F42
:10FB800048F4879577956795B795F7959E3F08F068
:10FB9000B3CF9395880F08F09927EE0F9795879527
:10FBA00008955CD158F080E891E009F49EEF5DD1B2
:10FBB00028F040E851E059F45EEF09C027C18FC139
:10FBC000E92FE0786AD168F3092E052AC1F32617D8
:10FBD00037074807590738F00E2E07F8E02569F077
:10FBE000E025E0640AC0EF6307F8009407FADB0140
:10FBF000B9019D01DC01CA01AD01EF9347D03CD1B1
:10FC00000AD05F91552331F02BED3FE049E450FDE0
:10FC100049EC63CF0895DF93DD27B92FBF7740E824
:10FC20005FE31616170648075B0710F4D92F5ED15D
:10FC30009F938F937F936F930FD2E0E2F1E0E9D02F
:10FC40001BD12F913F914F915F9163D1DD2349F0FB
:10FC50009058A2EA2AED3FE049EC5FE3D0785D27B7
:10FC60004DDFDF9109C1A8D008F481E008950CD0E0
:10FC700003C1FBD040F0F2D030F021F45F3F19F027
:10FC8000BFC051112DC1C2C008D198F39923C9F347
:10FC90005523B1F3951B550BBB27AA276217730792
:10FCA000840738F09F5F5F4F220F331F441FAA1F46
:10FCB000A9F333D00E2E3AF0E0E830D09150504006
:10FCC000E695001CCAF729D0FE2F27D0660F771FB4
:10FCD000881FBB1F261737074807AB07B0E809F096
:10FCE000BB0B802DBF01FF2793585F4F2AF09E3F2B
:10FCF000510568F085C0F4C05F3FECF3983EDCF33B
:10FD0000869577956795B795F7959F5FC9F7880FA3
:10FD1000911D9695879597F90895E1E0660F771FF5
:10FD2000881FBB1F621773078407BA0720F0621B86
:10FD3000730B840BBA0BEE1F88F7E0950895E894D7
:10FD400009C097FB3EF490958095709561957F4F23
:10FD50008F4F9F4F9923A9F0F92F96E9BB279395D1
:10FD6000F695879577956795B795F111F8CFFAF4E1
:10FD7000BB0F11F460FF1BC06F5F7F4F8F4F9F4F12
:10FD800016C0882311F096E911C0772321F09EE870
:10FD9000872F762F05C0662371F096E8862F70E0D6
:10FDA00060E02AF09A95660F771F881FDAF7880FB0
:10FDB0009695879597F90895990F0008550FAA0B06
:10FDC000E0E8FEEF16161706E807F907C0F012166E
:10FDD0001306E407F50798F0621B730B840B950B71
:10FDE00039F40A2661F0232B242B252B21F40895C6
:10FDF0000A2609F4A140A6958FEF811D811D089563
:10FE000097F99F6780E870E060E008959FEF80ECCD
:10FE10000895DF93CF931F930F93FF92EF92DF929A
:10FE20007B018C01689405C0DA2EEF0172D0FE01CF
:10FE3000E894A5912591359145915591AEF3EF0147
:10FE40005DDEFE019701A801DA9479F7DF90EF906B
:10FE5000FF900F911F91CF91DF91089500240A9494
:10FE60001616170618060906089500240A94121695
:10FE70001306140605060895092E0394000C11F4C8
:10FE8000882352F0BB0F40F4BF2B11F460FF04C075
:10FE90006F5F7F4F8F4F9F4F089557FD9058440FCE
:10FEA000551F59F05F3F71F04795880F97FB991FD9
:10FEB00061F09F3F79F08795089512161306140696
:10FEC000551FF2CF4695F1DF08C016161706180623
:10FED000991FF1CF86957105610508940895E894FE
:10FEE000BB2766277727CB0197F908959B01AC01C3
:10FEF00060E070E080E89FE3BACE0BD0BDCFAEDF0C
:10FF000028F0B3DF18F0952309F07ACF7FCF1124C2
:10FF1000E7CFC3DFA0F3959FD1F3950F50E0551FB6
:10FF2000629FF001729FBB27F00DB11D639FAA274E
:10FF3000F00DB11DAA1F649F6627B00DA11D661F9D
:10FF4000829F2227B00DA11D621F739FB00DA11DBE
:10FF5000621F839FA00D611D221F749F3327A00D78
:10FF6000611D231F849F600D211D822F762F6A2F14
:10FF700011249F5750408AF0E1F088234AF0EE0F99
:10FF8000FF1FBB1F661F771F881F91505040A9F7A6
:10FF90009E3F510570F034CFA3CF5F3FECF3983E06
:10FFA000DCF3869577956795B795F795E7959F5F0D
:10FFB000C1F7FE2B880F911D9695879597F90895A7
:10FFC000FA01EE0FFF1F30962105310599F16115F9
:10FFD000710561F48038BFE39B0749F1689490385C
:10FFE000810561F08038BFEF9B0741F0992342F50E
:10FFF000FF3FE1053105210511F1E8940894E795EB
:020000021000EC
:10000000D901AA2329F4AB2FBE2FF85FD0F310C07B
:10001000FF5F70F4A695E0F7F73950F019F0FF3A5A
:1000200038F49F779F930CD00F9007FC9058089559
:100030003EF0ECCE60E070E080E89FE308954FE78B
:100040009F775F934F933F932F9375D02F913F915D
:100050004F915F9152DF08C09B01AC014ECF19F464
:100060000EF0CECE3CCFD2CE20DFC8F39638C0F70C
:1000700007F80F92E8942BE33AEA48EB5FE74BDF8F
:100080000F920F920F924DB75EB70F9294D0EDE49E
:10009000F1E0BFDE4F915F91EF91FF91E595EE1F8B
:1000A000FF1F49F0FE57E0684427EE0F441FFA9502
:1000B000E1F74195550B06D00F9007FE17CF089535
:1000C0009FCEACC0F2DEE8F39923D9F3940F511D13
:1000D000BBF39150504094F059F0882332F0660FF2
:1000E000771F881F91505040C1F79E3F510544F73C
:1000F000880F911D9695879597F908955F3FACF00D
:10010000983E9CF0BB27869577956795B79508F440
:10011000B1609395C1F7BB0F58F711F460FFE8CFBA
:100120006F5F7F4F8F4F9F4FE3CFDACE0EF076C0D9
:100130006DCE689465CEB9DEC8F39923D1F3C6F3CA
:10014000DF93CF931F930F93FF92C92FDD2788234F
:100150002AF02197660F771F881FDAF720E030E03A
:1001600040E85FEB9FE3883920F0803E30F0219635
:100170008F77B3DCE5E7F1E003C0AFDCE2EAF1E062
:1001800048DE8B01BE01EC01FB2E6F57710975959E
:10019000771F880B990BD5DD28E132E741E35FE358
:1001A000B8DEAF2D9801AE01FF900F911F91CF9156
:1001B000DF91A4DC61CEFA01DC01AA0FBB1F9B0119
:1001C000AC01BF5728F422273327442750781FC09B
:1001D000B75188F4AB2F0024469537952795011C1D
:1001E000A395D2F3002069F0220F331F441FB3956B
:1001F000DAF30DD071CC61307105A0E88A07B946F9
:1002000030F49B01AC0166277727882790783096D9
:1002100021F0208331834283538308959F3F31F03F
:10022000915020F4879577956795B795880F911D24
:100230009695879597F90895629FD001739FF00175
:10024000829FE00DF11D649FE00DF11D929FF00D66
:10025000839FF00D749FF00D659FF00D9927729F9D
:10026000B00DE11DF91F639FB00DE11DF91FBD0128
:10027000CF0111240895AA1BBB1B51E107C0AA1F7F
:10028000BB1FA617B70710F0A61BB70B881F991F37
:100290005A95A9F780959095BC01CD01089597FBDB
:1002A000092E07260AD077FD04D0E5DF06D000200E
:1002B0001AF4709561957F4F0895F6F790958195A2
:1002C0009F4F0895A1E21A2EAA1BBB1BFD010DC072
:1002D000AA1FBB1FEE1FFF1FA217B307E407F507F6
:1002E00020F0A21BB30BE40BF50B661F771F881FD2
:1002F000991F1A9469F760957095809590959B0168
:10030000AC01BD01CF01089597FB092E05260ED043
:1003100057FD04D0D7DF0AD0001C38F45095409523
:10032000309521953F4F4F4F5F4F0895F6F79095C9
:100330008095709561957F4F8F4F9F4F08952F92B5
:100340003F924F925F926F927F928F929F92AF9265
:10035000BF92CF92DF92EF92FF920F931F93CF93B2
:10036000DF93CDB7DEB7CA1BDB0B0FB6F894DEBF49
:100370000FBECDBF09942A88398848885F846E846F
:100380007D848C849B84AA84B984C884DF80EE80B9
:10039000FD800C811B81AA81B981CE0FD11D0FB6C2
:1003A000F894DEBF0FBECDBFED010895AF92BF92AE
:1003B000CF92DF92EF92FF920F931F93CF93DF9331
:1003C000EC01688179818A819B81611571058105C4
:1003D000910521F464E279ED8BE597E02DE133EFAF
:1003E00041E050E00E94848179018A0127EA31E4EA
:1003F00040E050E00E941C815B016C01C801B70124
:100400002CEE34EF4FEF5FEF0E941C816A0D7B1DD5
:100410008C1D9D1D97FF04C0615070408040904826
:10042000688379838A839B837F77CB01DF91CF9128
:100430001F910F91FF90EF90DF90CF90BF90AF9002
:1004400008950E94D68108958DE297E00E94D6819A
:100450000895A0E0B0E080932D0790932E07A0931D
:100460002F07B093300708952F923F924F925F92DB
:100470007F928F929F92AF92BF92CF92DF92EF9234
:10048000FF920F931F93CF93DF934B01EA01611506
:10049000710519F0FB0180839183209739F09E014B
:1004A000225030402332310508F0F4C0A82EB92E76
:1004B000F50111915F017F01812F90E00E94698514
:1004C0000097B1F71D3229F4F50111917F0101E088
:1004D00006C01B3219F4F50111917F0100E020974D
:1004E00019F0C031D105B9F4103381F4F7018081DE
:1004F000883711F0883551F4F701118182E090E0DE
:10050000E80EF91E0260C0E1D0E005C0209719F4A2
:100510001033C1F422C0C830D105F9F0C930D1057B
:1005200024F4C230D10509F507C0CA30D10551F015
:10053000C031D105D1F427C0A12CB12CC12CF0E4DD
:10054000DF2E26C0CAE0D0E0ECECAE2EECECBE2EE6
:10055000ECECCE2EECE0DE2E1BC0C8E0D0E0A12CEF
:10056000B12CC12C70E1D72E13C09E01442737FD5A
:100570004095542F60E070E080E090E80E94628136
:1005800059016A0105C0A12CB12CC12C68E0D62EFE
:1005900040E060E070E0CB011E01442437FC409451
:1005A000542C50ED752E710EE72DEA3070F0212F8E
:1005B00021542A3118F439EC732E06C0212F21560C
:1005C0002A3130F529EA722E710E272D30E02C17D2
:1005D0003D07F4F447FD18C0A616B706C806D906AD
:1005E00080F0A20191010E941C81670D711D811D87
:1005F000911D6130F0E07F07F0E08F07F0E89F0782
:1006000010F04FEF01C041E0F70111917F01C9CF18
:100610008114910491F0442339F00894E108F10821
:10062000F401F182E08209C001FF1BC09701225052
:100630003040F4013183208314C047FF12C000FF13
:1006400005C060E070E080E090E804C06FEF7FEFED
:100650008FEF9FE722E230E030938D2E20938C2E97
:1006600016C000FF08C090958095709561957F4FEA
:100670008F4F9F4F0CC097FF0AC082E290E090938B
:100680008D2E80938C2E6FEF7FEF8FEF9FE79B0176
:10069000AC0103C020E030E0A901B901CA01DF913B
:1006A000CF911F910F91FF90EF90DF90CF90BF906F
:1006B000AF909F908F907F905F904F903F902F9042
:1006C00008952F923F924F925F926F927F929F92E6
:1006D000AF92BF92CF92DF92EF92FF920F931F9350
:1006E000CF93DF933B01EA016115710519F0FB011E
:1006F00080839183209739F09E012250304023322D
:10070000310508F0D5C0C82ED92EF60111916F0120
:100710007F01812F90E00E9469850097B1F71D321B
:1007200031F4F60111917F019924939406C01B3294
:1007300019F4F60111917F019924209719F0C03125
:10074000D105D1F4103389F4F7018081883711F095
:10075000883559F4F701118182E090E0E80EF91E26
:1007600092E0992AC0E1D0E007C0209729F4103325
:10077000B1F0CAE0D0E02BC0CA30D10541F1C031A0
:10078000D10521F0C830D105A9F409C02FEFA22E60
:100790002FEFB22E2FEFC22E2FE0D22E20C0C8E0B6
:1007A000D0E09FEFA92E9FEFB92E9FEFC92E9FE1BA
:1007B000D92E15C09E01442737FD4095542F6FEF69
:1007C0007FEFCB010E94628159016A0108C089E96B
:1007D000A82E89E9B82E89E9C82E89E1D82E60E0D3
:1007E00020E030E0A9011E01442437FC4094542C41
:1007F000012F00530A3060F0812F81548A3110F4A8
:10080000075006C0812F81568A3150F5012F0755B8
:10081000802F90E08C179D071CF56F3FE9F0A21622
:10082000B306C406D506A8F0CA01B901A201910118
:100830000E941C819B01AC01802F90E0A0E0B0E001
:10084000280F391F4A1F5B1F281739074A075B0704
:1008500010F46FEF01C061E0F70111917F01C8CF83
:100860006114710481F0662339F00894E108F108FD
:10087000F301F182E08207C091FE05C0C701029733
:10088000F3019183808390FE07C050954095309589
:1008900021953F4F4F4F5F4F67FF0DC082E290E0C1
:1008A00090938D2E80938C2E2FEF3FEFA90103C0E4
:1008B00020E030E0A901B901CA01DF91CF911F9179
:1008C0000F91FF90EF90DF90CF90BF90AF909F90EF
:1008D0007F906F905F904F903F902F900895662784
:1008E00077270C948787FC0188279927E894219122
:1008F0002032E9F3293010F02E30C8F32B3241F0CA
:100900002D3239F4689404C00E94DB85820F911D5A
:10091000219120532A30C0F31EF4909581959F4F6A
:100920000895283008F027E03327DA01990F311DA8
:1009300087FD916000966105710539F432602E5F84
:100940003D9330E32A95E1F708959F3F30F08038DA
:100950007105610509F03C5F3C5F3D93913008F003
:100960008068911DDF93CF931F930F93FF92EF92B7
:10097000192F987F9695E92F96959695E90FFF2761
:10098000EF5BFE4E99273327EE24FF24A701E701F2
:1009900005900894079428F4360FE71EF81E491FA7
:1009A000511D660F771F881F991F0694A1F70590A8
:1009B000079428F4E70EF81E491F561FC11D770F34
:1009C000881F991F661F0694A1F70590079428F4C5
:1009D000F80E491F561FC71FD11D880F991F661F8C
:1009E000771F0694A1F70590079420F4490F561F2E
:1009F000C71FD81F990F661F771F881F0694A9F776
:100A000084911095177041F0D695C79557954795E5
:100A1000F794E7941A95C1F7E7EEF0E16894159022
:100A2000159135916591959105907FE27395E11847
:100A3000F10A430B560BC90BD009C0F7E10CF11EAC
:100A4000431F561FC91FD01D7EF4703311F48A95C1
:100A5000E6CFE894015030F0080F0AF4002702179F
:100A600008F4202F2395022F7A3328F079E37D9321
:100A70002A95E9F710C07D932A9589F606949795F3
:100A80006795379517951794E118F10A430B560BA4
:100A9000C90BD00998F023957E9173957A3308F0AD
:100AA00070E37C932013B8F77E9170617D9330F0F2
:100AB000839571E37D9370E32A95E1F71124EF901C
:100AC000FF900F911F91CF91DF91992787FD90950E
:100AD00008959111AAC3803219F089508550D0F73A
:100AE0000895FC010590615070400110D8F7809581
:100AF00090958E0F9F1F08954EE558E10E94B48592
:100B00000895FB01DC0102C001900D92415050405C
:100B1000D8F70895DC0101C06D9341505040E0F7D3
:100B20000895FB01DC018D91019080190110D9F32A
:100B3000990B0895FB01DC014150504048F00190B1
:100B40000D920020C9F701C01D9241505040E0F7BE
:100B50000895FC016150704001900110D8F7809514
:100B600090958E0F9F1F0895FA01A191B081009773
:100B700019F41097E1F0CD01DC01CD010D900020BA
:100B800011F4C00113C0FB012191222319F020159B
:100B9000D9F7F3CFFB012191201519F41E9211967C
:100BA00006C02223C1F70D900020A1F7D001FA0161
:100BB000A193B08308957AE0979F902D879F802D11
:100BC000910D112408950F931F93CF93DF938C0100
:100BD000EB018B8181FF1BC082FF0DC02E813F8105
:100BE0008C819D812817390764F4E881F98101938C
:100BF000F983E88306C0E885F985802F0995009779
:100C000031F48E819F8101969F838E8302C00FEF06
:100C10001FEFC801DF91CF911F910F910895DF93CE
:100C2000CF93CDB7DEB7FE0135966191719180917A
:100C3000882E9091892EAF010E94BD79CF91DF91CE
:100C40000895DF93CF93CDB7DEB7FE01359661915E
:100C500071918091882E9091892EDC0113962C91B0
:100C60001397286013962C93AF010E94BD79E091F1
:100C7000882EF091892E2381277F2383CF91DF91C6
:100C80000895EF92FF920F931F93CF93DF938C0100
:100C9000E091882EF091892E838181FF1FC0C0E0F2
:100CA000D0E00AC0DB011896ED91FC9119970995E7
:100CB000009711F0CFEFDFEFF80181918F01609184
:100CC000882E7091892E882369F7DB011896ED91A3
:100CD000FC9119978AE00995009711F0CFEFDFEFAB
:100CE000CE01DF91CF911F910F91FF90EF9008956A
:100CF0000F931F93DF93CF93CDB7DEB72E970FB629
:100D0000F894DEBF0FBECDBF0D891E898F89988DE7
:100D100026E02C831A83098397FF02C080E090E8C5
:100D200001979E838D839E01255E3F4FCE010196E4
:100D3000698D7A8DA9010E94BD794D815E8157FD33
:100D40000AC02F813885421753070CF49A01020F0D
:100D5000131FF80110822E960FB6F894DEBF0FBE57
:100D6000CDBFCF91DF911F910F9108950F931F93E6
:100D7000DF93CF93CDB7DEB72E970FB6F894DEBFD3
:100D80000FBECDBF8C01CB01BA0146E04C831A8364
:100D9000098397FF02C080E090E801979E838D83CE
:100DA000CE010196A9010E94BD794D815E8157FD5A
:100DB0000AC02F813885421753070CF49A01020F9D
:100DC000131FF80110822E960FB6F894DEBF0FBEE7
:100DD000CDBFCF91DF911F910F910895FA01AA27FE
:100DE000283051F1203181F1E8946F936E7F6E5F6E
:100DF0007F4F8F4F9F4FAF4FB1E03ED0B4E03CD01C
:100E0000670F781F891F9A1FA11D680F791F8A1FFE
:100E1000911DA11D6A0F711D811D911DA11D20D065
:100E200009F468943F912AE0269F11243019305D1F
:100E30003193DEF6CF010895462F4770405D419310
:100E4000B3E00FD0C9F7F6CF462F4F70405D4A335D
:100E500018F0495D31FD4052419302D0A9F7EACF25
:100E6000B4E0A6959795879577956795BA95C9F754
:100E700000976105710508959B01AC010A2E069447
:100E80005795479537952795BA95C9F7620F731F00
:100E9000841F951FA01D0895DC01CB01FC01F99969
:100EA000FECF06C0F2BDE1BDF89A319600B40D92B6
:100EB00041505040B8F70895F999FECF92BD81BDD9
:100EC000F89A992780B50895A8E1B0E042E050E093
:100ED0000C944E87DC01CB0103C02D910E947587D5
:100EE00041505040D0F70895262FF999FECF1FBAF0
:100EF00092BD81BD20BD0FB6F894FA9AF99A0FBE43
:100F0000019608950E947487272F0C9475876F921D
:100F10007F928F929F92AF92BF92CF92DF92EF9289
:100F2000FF920F931F93DF93CF930F92CDB7DEB74E
:100F30005B016115710521F0DB018C9311969C9387
:100F4000482F592F6A01F601E1906F018F018E2D14
:100F500090E00E9469850097B1F7FE2DFD3229F4DB
:100F6000D601ED908D0121E007C0BE2DBB3219F4F2
:100F7000F601E1908F0120E068010894C108D108D2
:100F8000C60161EE71E143E050E029830E941889B7
:100F90002981009711F572E0E72EF12CE00EF11E89
:100FA000C70164EE71E145E050E00E941889298193
:100FB000009729F467E0E62EF12CE00EF11EA11453
:100FC000B10421F0D5011196FC92EE9220FF0FC1E1
:100FD00030E020E090E88FEF12C1C60169EE71E1C8
:100FE00043E050E029830E9418892981009731F05D
:100FF00060E070E0CB01662477240AC0A114B1043C
:1010000009F4F9C00E5F1F4FF50111830083F3C08F
:101010003E2D30533A30A0F52260E22FF0E0AF01D0
:101020004870507022FF07C04115510571F50894B2
:10103000611C711C2AC04115510519F00894610802
:1010400071086B017C0152E0CC0CDD1CEE1CFF1C16
:101050005A95D1F76C0D7D1D8E1D9F1D660F771F54
:10106000881F991F630F711D811D911D6839F9E952
:101070007F07F9E98F07F9E19F0738F0246005C081
:101080003E3F39F423FD3FC02860D801ED908D012B
:10109000BFCF353311F03531B1F5F80131913D3223
:1010A00011F4206102C03B3241F4D80111963C9109
:1010B0001197319642E050E002C041E050E03053D9
:1010C0003A3020F08F01041B150B1DC040E050E0AA
:1010D000BCE040385B075CF4DA01AA0FBB1FAA0F23
:1010E000BB1F4A0F5B1F440F551F430F511D31910A
:1010F00030538F013A3060F324FF03C0509541957F
:101100005F4F640E751EC22EDD2421FF08C0A1149E
:10111000B10429F001501040F501118300830E94B1
:101120009F7E7B018C01F3E0CF22DD2433E0C316E8
:10113000D10421F417FB109517F91095C801B701D8
:1011400020E030E0A9010E94337E882309F44AC0E0
:1011500077FE09C040E0C42E42E1D42E7094619421
:101160007108739404C038E1C32E32E1D32E26E017
:10117000822E912C90E2A92EB12C0FC0F601259160
:10118000359145915491C801B7010E947D7FE62EAB
:10119000F72E082F192F6A187B086A147B0474F73E
:1011A000B594A7940894810891088114910429F0BA
:1011B0008CEF9FEFC80ED91EF0CFB701C801282FC2
:1011C000220F292F221F2F3F39F020E030E0A90104
:1011D0000E94337E882331F482E290E090938D2E3A
:1011E00080938C2E3E2D2F2D902F812F08C030E024
:1011F00020E090E803C030E020E090EC8FE7F901B8
:10120000AC016F2F722F852F942F0F90CF91DF910C
:101210001F910F91FF90EF90DF90CF90BF90AF9014
:101220009F908F907F906F900895992788270895B9
:10123000FB01DC014150504088F08D9181341CF05D
:101240008B350CF4805E659161341CF06B350CF4C9
:10125000605E861B611171F3990B0895881BFCCFAA
:04126000F894FFCF30
:1012640054696D656F757420414444523D252D6465
:101274002E252D64205345513D252D642052535372
:10128400493D252D75204C51493D252D750A0026D3
:101294003A202573205B414444523D252D642E257C
:1012A4002D64205345513D252D642054544C3D2537
:1012B4002D7520525353493D252D75204C51493DE0
:1012C400252D75204452503D252D642E2530326441
:1012D4005D0A00523D252D75204C3D252D7520536A
:1012E4003D252D642000284578745077722900002C
:1012F40065756936343D0025303278002530327802
:101304000A00736E3D00413A20256420256420259F
:1013140064200A00433A20256420256420256420A3
:10132400613D25352E31660A007374617475733D11
:101334003078253032780A20006669726D776172E0
:10134400653D53322D352E302D323031342D303130
:101354002D323800656570726F6D006F6E006F66B8
:1013640066006131007265736574006E6F6E6500AE
:10137400613200765F696E0073746174730074780F
:10138400743D25730A003100320033003400350007
:101394003600636820706B74730025327520252D28
:1013A4003130750A006175746F00666C757368007E
:1013B4004455503D252D6420414444523D252D641F
:1013C4002E252D64205345513D252D642054544C25
:1013D4003D252D752F252D7520525353493D252D1F
:1013E400752F252D75204C51493D252D750A006416
:1013F40065657000666F7263655F69646C6500742F
:1014040072696D00746573740043683D252D642012
:1014140054785077723D252D640A004572726F72BC
:10142400205458204C656E6774683D25640A005446
:1014340058543D2573200049443D004536343D0051
:101444002050533D25640020543D252D362E326610
:10145400002054313D252D362E32660020545F4D38
:1014640043553D252D352E31660020565F4D43559D
:101474003D252D342E3266002050303D252D6C58EC
:10148400002050305F543D252D372E336600205008
:10149400313D252D6C58002050315F543D252D37AA
:1014A4002E3366002055503D252D6C58002052489F
:1014B4003D252D342E31660020565F494E3D252DA5
:1014C400352E32660020565F41313D252D352E32B2
:1014D400660020565F41323D252D352E32660020B0
:1014E400565F41333D252D352E30660020565F4131
:1014F40044313D252D382E36660020565F41443256
:101504003D252D382E36660020565F4144333D2557
:101514002D382E36660020565F4144343D252D3843
:101524002E36660020503D252D6C64002050413D30
:10153400252D372E326600263A2025730A0054588A
:1015440020706B74206C656E203D2025640A0001B8
:1015540000D734EF3C22FFCC3B22FFCC3B1A2009BE
:101564000D00FE046162636465666768696A6B6C9A
:101574006D6E6F704C2801003C000A401A0F636DB9
:10158400642070726F636573730000001E05223A55
:1015940000000000737464696E2070726F63657379
:1015A40073000000340502110000000062726F61D4
:1015B40064636173742070726F63657373000000F9
:1015C4004C05023B00000000536C6565702070728E
:1015D4006F636573730000006805F4110000000078
:1015E400506572696F6469632070726F63657373A9
:1015F40000000080050D19000000002A0542055E68
:1016040005910576050000C30900001F004000682D
:1016140007A80710000000B044A4441810000000FC
:10162400004576656E742074696D6572000000C1B2
:1016340005BB48000000004374696D657220707238
:101644006F63657373000000D705F949000000005B
:10165400020306070A0B0E0F020306070A0B0E0FFE
:101664002843292032303132204865726A756C660D
:101674000055747665636B6C696E672020202020AA
:101684002000436F6E74696B6920322E35000000B0
:10169400000200000000345800000000C600C5002D
:1016A400C400C100C200000000CE00CD00CC00C9BF
:1016B40000CA00000000524632333020647269765A
:1016C40065720000005606EB5C000000005C5BDA0B
:1016D4005A3A5D845EFD5B8D5AFB58F5587C5ADEA0
:1016E400590001010101010101010101010101018F
:1016F400010052696D65009206EF60B66061646135
:1017040074612E6E756D20776179206F7574207405
:10171400686572653A2025640A00316230623A6471
:101724006965A1630080C0E0F0F8FCFEFF6E756C93
:101734006C6D616300CD061C66016607660D661359
:10174400661966736963736C6F776D616300E30692
:101754003D679E6634661D6623663166BA000800DE
:10176400E711EF1135000200BF17C1175443502F82
:10177400495020737461636B0000000C0797690083
:101784000000000208FFFFFFFF000000000100004E
:02179400000053
:00000001FF
